:100000000C94692E0C949A2E0C949A2E0C949A2E81
:100010000C949A2E0C9400690C949A2E0C949A2E9F
:100020000C9481680C949A2E0C949A2E0C94D0CA3D
:100030000C949A2E0D9459BC0C949A2E0C949A2ED2
:100040000C949A2E0D94BB1E0C949A2E0C949A2EFE
:100050000C949A2E0C949A2E0D9423350D9480B402
:100060000C949A2E0C9443400C949A2E0C949A2E35
:100070000C949A2E0C949A2E0C949A2E0C949A2EE0
:100080000C949A2E0C949A2E0C949A2E0C949A2ED0
:100090000C949A2E0C949A2E0C949A2E0C949A2EC0
:1000A0000C949A2E0C949A2E0C949A2E0C949A2EB0
:1000B0000C949A2E0C949A2E0C949A2E0C949A2EA0
:1000C0000C949A2E0C949A2E0C949A2E0C94834095
:1000D0000C949A2E0C949A2E0C949A2E0C949A2E80
:1000E0000C949A2E463F4A3F4F3F573F6C3F853F07
:1000F000AA3FD43F4F016B017B010D024301710107
:100100009F01E701DF017901D301DD015F016D018D
:1001100057017D01AB01B9019B01CB0161010302D4
:10012000F301D7013B010B02070209029301890188
:1001300087010502630137016901FF01BF01D10198
:10014000B301B301B301F101F101F10139014B0137
:10015000F1013D0195019901C3016F01D90101022E
:1001600055015D01CF01D501A101B501A701C10173
:1001700001024901A50165010F025901A301CD0149
:1001800013028B018101F501EF0191014D01350150
:100190003F0183018B01C701BB01F701084AD73B2F
:1001A0003BCE016E84BCBFFDC12F3D6C74319ABD46
:1001B00056833DDA3D00C77F11BED9E4BB4C3E916A
:1001C0006BAAAABE000000803F05A84CCDB2D44E59
:1001D000B93836A9020C50B9918688083CA6AAAA5B
:1001E0002ABE000000803F07634236B79BD8A71A9B
:1001F00039685618AEBAAB558C1D3CB7CC5763BDA9
:100200006DEDFD753EF6177231BF000000803F08AE
:10021000000000BE922449123EABAAAA2ABECDCC51
:10022000CC4C3E00000080BEABAAAAAA3E00000053
:1002300000BF000000803F0000000000084178D3AC
:10024000BB4387D1133D190E3CC3BD4282AD2B3E4B
:1002500068EC8276BED98FE1A93E4C80EFFFBE01EB
:10026000C4FF7F3F0000000000000D9499B60D947C
:1002700026840D94AD840D94A2820D94B7840D94C0
:100280009DB60D94B29C0D94FA350D941EA20D945A
:1002900086650D943AB60D94DB840D9493B60D9457
:1002A000A8350D9413910D9414700D94E9B50D9427
:1002B00084360D947DB60D94E7780D94F1B50D94C8
:1002C00056360D948B6C0D9415840D944EB60D948A
:1002D000A8680D9443840D94B6350D9464360D943E
:1002E000D5B50D9408360D948D680D9455470D9431
:1002F000AA450D942C360D94D2350D941A6C0D949C
:100300006E580D9481B60D94A1B60D944BB70D9413
:100310002B830D940E830D94B4B60D94904C0D94D4
:1003200046470D948FB60D94FA820D94C1B50D9485
:10033000355D0D94C6B50D94616C0D949F680D9458
:1003400022360D940DB60D946CB60D9444B60D94F2
:1003500026B60D9423530D942F6C0D94E5570D94F0
:1003600074AA0D9421670D94A5840D9417B60D946D
:10037000A76B0D94476C0D94ABB60D949D210D9415
:1003800095840D9430B60D94CBB50D9452690D94AF
:10039000A7B60D9449A50D94866C0D9470B60D9476
:1003A000F9B50D949D840D942E360D9403B60D94DD
:1003B000C46C0D94DFB50D942A490D943C360D9410
:1003C00028360D940B440D94EA970D94B7450D947F
:1003D00026360D9402990D94E8520D9496680D946A
:1003E0008BB60D94CB840D94AF6C0D9485B60D94A3
:1003F000AFB60D94795B0D948D420D947E6A0D9489
:100400006C840D9458B60D94956C0D94F3830D94F3
:10041000D1820D94E6820D94BA820D94E0350D944C
:100420007AB60D945B470D9476B60D944C73486183
:100430007264636F6465642044656661756C7420E2
:1004400053657474696E6773204C6F6164656400F2
:1004500053746F7265642073657474696E6773207A
:1004600072657472696576656400202020452F44AA
:10047000203D20002020204D393030204B004C6999
:100480006E65617220616476616E63652073657468
:1004900074696E67733A0046696C616D656E7420AD
:1004A00073657474696E67733A2044697361626C32
:1004B0006564002020204D32303020440046696CB5
:1004C000616D656E742073657474696E67733A004C
:1004D0002020204D3230392053004175746F2D5249
:1004E0006574726163743A20533D3020746F2064E8
:1004F000697361626C652C203120746F20696E74A1
:1005000065727072657420657874727564652D6F9C
:100510006E6C79206D6F76657320617320726574DF
:100520007261637473206F72207265636F76657297
:10053000696573002046002020204D32303820535A
:10054000005265636F7665723A20533D4578747248
:1005500061206C656E67746820286D6D2920463AAD
:10056000537065656420286D6D2F6D2900205A0039
:100570002046002020204D32303720530052657431
:10058000726163743A20533D4C656E67746820282D
:100590006D6D2920463A537065656420286D6D2F76
:1005A0006D29205A3A205A4C69667420286D6D29AD
:1005B000002044002049002020204D3330342050BA
:1005C00000504944206865617462656420736574F5
:1005D00074696E67733A002044002049002020208F
:1005E0004D33303120500050494420736574746994
:1005F0006E67733A00205A0020590020204D323097
:1006000036205800486F6D65206F666673657420EC
:10061000286D6D293A00204500205A0020590020FD
:10062000580020420020540020204D323035205305
:1006300000416476616E636564207661726961620F
:100640006C65733A20533D4D696E20666565647232
:1006500061746520286D6D2F73292C20543D4D69E0
:100660006E2074726176656C206665656472617473
:100670006520286D6D2F73292C20423D6D696E69B0
:100680006D756D207365676D656E742074696D6539
:1006900020286D73292C20583D6D6178696D756D2A
:1006A000205859206A65726B20286D6D2F73292C94
:1006B00020205A3D6D6178696D756D205A206A65FC
:1006C000726B20286D6D2F73292C2020453D6D61A4
:1006D00078696D756D2045206A65726B20286D6D97
:1006E0002F73290020540020204D32303420530035
:1006F000416363656C65726174696F6E3A20533D46
:10070000616363656C65726174696F6E2C20543D22
:100710007265747261637420616363656C65726194
:1007200074696F6E00204500205A00205900202077
:100730004D3230312058004D6178696D756D204122
:100740006363656C65726174696F6E20286D6D2FCF
:100750007332293A00204500205A002059002020F9
:100760004D3230332058004D6178696D756D2066CB
:10077000656564726174657320286D6D2F73293A05
:1007800000204500205A0020590020204D393220F9
:10079000580053746570732070657220756E6974AB
:1007A0003A0053657474696E67732053746F726591
:1007B0006400454550524F4D204572726F72004D96
:1007C0006561737375726520617667203D202564CD
:1007D0000A004432313330202D20544D433231331E
:1007E000300A0074656D705F70696E64613D2564E8
:1007F000206F66667365745F7A3D25642E253033FD
:10080000640A0074656D705F70696E64613D256493
:10081000432074656D705F73686966743D25647507
:100820006D0A0063616C5F7374617475733D256458
:100830000A004438202D20526561642F5772697474
:10084000652050494E44410A000020006D657368E0
:1008500020626564206C6576656C696E673A20007D
:1008600029002C20002C2000706879736963616C6A
:1008700020636F6F7264696E617465733A2028003B
:1008800029002C20002C2000776F726C6420636F8D
:100890006F7264696E617465733A202800204600A7
:1008A0002045004731205A004D3234004D32362069
:1008B00053256C75004D31303620530047312046AA
:1008C0002564004731204531204634383000473117
:1008D000205A002046323030300020590047312065
:1008E00058004D383300506F736974696F6E207211
:1008F0006561642066726F6D20656570726F6D3A18
:10090000004D3233202573002E67636F0046656506
:1009100064726174653A007265636F7665725F6DCB
:10092000616368696E655F73746174655F61667445
:1009300065725F706F7765725F70616E69632C209E
:10094000696E697469616C20007265636F766572A7
:100950005F6D616368696E655F73746174655F6123
:10096000667465725F706F7765725F70616E6963E0
:100970002C20696E697469616C20007265636F7602
:1009800065725F6D616368696E655F7374617465DC
:100990005F61667465725F706F7765725F70616EBC
:1009A00069632C20696E697469616C2000637572DB
:1009B00072656E745F706F736974696F6E5B5A5F96
:1009C000415849535D3A0043757272656E742070E8
:1009D0006F736974696F6E20595F415849533A00CB
:1009E00043757272656E7420706F736974696F6E8F
:1009F00020585F415849533A004166746572207728
:100A0000616974696E6720666F722074656D703AF3
:100A1000004739322045004D383200473120452DFE
:100A200031204634383000473120453520463132B8
:100A300030004D3833004D31393020532564004D9E
:100A4000313039205325640047323820582059006E
:100A50004731205A32352046383030004D3134305D
:100A600020532564004D3130342053256400494E15
:100A700054340055564C4F202D20656E640073741D
:100A800070730055564C4F0020423A0020453A0002
:100A9000543A005A206C6976652061646A757374F3
:100AA000206F7574206F662072616E67652E20530B
:100AB000657474696E6720746F20302E20436C69F2
:100AC000636B20746F20636F6E74696E75652E00A2
:100AD0005A206C6976652061646A757374206F753D
:100AE00074206F662072616E67652E205365747482
:100AF000696E6720746F20300020573A0020453A15
:100B000000543A004B494C4C3A20004175746F0038
:100B100020452F443D00416476616E6365204B3D66
:100B20000022283229005400496E76616C696420E5
:100B30005420636F64652E00496E76616C69642091
:100B40004D20636F64652E004D323230205325698D
:100B500000203A2000004C414E472053454C20468F
:100B60004F5243454400222831290020453A0020B5
:100B70005A3A0020593A0020453A00205A3A0020BB
:100B8000593A00583A004D31313320530020002E9D
:100B90000020423A0020453A00543A0020413A00F1
:100BA00020503A002042403A0020403A00202F00D6
:100BB0003A00205400202F0020423A00202F006FDE
:100BC0006B20543A002569206D696E2C2025692020
:100BD00073656300496E76616C6964204D20636FB4
:100BE0006465004D65736820626564206C65766598
:100BF0006C696E67206E6F74206163746976652E10
:100C0000000A002020000A4D65617375726564203A
:100C1000706F696E74733A000A5A2073656172636B
:100C200068206865696768743A20002C004E756D0D
:100C300020582C593A2000476F20686F6D65206658
:100C4000696E6973686564004D65736820626564E8
:100C5000206C6576656C696E672061637469766186
:100C600074656400557073616D706C652066696EA3
:100C7000697368656400426564206C6576656C69BB
:100C80006E6720636F7272656374696F6E20666948
:100C90006E697368656400206D6963726F6E7300BE
:100CA00045786365737369766520626564206C6559
:100CB00076656C696E6720636F7272656374696FC5
:100CC0006E3A2000626162797374657020617070A1
:100CD0006C69656400636C65616E2075702066697F
:100CE0006E6973686564200000206F6666736574C2
:100CF0003A20006D65736820626564206C657665D6
:100D00006C696E673A2000473238205730003A202D
:100D10000054656D70657261747572652063616CF5
:100D20006962726174696F6E20646F6E652E204314
:100D30006F6E74696E75652077697468207072656E
:100D40007373696E6720746865206B6E6F622E0026
:100D500000205A20736869667420286D6D293A0056
:100D600050494E44412074656D70657261747572AE
:100D7000653A2000002F3600537465703A20000059
:100D8000205A20736869667420286D6D293A0050D6
:100D9000494E44412074656D706572617475726569
:100DA0003A20002F362028736B6970706564290023
:100DB000537465703A2000005A45524F3A200000A3
:100DC00073746172742074656D706572617475728C
:100DD000653A200050494E44412070726F62652090
:100DE00063616C6962726174696F6E2073746172A1
:100DF0007400473238205730000A00205A3A200049
:100E000020593A200020583A20004732382C2066DA
:100E1000696E616C20004732382C2066696E616C07
:100E200020004732382C2066696E616C2000473202
:100E3000382C20696E697469616C20004732382C47
:100E400020696E697469616C200043524153485FA8
:100E50004445544543544544004D3239006275734E
:100E6000793A2070617573656420666F7220696ECF
:100E700070757400627573793A207061757365647A
:100E800020666F72207573657200627573793A20FF
:100E900070726F63657373696E67002055706C6F55
:100EA000616420696E2070726F6772657373006988
:100EB0006E697469616C207A737465707320616601
:100EC0007465722072657365743A2000696E697486
:100ED00069616C207A7374657073206F6E20706F17
:100EE0007765722075703A2000466163746F72797D
:100EF0002052455345540044495341424C45440A0D
:100F000000454E41424C45440A004653656E736F9E
:100F1000722000504154393132355F696E69743A3C
:100F200025640A004E6F7620323920323031370086
:100F3000436F6D70696C65643A2000286E6F6E6552
:100F40002C2064656661756C7420636F6E666967DA
:100F500029004E6F76203239203230313720303040
:100F60003A31303A3338007374617274001B5B326B
:100F70004A1B5B313B31484F726967696E616C2077
:100F800050727573612069331B5B323B334850727A
:100F90007573612052657365617263680025002076
:100FA0002020202020002020202020200045524109
:100FB00053494E4720616C6C206461746100466146
:100FC00063746F7279205245534554004352415324
:100FD000485F5245434F564552004732382059002A
:100FE000473238205800FFFFFF0000A0400000A05B
:100FF000400000004000007F43000056439AD95152
:101000004300000000000080C09A99193E00007F54
:1010100043000052430000524300000000000080E3
:10102000C09A99193E6563686F3A004572726F7293
:101030003A0000002110422063308440A550C66071
:10104000E770088129914AA16BB18CC1ADD1CEE185
:10105000EFF13112100273325222B5529442F772FC
:10106000D662399318837BB35AA3BDD39CC3FFF3D5
:10107000DEE36224433420040114E664C774A4440C
:1010800085546AA54BB528850995EEE5CFF5ACC525
:101090008DD55336722611163006D776F6669556DC
:1010A000B4465BB77AA719973887DFF7FEE79DD775
:1010B000BCC7C448E5588668A7784008611802286C
:1010C0002338CCC9EDD98EE9AFF9488969990AA9C5
:1010D0002BB9F55AD44AB77A966A711A500A333A3C
:1010E000122AFDDBDCCBBFFB9EEB799B588B3BBB15
:1010F0001AABA66C877CE44CC55C222C033C600CCC
:10110000411CAEED8FFDECCDCDDD2AAD0BBD688D64
:10111000499D977EB66ED55EF44E133E322E511E1B
:10112000700E9FFFBEEFDDDFFCCF1BBF3AAF599FB4
:10113000788F8891A981CAB1EBA10CD12DC14EF154
:101140006FE18010A100C230E320045025404670BA
:101150006760B9839893FBA3DAB33DC31CD37FE3E5
:101160005EF3B1029012F322D2323542145277620A
:101170005672EAB5CBA5A89589856EF54FE52CD5B5
:101180000DC5E234C324A01481046674476424545A
:101190000544DBA7FAB79987B8975FE77EF71DC7C5
:1011A0003CD7D326F2369106B016576676761546AA
:1011B00034564CD96DC90EF92FE9C899E9898AB915
:1011C000ABA94458654806782768C018E1088238FA
:1011D000A3287DCB5CDB3FEB1EFBF98BD89BBBAB25
:1011E0009ABB754A545A376A167AF10AD01AB32A4A
:1011F000923A2EFD0FED6CDD4DCDAABD8BADE89D75
:10120000C98D267C076C645C454CA23C832CE01C99
:10121000C10C1FEF3EFF5DCF7CDF9BAFBABFD98F04
:10122000F89F176E367E554E745E932EB23ED10EE9
:10123000F01E7C3C3E5E2B3D3F2F5B5D3B2C2A220B
:101240005C004D383420582059205A2045004D323A
:1012500034004D3233202573006175746F25692E7B
:1012600067000A002F000A002E0044656C6574694F
:101270006F6E206661696C65642C2046696C653A06
:10128000200046696C652064656C657465643A008D
:101290002E002E002E002E004E6F77206672657392
:1012A000682066696C653A20004E6F7720646F692C
:1012B0006E672066696C653A20002220706F7300AB
:1012C0002220706172656E743A2200535542524F6B
:1012D0005554494E452043414C4C2074617267651A
:1012E000743A2200747279696E6720746F206361AA
:1012F0006C6C207375622D67636F64652066696C22
:101300006573207769746820746F6F206D616E79E2
:10131000206C6576656C732E204D4158206C657687
:10132000656C2069733A00256920686F75727320B7
:101330002569206D696E757465730054494D454F7C
:1013400055543A004D3131300046756C6C2052587E
:10135000204275666665720022206661696C65646C
:101360003A204275666665722066756C6C21004590
:101370006E717565696E6720746F2074686520668C
:10138000726F6E743A2022002200456E7175656995
:101390006E6720746F207468652066726F6E743A91
:1013A00020220022206661696C65643A20427566DD
:1013B0006665722066756C6C210022004D363030F7
:1013C000006673656E736F725F64697361626C65EA
:1013D0000A00504154393132355F696E69743A25DB
:1013E000640A006673656E736F725F656E61626C2E
:1013F000650A005072757361206933204D4B3320AC
:101400006F6B005072757361206933204D4B332030
:1014100072656164792E007A5F6D696E3A20007A98
:101420005F6D61783A20005A204F666673657400DC
:10143000795F6D696E3A2000795F6D61783A2000BE
:101440005920767A64616C656E6F7374206F6420C6
:101450006D696E3A00592064697374616E6365202A
:1014600066726F6D206D696E3A00416E6F0059654E
:101470007300785F6D696E3A2000785F6D61783A2D
:10148000200044657461696C792058595A206B6159
:101490006C2E0058595A2063616C2E20646574616B
:1014A000696C73004E796E692070726F7665647531
:1014B000207A206B616C6962726163692E00492039
:1014C00077696C6C2072756E207A2063616C69623A
:1014D000726174696F6E206E6F772E004E796E693F
:1014E0002070726F766564752078797A206B616CF4
:1014F0006962726163692E205A6162657265207447
:101500006F20707269626C697A6E65203132206D6D
:10151000696E2E00492077696C6C2072756E207898
:10152000797A2063616C6962726174696F6E206E92
:101530006F772E2049742077696C6C2074616B651D
:1015400020617070726F782E203132206D696E7359
:101550002E004E796E692070726564656872656AE6
:101560006920747279736B752070726F20504C41D2
:101570002E004E6F7720492077696C6C2070726561
:1015800068656174206E6F7A7A6C6520666F722070
:10159000504C412E00446F6272792064656E2C209D
:1015A0006A73656D2076617365207469736B61720F
:1015B0006E61204F726967696E616C20507275733D
:1015C000612069332E204368636574652061627908
:1015D0006368205661732070726F7665646C612059
:1015E0006B616C69627261636E696D2070726F63AA
:1015F0006573656D3F0048692C204920616D207935
:101600006F7572204F726967696E616C20507275D8
:101610007361206933207072696E7465722E205771
:101620006F756C6420796F75206C696B65206D65D2
:1016300020746F20677569646520796F7520746800
:10164000726F7567682074686520736574757020A3
:1016500070726F636573733F005A61636E752074B7
:1016600069736B6E6F7574206C696E6B7520612089
:1016700056792062756465746520706F7374757037
:101680006E6520736E697A6F7661742074727973F7
:101690006B75206F746163656E696D20746C616336
:1016A00069746B6120646F6B7564206E65646F7321
:1016B00061686E657465206F7074696D616C6E69C8
:1016C000207679736B792E2050726F686C65646E2A
:1016D000657465207369206F6272617A6B79207618
:1016E000206E61736920707269727563636520761C
:1016F000206B617069746F6C65204B616C696272FC
:1017000061636500492077696C6C20737461727441
:1017100020746F207072696E74206C696E65206130
:101720006E6420796F752077696C6C2067726164D4
:1017300075616C6C79206C6F7765722074686520B8
:101740006E6F7A7A6C6520627920726F7461746949
:101750006E6720746865206B6E6F622C20756E74E6
:10176000696C20796F75207265616368206F707491
:10177000696D616C206865696768742E20436865CF
:10178000636B20746865207069637475726573207B
:10179000696E206F75722068616E64626F6F6B2076
:1017A000696E20636861707465722043616C696260
:1017B000726174696F6E2E004E796E69207A6B616A
:1017C0006C696272756A6920767A64616C656E6FA5
:1017D0007374206D657A69206B6F6E63656D20741C
:1017E0007279736B79206120706F76726368656DB2
:1017F0002068656174626564752E004E6F772049BC
:101800002077696C6C2063616C6962726174652019
:1018100064697374616E6365206265747765656E73
:1018200020746970206F6620746865206E6F7A7A04
:101830006C6520616E642068656174626564207304
:101840007572666163652E004E656A647269762002
:10185000706F6D6F63692073656C66746573747502
:10186000207A6B6F6E746F6C756A69206E656A633F
:10187000617374656A736920636879627920767A26
:101880006E696B616A696369207072692073657340
:10189000746176656E69207469736B61726E792EFE
:1018A0000046697273742C20492077696C6C207231
:1018B000756E207468652073656C6674657374203A
:1018C000746F20636865636B206D6F737420636F42
:1018D0006D6D6F6E20617373656D626C79207072CF
:1018E0006F626C656D732E005370757374656E69ED
:1018F0002057697A617264612076796D617A65201A
:10190000756C6F7A656E65207679736C65646B793A
:10191000207673656368206B616C696272616369CC
:10192000206120737075737469206B616C696272D9
:1019300061636E692070726F636573206F64207AD3
:10194000616361746B752E20506F6B7261636F768B
:1019500061743F0052756E6E696E672057697A61D7
:1019600072642077696C6C2064656C6574652063B3
:10197000757272656E742063616C696272617469FC
:101980006F6E20726573756C747320616E64207362
:10199000746172742066726F6D2074686520626570
:1019A00067696E6E696E672E20436F6E74696E751F
:1019B000653F00436863657465206F70616B6F7687
:1019C000617420706F736C65646E69206B726F6BED
:1019D000206120706F7A6D656E697420767A64611B
:1019E0006C656E6F7374206D657A6920747279739B
:1019F0006B6F75206120686561746265643F0044A7
:101A00006F20796F752077616E7420746F20726516
:101A100070656174206C61737420737465702074D8
:101A20006F20726561646A75737420646973746190
:101A30006E6365206265747765656E206E6F7A7A75
:101A40006C6520616E6420686561746265643F0046
:101A500057697A61726461206D757A657465206B6F
:101A600064796B6F6C6976207A6E6F76752073700F
:101A70007573746974207A206D656E752043616C8E
:101A80006962726174696F6E202D3E2057697A61B8
:101A9000726400596F752063616E20616C776179A3
:101AA0007320726573756D65207468652057697A57
:101AB0006172642066726F6D2043616C696272614D
:101AC00074696F6E202D3E2057697A6172642E0012
:101AD0004A6520746F20504C412066696C616D65C9
:101AE0006E743F00497320697420504C4120666930
:101AF0006C616D656E743F0050726F73696D207616
:101B00006C6F7A746520504C412066696C616D651C
:101B10006E7420646F206578747275646572752CBC
:101B200020706F20746520737469736B6E657465C3
:101B300020746C616369746B6F2070726F207A61BE
:101B4000766564656E692066696C616D656E747535
:101B50002E00506C6561736520696E736572742028
:101B6000504C412066696C616D656E7420746F2005
:101B70007468652065787472756465722C20746869
:101B8000656E207072657373206B6E6F6220746F68
:101B9000206C6F61642069742E0050726F73696DE0
:101BA000207A61766564746520504C412066696CCA
:101BB000616D656E74206120706F207465206F62A6
:101BC0006E6F7674652057697A61726461207374F0
:101BD00069736B6E7574696D2072657365742074BA
:101BE0006C616369746B612E00506C656173652074
:101BF0006C6F616420504C412066696C616D656E4C
:101C00007420616E64207468656E20726573756DF2
:101C1000652057697A617264206279207265626F0B
:101C20006F74696E6720746865207072696E746580
:101C3000722E00507265646568726976616D2074F9
:101C40007279736B752E2050726F73696D206365A6
:101C50006B656A74652E0050726568656174696EA3
:101C600067206E6F7A7A6C652E20506C65617365A3
:101C700020776169742E004A652066696C616D6524
:101C80006E74207A61766564656E3F0049732066E4
:101C9000696C616D656E74206C6F616465643F0092
:101CA000567365206A6520686F746F766F2E0041E9
:101CB0006C6C20697320646F6E652E2048617070B3
:101CC00079207072696E74696E67210050726F734B
:101CD000696D206F636973746574652068656174EC
:101CE000626564206120737469736B6E657465202E
:101CF000746C616369746B6F2E00506C6561736501
:101D000020636C65616E2068656174626564206142
:101D10006E64207468656E207072657373207468D9
:101D200065206B6E6F622E0050726F73696D206E4E
:101D300061686C65646E65746520646F206D616EAA
:101D400075616C752061206F7072617674652070AA
:101D5000726F626C656D2E20506F207465206F620B
:101D60006E6F7674652057697A617264612072655E
:101D7000626F6F746F76616E696D207469736B61E9
:101D8000726E792E00506C656173652063686563BF
:101D90006B206F75722068616E64626F6F6B20617B
:101DA0006E6420666978207468652070726F626C5A
:101DB000656D2E205468656E20726573756D6520A3
:101DC0007468652057697A6172642062792072654F
:101DD000626F6F74696E6720746865207072696ED7
:101DE0007465722E0057697A6172640020576174BD
:101DF0006368646F6720526573657400496E666F2F
:101E0000726D61636500496E666F2073637265650C
:101E10006E004B616C2E207072766E692076727344
:101E2000747679004669727374206C6179657220EA
:101E300063616C2E005761697420666F7220757340
:101E400065722E2E2E00506F757A6974652062655A
:101E500068656D207469736B7500557365642064E3
:101E60007572696E67207072696E74004F70616B75
:101E70006F76617420767973756E75746920666902
:101E80006C616D656E74753F00526570656174209C
:101E9000756E6C6F6164696E672066696C616D65F3
:101EA0006E743F0056796A6D6F75742066696C6157
:101EB0006D656E7400556E6C6F61642066696C614F
:101EC0006D656E74005679736F7576616D20666905
:101ED0006C616D656E7400556E6C6F6164696E67E0
:101EE0002066696C616D656E7400556E6B6E6F7700
:101EF0006E20636F6D6D616E643A2022004C6164E8
:101F000069740054756E65005344206361726420E7
:101F10005B466C73684169725D0053442063617273
:101F200064205B6E6F726D616C5D005465706C2E29
:101F3000206B616C2E20205B7A61705D0054656DB2
:101F4000702E2063616C2E2020205B6F6E5D00542C
:101F500065706C2E206B616C2E20205B7679705D35
:101F60000054656D702E2063616C2E20205B6F66BF
:101F7000665D005465706C6F746E69206B616C698E
:101F8000627261636520646F6B6F6E63656E612E54
:101F900020506F6B726163756A7465207374697326
:101FA0006B656D20746C616369746B612E005465A0
:101FB0006D70657261747572652063616C696272BF
:101FC0006174696F6E2069732066696E69736865F4
:101FD000642E20436C69636B20746F20636F6E7492
:101FE000696E75652E005465706C2E206B616C2EC9
:101FF000202020202020202020200054656D702EDD
:102000002063616C2E202020202020202020200012
:102010005465706C6F74610054656D7065726174A5
:1020200075726500506F64706F72610053757070E7
:102030006F7274005A617374617669742074697385
:102040006B0053746F70207072696E740053544F3C
:10205000505045442E2000537465707261746520A1
:10206000746F6F20686967683A20004A6520746958
:10207000736B6F767920706C6174206E6120686577
:1020800061746265643F00497320737465656C20F8
:102090007368656574206F6E20686561746265643D
:1020A0003F0043656C6B6F767920636173203A0063
:1020B000546F74616C207072696E742074696D6500
:1020C000203A0046696C616D656E742063656C6BC7
:1020D000656D203A00546F74616C2066696C616DA7
:1020E000656E74203A00436173207469736B7520C8
:1020F0003A2020005072696E742074696D653A2030
:10210000200046696C616D656E74203A202000469F
:10211000696C616D656E7420757365643A2020008A
:1021200053746174697374696B6120200053746126
:10213000746973746963732020004572726F722032
:102140002D20737461746963206D656D6F727920E1
:10215000686173206265656E206F7665727772695B
:102160007474656E00527963686C6F737400537099
:102170006565640020536F667477617265205265EF
:10218000736574004C65686B65207A6B6F73656E60
:10219000693A00536C6967687420736B65773A001D
:1021A0004D6F6420202020205B537465616C74683F
:1021B0005D004D6F6465202020205B537465616C69
:1021C00074685D004D6F642020202020205B4E6FDE
:1021D000726D616C5D004D6F646520202020205B76
:1021E0004E6F726D616C5D0053746176206B6F6E23
:1021F000632E207370696E2E0053686F7720656EB2
:10220000642073746F70730054657A6B65207A6B09
:102210006F73656E693A0053657665726520736BFE
:1022200065773A004E6173746176746520746570E9
:102230006C6F74753A005365742074656D706572C7
:1022400061747572653A004E6173746176656E698A
:102250000053657474696E67730043687962612026
:102260007A61706F6A656E6900576972696E67207E
:102270006572726F720053656C66207465737420AA
:1022800073746172742020005A6B6F6E74726F6C7D
:10229000756A7465203A00506C65617365206368E7
:1022A00065636B203A0053656C6620746573742017
:1022B0004F4B004E657A61706F6A656E6F2020200B
:1022C00020004E6F7420636F6E6E656374656400EA
:1022D0004D6F746F72004865617465722F54686544
:1022E000726D6973746F7200546573742076656ED5
:1022F00074696C61746F72750046616E20746573E9
:10230000740053656C66746573742073656C6861E2
:102310006C20200053656C66746573742066616977
:102320006C65642020004C6576792076656E74209B
:102330006E61207472797363653F004C656674202A
:10234000686F74656E642066616E3F0053656C66ED
:1023500074657374206572726F72202100456E641B
:1023600073746F70206E6F742068697400456E64BA
:1023700073746F707300456E6473746F7000507285
:1023800065646E69207469736B6F76792076656E0B
:10239000743F0046726F6E74207072696E742066AE
:1023A000616E3F004B6F6E74726F6C61205A2061DA
:1023B000786973202000436865636B696E67205AF3
:1023C00020617869732020004B6F6E74726F6C61AE
:1023D00020592061786973202000436865636B6928
:1023E0006E67205920617869732020004B6F6E74EE
:1023F000726F6C61205820617869732020004368F7
:1024000065636B696E6720582061786973202000CE
:102410004B6F6E74726F6C6120686F74656E6420B0
:102420002000436865636B696E6720686F74656E32
:10243000642020004B6F6E74726F6C6120656E6457
:1024400073746F707300436865636B696E672065B2
:102450006E6473746F7073004B6F6E74726F6C6127
:1024600020626564202020202000436865636B693A
:102470006E6720626564202020202000567365204E
:102480004F4B202020202020202020202000416CA5
:102490006C20636F727265637420202020202000FE
:1024A000426564202F204865617465720044656C44
:1024B0006B61206F73790041786973206C656E677A
:1024C0007468004F736100417869730053656C66EE
:1024D0007465737420202020202020202000577253
:1024E0006974696E6720746F2066696C653A2000B4
:1024F000766F6C756D652E696E6974206661696CA6
:102500006564002053697A653A20004B61727461FA
:102510002076796A6D75746100436172642072651A
:102520006D6F766564005344207072696E74696ED5
:1025300067206279746520006F70656E206661693E
:102540006C65642C2046696C653A20006F70656E7E
:10255000526F6F74206661696C6564004B617274C0
:102560006120766C6F7A656E6100436172642069E8
:102570006E73657274656400534420696E697420DB
:102580006661696C0046696C652073656C6563748F
:1025900065640046696C65206F70656E65643A20FD
:1025A000006572726F722077726974696E67207449
:1025B0006F2066696C650053442063617264206F0C
:1025C0006B0043616E6E6F7420656E74657220736C
:1025D00075626469723A200050726176793A0052ED
:1025E000696768743A004F626E6F766F76616E69E4
:1025F000207469736B7500526573756D696E672021
:102600007072696E74004F626E6F76656E692074C9
:1026100069736B7500526573756D696E67207072B2
:10262000696E7400506F6B7261636F7661740052F3
:102630006573756D65207072696E7400526573659F
:102640006E643A20004F64737472616E7465207416
:1026500069736B6F767920706C6174207A2068657D
:1026600061746265642070726F73696D2E00506CC6
:10267000656173652072656D6F766520737465653D
:102680006C2073686565742066726F6D2068656183
:10269000746265642E00446574656B6F76616E20AC
:1026A0007679706164656B2070726F7564752E4FFA
:1026B000626E6F766974207469736B3F00426C615F
:1026C000636B6F7574206F636375727265642E201F
:1026D0005265636F766572207072696E743F004F49
:1026E000626E6F766F76616E69207469736B7520A8
:1026F000202020005265636F766572696E672070D6
:1027000072696E742020202000686F77746F2E70BD
:102710007275736133642E637A00686F77746F2EFD
:10272000707275736133642E636F6D00666F7275BE
:102730006D2E707275736133642E637A00666F72EA
:10274000756D2E707275736133642E636F6D0070DA
:102750007275736133642E637A00707275736133BE
:10276000642E636F6D005469736B20706F7A6173B0
:10277000746176656E005072696E74207061757355
:102780006564005469736B20707265727573656E51
:10279000005072696E742061626F727465640050DB
:1027A00072696E74657220646973636F6E6E6563BF
:1027B0007465640050726F20767973756E757469F4
:1027C0002066696C616D656E747520737469736BD6
:1027D0006E6574652070726F73696D20746C6163CF
:1027E00069746B6F00506C656173652070726573FE
:1027F0007320746865206B6E6F6220746F20756E35
:102800006C6F61642066696C616D656E7400612037
:10281000737469736B6E65746520746C616369743D
:102820006B6F00616E6420707265737320746865ED
:10283000206B6E6F620050726564656872656A74C1
:102840006520747279736B752100507265686561DB
:102850007420746865206E6F7A7A6C6521005072FE
:1028600065646568726576005072656865617400BC
:10287000506F77657255700050726F73696D206389
:10288000656B656A746500506C656173652077617E
:102890006974004E656A6472697665207A6176654E
:1028A00064746520504C412066696C616D656E747E
:1028B0002070726F73696D2E00506C6561736520B6
:1028C0006C6F616420504C412066696C616D656E6F
:1028D000742066697273742E004A6520504C412042
:1028E00066696C616D656E74207A61766564656E8B
:1028F0003F00497320504C412066696C616D656EE4
:1029000074206C6F616465643F002020506C616EC0
:102910006E657242756666657242797465733A20B7
:1029200000556D6973746574652070726F73696D9D
:10293000207469736B6F767920706C6174206E619E
:10294000206865617462656400506C656173652020
:10295000706C61636520737465656C207368656570
:1029600074206F6E20686561746265642E004E612C
:1029700068726976616E692050494E444100504941
:102980004E44412048656174696E67005049442097
:102990006B616C2E20202020202020202020200071
:1029A0005049442063616C2E2020202020202020CC
:1029B00020202000504944206B616C2E20756B6FE5
:1029C0006E63656E61005049442063616C2E206621
:1029D000696E697368656400504944206B616C6975
:1029E0006272616365005049442063616C69627280
:1029F0006174696F6E00506F7A6173746176697487
:102A0000207469736B005061757365207072696E14
:102A10007400556D697374657465206C69737420F6
:102A2000706170697275206E6120706F646C6F7A6E
:102A30006B752061207564727A756A7465206A65A9
:102A40006A20706F6420747279736B6F7520626591
:102A500068656D206D6572656E69207072766E694D
:102A60006368203420626F64752E20506F6B75642C
:102A700020747279736B61207A616368797469205C
:102A800070617069722C207679706E65746520743F
:102A900069736B61726E752E00506C6163652061A5
:102AA000207368656574206F6620706170657220A0
:102AB000756E64657220746865206E6F7A7A6C65D5
:102AC00020647572696E67207468652063616C6943
:102AD00062726174696F6E206F66206669727374CA
:102AE000203420706F696E74732E204966207468DC
:102AF00065206E6F7A7A6C652063617463686573B4
:102B0000207468652070617065722C20706F776525
:102B100072206F666620746865207072696E7465D5
:102B20007220696D6D6564696174656C792E006FE2
:102B30006B004F6666004E6F206D6F76652E005AF3
:102B400061646E61205344206B61727461004E6F4A
:102B5000205344206361726400547279736B610086
:102B60004E6F7A7A6C650046696C616D656E742093
:102B70006E657A61766564656E0046696C616D6547
:102B80006E74206E6F74206C6F61646564004261C6
:102B9000727661206E656E692063697374610043AB
:102BA0006F6C6F72206E6F7420636C656172004E83
:102BB00065004E6F0050726F73696D20616B7475A4
:102BC000616C697A756A74652E00506C6561736515
:102BD00020757067726164652E005679736C612090
:102BE0006E6F7661207665727A65206669726D77A0
:102BF0006172653A004E6577206669726D77617221
:102C0000652076657273696F6E20617661696C61AB
:102C1000626C653A00506F73756E6F7574205A0060
:102C20004D6F7665205A00506F73756E6F75742006
:102C300059004D6F7665205900506F73756E6F7532
:102C4000742058004D6F7665205800457874727571
:102C500064657200506F73756E6F7574206F737555
:102C6000004D6F76652061786973004D657368204B
:102C7000426564204C6576656C696E67004B616CDB
:102C80006962726163650043616C69627261746953
:102C90006F6E00207A203900206F662039004D6564
:102CA00072696D207265666572656E636E69207605
:102CB00079736B75206B616C69627261636E6968B0
:102CC0006F20626F6475004D6561737572696E6720
:102CD000207265666572656E636520686569676800
:102CE00074206F662063616C6962726174696F6ED3
:102CF00020706F696E74004D6572656E65207A6B29
:102D00006F73656E693A004D656173757265642015
:102D1000736B65773A00486C61766E69206E61620C
:102D200069646B61004D61696E004D32323120493A
:102D30006E76616C69642065787472756465722062
:102D4000004D32313820496E76616C6964206578B7
:102D500074727564657220004D32303020496E7691
:102D6000616C6964206578747275646572200052C4
:102D700065706F7274696E6720656E6473746F70CE
:102D800020737461747573004D313137204B616C61
:102D90002E207072766E6920767273747679004D8B
:102DA000313137204669727374206C617965722005
:102DB00063616C2E004649524D574152455F4E416A
:102DC0004D453A4D61726C696E2056312E302E326F
:102DD0003B20537072696E7465722F6772626C204B
:102DE0006D617368757020666F722067656E36203E
:102DF0004649524D574152455F55524C3A6874749A
:102E000070733A2F2F6769746875622E636F6D2F28
:102E1000707275736133642F50727573612D6933ED
:102E20002D506C75732F2050524F544F434F4C5FB1
:102E300056455253494F4E3A312E30204D4143486A
:102E4000494E455F545950453A5072757361206937
:102E500033204D4B332045585452554445525F431F
:102E60004F554E543A3120555549443A3030303060
:102E7000303030302D303030302D303030302D305B
:102E80003030302D30303030303030303030303045
:102E90000A004D31303920496E76616C69642065D5
:102EA0007874727564657220004D31303520496E3A
:102EB00076616C696420657874727564657220004F
:102EC0004D31303420496E76616C696420657874C8
:102ED0007275646572200055766F6C6E656E612048
:102EE00072656D656E69636B61004C6F6F73652011
:102EF00070756C6C6579005A6176657374206669CB
:102F00006C616D656E74004C6F61642066696C6104
:102F10006D656E74005A61766164656E69206669DC
:102F20006C616D656E7475004C6F6164696E6720CD
:102F300066696C616D656E740043697374656E6972
:102F4000206261727679004C6F6164696E672063FC
:102F50006F6C6F72004C6576793A004C6566743A16
:102F6000005679626572206A617A796B61005365F7
:102F70006C656374206C616E67756167650043659D
:102F80007374696E6100456E676C697368004B49C4
:102F90004C4C45442E2000496E76616C6964206576
:102FA0007874727564657200566C6F7A7465206609
:102FB000696C616D656E7400496E7365727420662C
:102FC000696C616D656E74005072696E7420464163
:102FD0004E3A20004E6F7A7A6C652046414E3A0098
:102FE000457874727564657220696E666F00207A28
:102FF000203400206F662034005A6C657073756A47
:103000006920707265736E6F7374206B616C696296
:103010007261636E69686F20626F647500496D70DC
:10302000726F76696E67206265642063616C6962A5
:10303000726174696F6E20706F696E74004B616CA1
:10304000696272756A69205A0043616C69627261D3
:1030500074696E67205A004B616C696272616365C6
:10306000204F4B0043616C6962726174696F6E201E
:10307000646F6E65004B616C6962726F766174207B
:103080005A0043616C696272617465205A005A612A
:1030900068726976616E69204F4B2E0048656174D5
:1030A000696E6720646F6E652E005A61687269767A
:1030B000616E690048656174696E670046696C2ECF
:1030C0002073656E7A6F72205B7A61705D0046696D
:1030D0006C2E2073656E736F7220205B6F6E5D00C7
:1030E00046696C2E2073656E7A6F72205B767970FC
:1030F0005D0046696C2E2073656E736F72205B6F86
:1031000066665D002046726565204D656D6F72795B
:103110003A20005469736B61726E61206E6562794A
:103120006C61206A65737465207A6B616C69627288
:103130006F76616E612E20506F73747570756A744E
:10314000652070726F73696D20706F646C65206D9F
:10315000616E75616C752C206B617069746F6C6148
:10316000205A6163696E616D652C206F64737461B0
:1031700076656320506F73747570206B616C696243
:10318000726163652E005072696E746572206861A9
:1031900073206E6F74206265656E2063616C696276
:1031A0007261746564207965742E20506C6561735A
:1031B0006520666F6C6C6F7720746865206D616E3A
:1031C00075616C2C20636861707465722046697249
:1031D00073742073746570732C2073656374696FE6
:1031E0006E2043616C6962726174696F6E20666CF7
:1031F0006F772E00507275746F6B00466C6F77009E
:10320000446F6B6F6E636F76616E6920706F687963
:1032100062750046696E697368696E67206D6F76C6
:10322000656D656E747300207A203400206F66200F
:103230003400486C6564616D206B616C6962726119
:10324000636E6920626F6420706F646C6F7A6B7953
:1032500000536561726368696E672062656420630C
:10326000616C6962726174696F6E20706F696E74EF
:103270000049746572616365200049746572617408
:10328000696F6E2000446F6E6520736176696E67AA
:103290002066696C652E00446F6E65207072696EE1
:1032A00074696E672066696C65004A6520626172A8
:1032B00076612063697374613F00497320636F6CAA
:1032C0006F7220636C6561723F0056796D656E693F
:1032D000742066696C616D656E74004368616E6729
:1032E000652066696C616D656E7400527963686C07
:1032F0006F73742076656E742E0046616E20737055
:10330000656564004B6F6E74722E2076656E742E48
:103310005B7A61705D0046616E7320636865636B04
:103320002020205B6F6E5D004B6F6E74722E2076D6
:10333000656E742E5B7679705D0046616E732063F6
:103340006865636B20205B6F66665D00656E7175F6
:1033500065696E6720220045787472756465720035
:103360002045787465726E616C20526573657400D7
:103370005072696E7465722073746F70706564202A
:1033800064756520746F206572726F72732E2046AB
:10339000697820746865206572726F7220616E644E
:1033A00020757365204D39393920746F207265732B
:1033B000746172742E202854656D70657261747525
:1033C00072652069732072657365742E205365746D
:1033D000206974206166746572207265737461720D
:1033E00074696E6729004E6F204C696E65204E75BA
:1033F0006D626572207769746820636865636B73BA
:10340000756D2C204C617374204C696E653A2000F8
:103410004E6F20436865636B73756D2077697468C0
:10342000206C696E65206E756D6265722C204C6132
:103430007374204C696E653A200020746F6F206CA5
:103440006F6E6720657874727573696F6E20707225
:103450006576656E746564004C696E65204E756DA9
:10346000626572206973206E6F74204C61737420E2
:103470004C696E65204E756D6265722B312C204C47
:10348000617374204C696E653A20005072696E74E5
:1034900065722068616C7465642E206B696C6C28A1
:1034A000292063616C6C6564210020636F6C64206B
:1034B000657874727573696F6E2070726576656E6B
:1034C00074656400636865636B73756D206D697303
:1034D0006D617463682C204C617374204C696E6557
:1034E0003A200043485942413A004552524F523A1D
:1034F00000456E642066696C65206C697374006FAA
:1035000070656E0054524947474552454400656E08
:103510006473746F7073206869743A2000536C652B
:1035200065702E2E2E005679706E6F7574206D6F3B
:10353000746F72790044697361626C65207374659D
:10354000707065727300446174756D3A0044617403
:10355000653A00506F757A6520616B7475616C6EA9
:10356000690043757272656E7400437261736820FE
:103570006465742E20205B7A61705D004372617314
:1035800068206465742E2020205B6F6E5D0043729E
:10359000617368206465742E20205B7679705D000D
:1035A0004372617368206465742E20205B6F6666C9
:1035B0005D0020436F756E7420583A200056796D77
:1035C000656E61206F6B3F004368616E67656420C4
:1035D000636F72726563746C793F005A63686C61E3
:1035E00064697400436F6F6C646F776E0050726F24
:1035F0002075737065736E6F75206B616C69627294
:10360000616369206F636973746574652070726F9C
:1036100073696D207469736B6F766F75207472793E
:10362000736B752E20506F74767264746520746CA1
:10363000616369746B656D2E00506C656173652004
:10364000636C65616E20746865206E6F7A7A6C6554
:1036500020666F722063616C6962726174696F6E5B
:103660002E20436C69636B207768656E20646F6EF3
:10367000652E00204C61737420557064617465641C
:103680003A200056796265727465206578747275A7
:103690006465723A0043686F6F7365206578747271
:1036A000756465723A005A6D656E61207573706558
:1036B000736E6121004368616E6765207375636393
:1036C00065737321005469736B207A205344005052
:1036D00072696E742066726F6D2053440054657079
:1036E0006C6F742E206B616C69627261636500544B
:1036F000656D702E2063616C6962726174696F6EB2
:10370000004B616C696272756A69205A0043616C92
:103710006962726174696E67205A005A6B616C69E4
:1037200062726F7661740043616C69627261746584
:103730000052657365742058595A206B616C696238
:10374000722E0052657365742058595A2063616C5B
:103750006962722E004B616C696272616365205808
:10376000595A0043616C6962726174652058595AF4
:10377000002042726F776E206F75742052657365FA
:103780007400426567696E2066696C65206C6973B8
:1037900074004B616C6962726163652058595A20EC
:1037A0006E65707265736E612E204C65767920703F
:1037B0007265646E6920626F64206D6F632076703D
:1037C000726564752E0058595A2063616C69627283
:1037D0006174696F6E20636F6D70726F6D69736570
:1037E000642E204C6566742066726F6E742063616F
:1037F0006C6962726174696F6E20706F696E74209B
:103800006E6F7420726561636861626C652E004B37
:10381000616C6962726163652058595A206E6570E7
:103820007265736E612E20507265646E69206B61E3
:103830006C69627261636E6920626F6479206D6F7A
:1038400063207670726564752E0058595A20636142
:103850006C6962726174696F6E20636F6D70726FF4
:103860006D697365642E2046726F6E742063616C9F
:103870006962726174696F6E20706F696E74732013
:103880006E6F7420726561636861626C652E004BB7
:10389000616C6962726163652058595A20762070A4
:1038A0006F7261646B752E20582F59206F737920C9
:1038B0006D69726E65207A6B6F73656E652E20443C
:1038C0006F627261207072616365210058595A20DD
:1038D00063616C6962726174696F6E20616C6C20E7
:1038E00072696768742E20582F592061786573209B
:1038F00061726520736C696768746C7920736B659D
:103900007765642E20476F6F64206A6F6221004BD9
:10391000616C6962726163652058595A2076207023
:103920006F7261646B752E205A6B6F73656E6920C0
:1039300062756465206175746F6D617469636B791C
:10394000207679726F766E616E6F20707269207466
:1039500069736B752E0058595A2063616C696272E5
:103960006174696F6E20616C6C2072696768742E77
:1039700020536B65772077696C6C20626520636FDC
:1039800072726563746564206175746F6D617469CA
:1039900063616C6C792E004B616C69627261636566
:1039A0002058595A2073656C68616C612E204B61F8
:1039B0006C69627261636E6920626F6420706F640B
:1039C0006C6F7A6B79206E656E616C657A656E2EB0
:1039D0000058595A2063616C6962726174696F6E34
:1039E000206661696C65642E204265642063616CA9
:1039F0006962726174696F6E20706F696E7420778E
:103A00006173206E6F7420666F756E642E004B615B
:103A10006C6962726163652058595A207620706F14
:103A20007261646B752E20582F59206F7379206A4C
:103A3000736F75206B6F6C6D652E204772617475A6
:103A40006C756A69210058595A2063616C69627209
:103A50006174696F6E206F6B2E20582F592061782A
:103A60006573206172652070657270656E6469634C
:103A7000756C61722E20436F6E67726174756C6134
:103A800074696F6E7321004B616C6962726163656A
:103A90002058595A2073656C68616C612E204E6104
:103AA000686C65646E65746520646F206D616E7509
:103AB000616C752E0058595A2063616C696272619D
:103AC00074696F6E206661696C65642E20506C6548
:103AD00061736520636F6E73756C74207468652004
:103AE0006D616E75616C2E004B616C696272616311
:103AF000652058595A2073656C68616C612E204CA2
:103B000065767920707265646E6920626F64206DDD
:103B10006F63207670726564752E2053726F766EB7
:103B2000656A7465207469736B61726E752E0058D6
:103B3000595A2063616C6962726174696F6E2066A4
:103B400061696C65642E204C6566742066726F6EC8
:103B5000742063616C6962726174696F6E20706F4A
:103B6000696E74206E6F7420726561636861626C47
:103B7000652E004B616C6962726163652058595A09
:103B80002073656C68616C612E20507265646E698B
:103B9000206B616C69627261636E6920626F647927
:103BA000206D6F63207670726564752E2053726F7E
:103BB000766E656A7465207469736B61726E752EBA
:103BC0000058595A2063616C6962726174696F6E42
:103BD000206661696C65642E2046726F6E74206386
:103BE000616C6962726174696F6E20706F696E7466
:103BF00073206E6F7420726561636861626C652EFC
:103C0000004B616C696272616365205A2073656C58
:103C100068616C612E2053656E736F72206A652037
:103C20006F64706F6A656E79206E65626F20707266
:103C300065727573656E79206B6162656C2E2043C9
:103C4000656B616D206E612072657365742E004234
:103C50006564206C6576656C696E67206661696C69
:103C600065642E2053656E736F7220646973636F91
:103C70006E6E6563746564206F72206361626C654B
:103C80002062726F6B656E2E2057616974696E6772
:103C900020666F722072657365742E004B616C69CB
:103CA0006272616365205A2073656C68616C612E75
:103CB0002053656E736F72206E657365706E756CE0
:103CC0002E205A6E6563697374656E612074727913
:103CD000736B613F2043656B616D206E612072657F
:103CE0007365742E00426564206C6576656C696E40
:103CF00067206661696C65642E2053656E736F7210
:103D0000206469646E7420747269676765722E201E
:103D1000446562726973206F6E206E6F7A7A6C658B
:103D20003F2057616974696E6720666F7220726503
:103D30007365742E004B616C696272616365205A11
:103D40002073656C68616C612E2053656E736F72B1
:103D5000207365706E756C207072696C6973207663
:103D600079736F6B6F2E2043656B616D206E6120E0
:103D700072657365742E00426564206C6576656CAF
:103D8000696E67206661696C65642E2053656E7389
:103D90006F722074726967676572656420746F6FF3
:103DA00020686967682E2057616974696E672066AC
:103DB0006F722072657365742E005A61687269763D
:103DC000616E6920626564004265642048656174C3
:103DD000696E6700426564204F4B2E004265642087
:103DE000646F6E650056707261766F205B756D5DF5
:103DF00000526967687420736964655B756D5D0066
:103E0000526573657400567A61647520205B756D28
:103E10005D00526561722073696465205B756D5D3C
:103E2000004B6F72656B636520706F646C6F7A6BAB
:103E30007900426564206C6576656C20636F7272F0
:103E400065637400566C65766F20205B756D5D0050
:103E50004C6566742073696465205B756D5D005602
:103E60007072656475205B756D5D0046726F6E746F
:103E700020736964655B756D5D00426564004E6525
:103E80006E69207A6B616C6962726F76616E612017
:103E9000767A64616C656E6F737420747279736B7B
:103EA00079206F64207469736B6F766520706F641E
:103EB0006C6F7A6B792E20506F73747570756A749D
:103EC000652070726F73696D20706F646C65206D12
:103ED000616E75616C752C206B617069746F6C61BB
:103EE000205A6163696E616D652C206F6473746123
:103EF000766563204E6173746176656E69207072B9
:103F0000766E69207672737476792E0044697374C4
:103F1000616E6365206265747765656E2074697093
:103F2000206F6620746865206E6F7A7A6C652061F8
:103F30006E642074686520626564207375726661C2
:103F4000636520686173206E6F74206265656E2002
:103F5000736574207965742E20506C6561736520DB
:103F6000666F6C6C6F7720746865206D616E75612B
:103F70006C2C20636861707465722046697273747A
:103F80002073746570732C2073656374696F6E2081
:103F90004669727374206C617965722063616C6923
:103FA00062726174696F6E2E00446F6C6164656E3D
:103FB00069206F7379205A004C6976652061646AC4
:103FC000757374205A0041646A757374696E672052
:103FD0005A004175746F20686F6D6500207C204128
:103FE0007574686F723A200056736500416C6C00FE
:103FF0004163746976652045787472756465723AB8
:1040000020000314F31317141F142714301438144A
:10401000551440146E146A1472147A149314821492
:10402000BE14A4141415DC1472155215F61595154A
:1040300004175916FB17B817A11848185419E8188F
:10404000FF19B319931A501AE41AD01A521BF81A0E
:10405000E91B9A1B571C331C8C1C771CAF1CA01C23
:10406000FA1CCC1C851D281DE51DEC1D061EFC1D23
:10407000241E121E351E5A1E461E891E6C1EB51E9B
:10408000A41ED71EC51EEA1E031FFD1E081F1A1FF1
:104090003D1F2B1F611F4F1FAE1F731FFB1FE61F0E
:1040A000182010202C202420422034204D2057207E
:1040B00087206B20B020A220D520C320F420E6204A
:1040C0000F2102212D2120213A216E216521742109
:1040D00093218421B221A021D621C421F921E821F4
:1040E00017220822362224225122472269225A22EC
:1040F000762297228822A622C222B322D022D6225A
:10410000F922E822142302233B2326234C235D2398
:104110006D23762393237E23B623A423DA23C82397
:10412000FE23EC2322241024462434246A24582419
:104130008E247C24A024B724AD24C724C324CC24FB
:10414000DE24F024032519250B25262538254C25AA
:104150006A255C25782585259325A125B725C225C7
:10416000DF25D825F725E625152606262F26242621
:104170003C266E264526BD269626F426DF261A27DF
:1041800009273D272C275A274F277627662791276F
:1041900083279F27E527B42723280E284A28362877
:1041A00068285E28702887287828B9289328F2285C
:1041B000D9280A29492921297E296E29A0298C2953
:1041C000C629B429E629D829062AF629992A122AC5
:1041D0002F2B322B362B4E2B3F2B602B592B7A2B30
:1041E000672B9F2B8E2BB22BAF2BCA2BB52BF52B0E
:1041F000DA2B202C152C322C272C442C392C4B2C30
:10420000612C542C6B2C872C7D2C982C932CC72C38
:104210009E2C072DF72C252D162D2A2D412D582D9E
:104220006F2D9F2D882DB52D922EA92EC02EEA2EF2
:10423000D72E072FF72E282F152F472F392F5B2F1B
:10424000552F6E2F612F862F7E2F8E2F972FB82FF1
:10425000A82FC82FD42FE02FF32FEE2F1D30F92FCA
:1042600049303D3064305730823075309C308E306C
:10427000B430AA30CE30BC30F230E0300431863178
:104280001331FB31F431133200322C3227325132E8
:1042900032327A32713285329732BA32AA32DB3216
:1042A000CA32FA32EB32163304333A3328334C3302
:1042B000573360337033E63310343A3458348B3428
:1042C000AA34C434EA34E334F134FF3404350E350F
:1042D0001D35353526354D354635623553357C35FA
:1042E0006A35A0358E35B235C835BD35E435DB3598
:1042F0003936ED35733695368336B536A636CF3634
:10430000C536EF36DD360D37013727371B374337D4
:1043100031376337553771378237C63792374A3866
:104320000F38CC388F3856390F39D1399739463A4A
:104330000E3AB53A873A2F3BE83AC13B733B4F3CC4
:10434000013CE53C9C3C773D353DC83DBA3DDC3DFC
:10435000D43DF13DE53D003E123E063E323E213E5B
:10436000503E443E6B3E5F3E7A3E0C3F7E3EB83F41
:10437000A93FC63FD23FDC3FEC3FE83FF03F4578E6
:1043800072656D65207370616E206F66207468655C
:10439000205A2076616C756573210043616C6375EA
:1043A0006C6174696F6E206F6620746865206D6142
:1043B0006368696E6520736B657720616E64206F3A
:1043C0006666736574206661696C65642E00203CC6
:1043D00020005741524E494E473A2046726F6E7444
:1043E00020706F696E74206E6F74207265616368EF
:1043F00061626C652E205920636F6F7264696E6113
:1044000074653A0000497465726174696F6E3A2090
:1044100000496E76616C69642062656420636F7226
:1044200072656374696F6E206D61747269782E2095
:10443000526573657474696E6720746F2069646572
:104440006E746974792E00496E76616C69642062BD
:10445000656420636F7272656374696F6E206D614D
:10446000747269782E20582F592061786573206105
:104470007265206661722066726F6D206265696E7A
:10448000672070657270656E646963756C61722E09
:1044900000496E76616C69642062656420636F72A6
:1044A00072656374696F6E206D61747269782E2015
:1044B0005368696674206F7574206F662072616E30
:1044C00067652E005A65726F20706F696E74206385
:1044D0006F7272656374696F6E3A00496E76616CD3
:1044E00069642062656420636F7272656374696FCA
:1044F0006E206D61747269782E204C656E677468E9
:10450000206F6620746865205920766563746F7229
:10451000206F7574206F662072616E67652E00597A
:1045200020766563746F72206C656E6774683A00FC
:10453000496E76616C69642062656420636F727293
:10454000656374696F6E206D61747269782E204C9A
:10455000656E677468206F662074686520582076E1
:104560006563746F72206F7574206F662072616E60
:1045700067652E005820766563746F72206C656ED7
:104580006774683A00556E646566696E656420629A
:10459000656420636F7272656374696F6E206D610C
:1045A000747269782E0000004041FFFFBF40000098
:1045B0005C43FFFFBF4000005C4300004643000037
:1045C00040410000464300004041FFFFBF40000063
:1045D000E442FFFFBF4000005743FFFFBF40000021
:1045E00057430000CC420000E4420000CC420000EF
:1045F00040410000CC420000404100004643000022
:10460000E4420000464300005743000046435A007E
:10461000205A3A00590020593A00580020583A00D0
:1046200024F4D43050C38E20C2A24017828B701164
:10463000127A910D816CD90AA861E108C758660702
:10464000615143061E4B5D05C145A7041A41110483
:10465000093D9803713931034036DB02653391021D
:10466000D4305402802E1D02632CEE01752AC50140
:10467000B028A001102781018F2564012B244B0154
:10468000E0223401AC211F018D200D01801FFC00B0
:10469000841EED00971DDF00B81CD200E61BC6008B
:1046A000201BBC00641AB200B219A8000A19A000AD
:1046B0006A189900D117910040178B00B516840035
:1046C00031167E00B31579003A157300C7146F00D8
:1046D00058146A00EE1366008813630025135E0009
:1046E000C7125B006C12570015125400C111510023
:1046F00070114F0021114B00D61049008D1047005A
:104700004610440002104200C00F4000800F3E00DF
:10471000420F3C00060F3B00CB0E3800930E3700D3
:104720005C0E3500270E3400F30D3200C10D310050
:10473000900D3000600D2E00320D2D00050D2C0067
:10474000D90C2B00AE0C2900850C29005C0C27002D
:10475000350C27000E0C2600E80B2400C40B2400A7
:10476000A00B23007D0B23005A0B2100390B2100E5
:10477000180B2000F80A1F00D90A1E00BB0A1E00F1
:104780009D0A1D00800A1D00630A1C00470A1B00C9
:104790002C0A1B00110A1A00F7091A00DD0919007A
:1047A000C4091900AB091900920917007B09180008
:1047B000630917004C091600360916002009160077
:1047C0000A091500F5081500E0081400CC081400CB
:1047D000B8081400A4081400900813007D08120003
:1047E0006B08130058081200460812003408110024
:1047F000230811001208110001081100F007100031
:10480000E0071000D0071000C0071000B0070F002D
:10481000A107100091070E0083070F0074070F0017
:1048200065070E0057070E0049070E003B070D00F5
:104830002E070E0020070D0013070D0006070D00C0
:10484000F9060C00ED060D00E0060C00D4060C0085
:10485000C8060C00BC060C00B0060C00A4060B0039
:1048600099060C008D060B0082060B0077060B00E4
:104870006C060B0061060A0057060B004C060A0086
:1048800042060A0038060A002E060A0024060A001C
:104890001A060A001006090007060A00FD050900AD
:1048A000F4050900EB050900E2050900D905090036
:1048B000D0050900C7050900BE050900B5050800B7
:1048C000AD050800A50509009C0508009405080031
:1048D0008C050800840508007C05080074050800A4
:1048E0006C050700650508005D0507005605080012
:1048F0004E0507004705070040050800380507007A
:10490000310507002A050700230507001C050600DE
:10491000160507000F050700080506000205070039
:10492000FB040600F5040700EE040600E804060098
:10493000E2040700DB040600D5040600CF040600ED
:10494000C9040600C3040600BD040600B70406003F
:10495000B1040500AC040600A6040600A00405008E
:104960009B04060095040500900406008A040500D7
:1049700085040500800406007A040500750405001E
:10498000700405006B040500660405006104050061
:104990005C04050057040500520405004D040500A1
:1049A00048040500430405003E0404003A040500E1
:1049B00035040500300404002C040500270404001D
:1049C000230405001E0404001A0404001604050054
:1049D000110404000D04040009040500040404008B
:1049E00000040400FC030400F8030400F4030400C2
:1049F000F0030400EC030400E8030400E4030400F3
:104A0000E0030400DC030400D8030400D403040022
:104A1000D0030400CC030400C8030300C503030053
:104A200024F404D9201BC40C5C0E9804C4095F0252
:104A300065077101F405F900FB04B3004804870021
:104A4000C10369005803550003034500BE023A0044
:104A50008402310053022A002902250004022000AA
:104A6000E4011C00C8011900AF01170098011400EF
:104A700084011300710110006101100051010E004A
:104A800043010D0036010B002B010B0020010B0030
:104A9000150109000C01090003010800FB000800D2
:104AA000F3000800EB000700E4000600DE0006004B
:104AB000D8000600D2000600CC000500C7000500A3
:104AC000C2000500BD000400B9000400B5000400E8
:104AD000B1000400AD000400A9000400A50003001B
:104AE000A20003009F0004009B0003009800030045
:104AF0009500020093000300900003008D00020067
:104B00008B0003008800020086000200840003007E
:104B1000810002007F0002007D0002007B00020095
:104B200079000200770001007600020074000200A4
:104B300072000100710002006F0002006D000100B0
:104B40006C0002006A0001006900020067000100B9
:104B500066000100650001006400020062000100BF
:104B600061000100600001005F0002005D000100C3
:104B70005C0001005B0001005A00010059000100C7
:104B800058000100570001005600010055000100C7
:104B900054000100530000005300010052000100C6
:104BA00051000100500001004F0001004E000000C4
:104BB0004E0001004D0001004C0001004B000000C0
:104BC0004B0001004A0001004900010048000000BC
:104BD00048000100470001004600000046000100B7
:104BE00045000000450001004400010043000000B2
:104BF00043000100420000004200010041000000AB
:104C000041000100400001003F0000003F000100A2
:104C10003E0000003E0001003D0000003D0001009C
:104C20003C0000003C0000003C0001003B00000094
:104C30003B0001003A0000003A000100390000008A
:104C40003900010038000000380000003800010081
:104C50003700000037000100360000003600000079
:104C6000360001003500000035000000350001006D
:104C70003400000034000000340001003300000064
:104C80003300000033000100320000003200000059
:104C9000320001003100000031000000310001004D
:104CA0003000000030000000300001002F00000044
:104CB0002F0000002F0000002F0001002E00000038
:104CC0002E0000002E0001002D0000002D0000002D
:104CD0002D0000002D0001002C0000002C00000021
:104CE0002C0000002C0001002B0000002B00000015
:104CF0002B0000002B0001002A0000002A00000009
:104D00002A0000002A0001002900000029000000FC
:104D100029000000290000002900010028000000EF
:104D200028000000280000002800000028000100E2
:104D300027000000270000002700000027000000D7
:104D400027000100260000002600000026000000C9
:104D500026000000260001002500000025000000BC
:104D600025000000250000002500000025000100AE
:104D700024000000240000002400000024000000A3
:104D80002400010023000000230000002300000095
:104D90002300000023000000230000002300010086
:104DA000220000002200000022000000220000007B
:104DB000220000002200010021000000210000006C
:104DC000210000002100000021000000210000005F
:104DD0002100010020000000200000002000000051
:104DE0002000000020000000200000002000000043
:104DF000200001001F0000001F0000001F00000035
:104E00001F0000001F0000001F0000001F00010025
:104E10001E0000001E0000001E0000001E0000001A
:104E20004572723A204D494E54454D5020424544FA
:104E30000054656D70657261747572652068656196
:104E4000746564206265642073776974636865645F
:104E5000206F66662E204D494E54454D5020747289
:104E6000696767657265642021004572723A204D5A
:104E7000415854454D50204245440054656D70657D
:104E8000726174757265206865617465642062651D
:104E900064207377697463686564206F66662E208A
:104EA0004D415854454D502074726967676572656D
:104EB000642021004572723A204D494E54454D50B0
:104EC000003A20457874727564657220737769744E
:104ED00063686564206F66662E204D494E54454DCB
:104EE000502074726967676572656420210045729D
:104EF000723A204D415854454D50003A204578743F
:104F00007275646572207377697463686564206F75
:104F100066662E204D415854454D50207472696785
:104F2000676572656420210020484F54454E442037
:104F3000544845524D414C2052554E41574159001D
:104F4000204845415442454420544845524D414C27
:104F50002052554E4157415900544845524D414CFD
:104F60002052554E4157415900424544205448452E
:104F7000524D414C2052554E415741590020544802
:104F800045524D414C2052554E4157415920282001
:104F90005052454845415420484F54454E442900FD
:104FA00020544845524D414C2052554E415741598D
:104FB00020282050524548454154204845415442FC
:104FC0004544290050524548454154204552524FCE
:104FD00052004245442050524548454154204552D4
:104FE000524F52004572723A205052494E54204658
:104FF000414E204552524F52004552524F523A2094
:105000005072696E742066616E20737065656420ED
:105010006973206C6F776572207468656E2065789F
:10502000706563746564004572723A204558545245
:105030002E2046414E204552524F52004552524F6B
:10504000523A2045787472756465722066616E20EC
:105050007370656564206973206C6F776572207466
:1050600068656E20657870656374656400202D2026
:10507000496E76616C6964206578747275646572D6
:10508000206E756D62657220210050494420417583
:10509000746F74756E652066696E697368656421E6
:1050A0002050757420746865206C617374204B7097
:1050B0002C204B6920616E64204B6420636F6E73FB
:1050C00074616E74732066726F6D2061626F7665B5
:1050D00020696E746F20436F6E66696775726174C4
:1050E000696F6E2E6800504944204175746F747565
:1050F0006E65206661696C6564212074696D656FF9
:1051000075740020403A006F6B20543A006F6B209A
:10511000423A00504944204175746F74756E6520A1
:105120006661696C6564212054656D706572617497
:1051300075726520746F6F206869676800204B6422
:105140003A2000204B693A2000204B703A20002082
:10515000436C617373696320504944200020547587
:105160003A2000204B753A2000206D61783A2000EB
:10517000206D696E3A200020643A20002062696147
:10518000733A200010137D0020157800601773001B
:10519000C0196E00401C6900E01E640080215F00A1
:1051A00040245A00F026550090295000202C4B0036
:1051B000802E4600C0304100D0323C00B034370071
:1051C00050363200C0372D0000392800103A230035
:1051D000F03A1E00B03B1900503C1400D03C0F00C8
:1051E000303D0A00803D0500C03D0000F03DFBFF62
:1051F000103EF6FF303EF1FF403EECFF503EE7FF31
:10520000603EE2FF703EDDFF703ED8FF1000C90235
:1052100010012C014001220170011801B0010E01A2
:10522000F00104015002FA00B002F0003003E60081
:10523000D003DC009004D2007005C800A006BE00B8
:105240000008B400B009AA00D00BA000600E9600C0
:1052500060118C000015820020197800C01D6E00BE
:10526000A0226400B0275A00902C50000031460064
:10527000E0343C0010383200903A2800603C1E00B8
:10528000A03D1400803E0A00203F000070012C0168
:1052900090012701B0012201C0011D01F001180198
:1052A0001002130130020E01600209019002040194
:1052B000C002FF000003FA004003F5008003F00085
:1052C000D003EB002004E6007004E100E004DC0001
:1052D0004005D700C005D2004006CD00D006C8006A
:1052E0008007C3003008BE00F008B900C009B40050
:1052F000B00AAF00B00BAA00D00CA500000EA000B1
:10530000500F9B00C01096005012910000148C00AA
:10531000C0158700B0178200B0197D00D01B78003F
:10532000001E730040206E0090226900F02464008B
:1053300040275F0090295A00E02B5500102E5000A6
:1053400020304B0010324600E033410090353C00E5
:105350001037370070383200A0392D00B03A2800DD
:10536000A03B2300603C1E00103D1900903D14003E
:10537000103E0F00703E0A00C03E0500003F0000D6
:10538000544D4320445249564552204F564552549D
:10539000454D502000436F6E74696E7565207769C6
:1053A000746820616E6F7468657220626F776465DF
:1053B0006E3F0053746174653A2000473736004DE4
:1053C0003435205A004D3435004738300020003E37
:1053D000003E0020003E003E003E003E0020003E19
:1053E000003E00200000002D2D2D2D2D2D2D2D2DCA
:1053F0002D2D2D2D2D2D2D2D2D2D2D004E2F410000
:105400004E2F41006D6D00004D373031004D37306B
:105410003200496E76616C696420504944206361B2
:105420006C2E20726573756C74732E204E6F742011
:1054300073746F72656420746F20454550524F4DF0
:105440002E004D353030004731205A31352046315D
:105450003530300047393100473120583530205938
:105460003139302045302046373030300047393030
:10547000004D373032004D3730322043004D373049
:10548000322055004D373032004731205A31352017
:1054900046313530300047393100473120583530FA
:1054A0002059313930204530204637303030004DDA
:1054B000383300473930004D3834004D3130342016
:1054C0005330004D383400473120583130205931A5
:1054D0003830204634303030004731205A313020C7
:1054E00046313330302E303030004D31343020539F
:1054F00030004D313034205330004D3130370047CB
:105500003120452D302E3037353030204632313085
:10551000302E30303030300047312058353020596F
:1055200035352045332E3632373733004731205852
:10553000323030205935352045302E343933383625
:105540000047312058323030205937352045332E2E
:105550003632373733004731205835302059373508
:105560002045302E34393338360047312058353015
:10557000205939352045332E3632373733004731FD
:105580002058323030205939352045302E343933C7
:1055900038360047312058323030205931313520EB
:1055A00045332E36323737330047312058353020D7
:1055B000593131352045302E3439333836004731B2
:1055C0002058353020593133352045332E36323787
:1055D00037330047312058323030205931333520AD
:1055E00045302E363631373400473120583230308E
:1055F00020593135352045322E3632373733004782
:10560000312058313030205931353520453200476E
:10561000312058373520593135352045322E350067
:10562000473120463130383000473120583530205E
:1056300059313535004731204634303030004D3255
:105640003034205331303030004731205A302E3141
:1056500035302046373230302E3030300047312060
:10566000452D312E35303030302046323130302E1D
:105670003030303030004D38330047393000473259
:1056800031004739322045302E3000473120583123
:1056900030302E30204531322E35204631303030FA
:1056A0002E30004731205836302E302045392E30EC
:1056B0002046313030302E30004739322045302EF0
:1056C000300047323800473837004D3130392053E9
:1056D000323130004D31393020533535004D3134C1
:1056E0003020533535004D313034205332313000C5
:1056F0004D31303700473930004731204531004DBA
:105700003832004731204531004D3833004D3130BB
:105710003620532564004D32323020532564003A40
:105720002000202020202020202020202020202099
:10573000202020202000203A20002020202020208F
:105740002020202020202020202020202020002079
:105750002020202020202020202020200025730031
:105760002020002D2D3A2D2D002000200020004C5F
:10577000002020002046002D2D2D003E55534200D4
:105780005344002D2D002520202020200020200023
:105790002020000120002020202D2D2D2000202061
:1057A0005A002020000120004D36303000464C4584
:1057B00058202D20203233302F35300050502020FB
:1057C000202D20203235342F3130300048495053BD
:1057D000202D20203232302F3130300041425320F2
:1057E000202D20203235352F3130300050455420C7
:1057F000202D20203234302F393000504C412020D1
:105800002D20203231352F3630006661726D202018
:105810002D20203235302F3430004D3234004D32BF
:105820003320257300052E2E00580059005A0045DC
:105830007874727564657200473939004469736120
:10584000626C65206661726D206D6F64653F004417
:10585000697361626C65206661726D206D6F64654D
:10586000004661726D206E756D626572004D383450
:10587000005072696E742066616E3A0045787472E9
:10588000756465722066616E3A0041786973206CB8
:10589000656E67746820646966666572656E6365C7
:1058A0003A004D6561737572656420617869732093
:1058B0006C656E6774683A0025632041584953202F
:1058C0005347313D25640A004D3834004731205A92
:1058D0003135004732382057005A30005A310059CC
:1058E0003000593100583000583100456E64207343
:1058F000746F70732064696167004D3434004732FF
:10590000382057001B5B303B314842656C74207374
:1059100074617475731B5B313B3248582025641BDE
:105920005B323B324859202564001B5B313B3148D8
:10593000416D6269656E743A2020256425631B5BA6
:10594000323B314850494E44413A202020202564C2
:1059500025630054656D70657261747572657300BE
:1059600042656C7420737461747573002D2D2D2D38
:105970002D2D2D2D2D2D2D2D00466C617368416927
:105980007220495020416464723A002D2D2D2D2D36
:105990002D2D2D2D2D2D2D004E6F762032392032BC
:1059A000303137002D2D2D2D2D2D2D2D2D2D2D2D43
:1059B00000453344763666756C6C0045494E595F38
:1059C00030346100315F37356D6D5F4D4B33002DE5
:1059D0002D2D2D2D2D2D2D2D2D2D2D0020332E3126
:1059E0002E312D5243312062313230004669726DC2
:1059F000776172653A0025642E25642E25642E2574
:105A000064004661696C207374617473004661724E
:105A10006D206E756D626572000072630062657460
:105A20006100616C70686100646576005052555386
:105A3000413344465700332E312E312D524331002D
:105A400000000A0B02090C0D0E08070304010000F8
:105A50000000000000000000000000000000000046
:105A60000000000000000000000000001211100003
:105A70000000000000000000000000000000000026
:105A80000000000000000000000000000000000016
:105A90000000000000000102102020080810204033
:105AA00010204080020102010804020101020408E2
:105AB0001020408080402010080402018004020170
:105AC00080402010080402010804020101020408B9
:105AD00010204080010204081020408010080408B3
:105AE00080102040044080102040048005050505FA
:105AF000070508080808020202020A0A0808040446
:105B00000404010101010101010103030303030373
:105B10000303040707070C0C0C0C0C0C0C0C020202
:105B2000020206060606060606060B0B0B0B0B0BFF
:105B30000B0B07070A0A0A0A0A0A050505040404EA
:105B40000808000020002300260029002C002F0058
:105B500032000001000003010601090100002200DB
:105B6000250028002B002E00310034000201000027
:105B7000050108010B0100002100240027002A0074
:105B80002D003000330001010000040107010A016B
:105B9000024E414E494E495459494E46CDCCCC3D1A
:105BA0000AD7233C17B7D13877CC2B329595E6240A
:105BB0001FB14F0A000020410000C84200401C46AF
:105BC00020BCBE4CCA1B0E5AAEC59D7400407A1054
:105BD000F35A00A0724E18090010A5D4E80000E89E
:105BE0007648170000E40B54020000CA9A3B0000FC
:105BF00000E1F505000080969800000040420F008B
:105C00000000A08601000000102700000000E8034B
:105C1000000000006400000000000A000000000016
:105C20000100000000002C76D888DC674F0823DFD5
:105C3000C1DFAE59E1B1B796E5E3E453C63AE651A8
:105C4000997696E8E6C28426EB898C9B62ED407CCF
:105C50006FFCEFBC9C9F40F2BAA56FA5F490055A6B
:105C60002AF75C936B6CF9676DC11BFCE0E40D4790
:105C7000FEF520E6B500D0ED902E030094357705B3
:105C80000080841E080000204E0A000000C80C336B
:105C90003333330F986E12831141EF8D2114893BFA
:105CA000E65516CFFEE6DB18D1844B381BF77C1D7A
:105CB000901DA4BBE424203284725E228100C9F1CD
:105CC00024ECA1E53D276CA311CAB0FBBD01B101D5
:105CD0009DA311241FBECFEFD1E2DEBFCDBF00E0F8
:105CE0000CBF19E0A0E0B2E0ECE7FAE903E00BBF7B
:105CF00002C007900D92AE37B107D9F72BE1AEE79E
:105D0000B9E001C01D92AC3FB207E1F71CE5C0ED60
:105D1000DCE500E006C022970109FE010BBF0F94ED
:105D2000E1C2C63CD10780E00807A9F70F94B9BCCF
:105D30000D942CCD0C940000CF92DF92EF92FF9245
:105D40000F931F93CF93DF938C01D42EC62FD72FA1
:105D5000D60EDC1671F1F801E080F180C990C70120
:105D60000F941FCAC816F1F06C2DC7010F944FCACB
:105D7000C7010F941FCA8C15A9F0E2EBF7E08491DC
:105D8000882341F09091C00095FFFCCF8093C6001E
:105D90003196F5CF8091C00085FFFCCF8AE08093DB
:105DA000C60007C0F80180819181019691838083AC
:105DB000D0CFDF91CF911F910F91FF90EF90DF90A7
:105DC000CF900895EF92FF920F931F93CF93DF939D
:105DD0001F92CDB7DEB78C017B01460FF8018081A1
:105DE000918149830F941FCAF70181937F01F801C4
:105DF0008081918101969183808349814E11EECFFC
:105E00000F90DF91CF911F910F91FF90EF90089528
:105E1000FF920F931F93CF93DF93CDB7DEB72C97ED
:105E20000FB6F894DEBF0FBECDBF8C01F62E80E317
:105E300090E3A0E3B0E08D839E83AF83B8871C8797
:105E40000B8744E0BE016B5F7F4FCE010B9674DF82
:105E500040E160E479E1CE010B966EDF40E160E560
:105E600079E1CE010B9668DF40E160E379E1CE0194
:105E70000B9662DF44E068E279E1CE010B965CDFCD
:105E800044E064E279E1CE010B9656DF44E06CE237
:105E900079E1CE010B9650DF44E060E179E1CE017B
:105EA0000B964ADF44E060E679E1CE010B9644DFD1
:105EB00044E064E179E1CE010B963EDF44E068E125
:105EC00079E1CE010B9638DF44E06CE179E1CE0157
:105ED0000B9632DF44E060E279E1CE010B962CDFD5
:105EE0004CE064ED7AE0CE010B9626DF44E06DECE9
:105EF0007AE0CE010B9620DF44E06DEA72E0CE013D
:105F00000B961ADF44E069EA72E0CE010B9614DFCB
:105F100044E065EA72E0CE010B960EDF44E06DE9E5
:105F200072E0CE010B9608DF44E069E972E0CE0131
:105F30000B9602DF44E065E972E0CE010B96FCDED1
:105F400080E290E09A87898742E0BE01675F7F4FD9
:105F5000CE010B96F1DE41E069EC7AE0CE010B96C2
:105F6000EBDE44E064E272E0CE010B96E5DE44E055
:105F70006CE172E0CE010B96DFDE44E064EC7AE087
:105F8000CE010B96D9DE44E060EC7AE0CE010B96B0
:105F9000D3DE44E068E172E0CE010B96CDDE41E055
:105FA00060EF7AE0CE010B96C7DE44E064E472E075
:105FB000CE010B96C1DE89E08F1560F444E06FE5F9
:105FC00073E1CE010B96B8DE44E06BE573E1CE01E0
:105FD0000B96B2DE46E551E360E070E049835A83F8
:105FE0006B837C831C870B8744E0BE016F5F7F4F10
:105FF000CE010B96A1DEE5E2F0E18491882341F029
:106000009091C00095FFFCCF8093C6003196F5CFEC
:10601000E2EAF7E08491882341F09091C00095FF77
:10602000FCCF8093C6003196F5CF8091C00085FFEC
:10603000FCCF8AE08093C6002C960FB6F894DEBFA2
:106040000FBECDBFDF91CF911F910F91FF900895AB
:106050001F93CF93DF93182FC5E2D0E1FE01849107
:10606000882341F09091C00095FFFCCF8093C6003B
:106070003196F5CFE2E9F7E08491882341F09091E1
:10608000C00095FFFCCF8093C6003196F5CF80917C
:10609000C00085FFFCCF8AE08093C600FE0184919A
:1060A000E5E2F0E1882349F09091C00095FFFCCF34
:1060B0008093C60031968491F5CF4091401950915C
:1060C000411960914219709143198AE897E00E9442
:1060D0003B4840914419509145196091461970917F
:1060E000471987E897E00E943B4840914819509132
:1060F000491960914A1970914B1984E897E00E9400
:106100003B4840914C1950914D1960914E19709136
:106110004F1981E897E00E943B488091C00085FFBD
:10612000FCCF8AE08093C600FE018491E5E2F0E1B5
:10613000882349F09091C00095FFFCCF8093C60062
:1061400031968491F5CFE7E6F7E08491882341F01A
:106150009091C00095FFFCCF8093C6003196F5CF9B
:106160008091C00085FFFCCF8AE08093C600FE01CD
:106170008491E5E2F0E1882349F09091C00095FF19
:10618000FCCF8093C60031968491F5CF4091501991
:106190005091511960915219709153198EE597E001
:1061A0000E943B48409154195091551960915619DD
:1061B000709157198BE597E00E943B484091581920
:1061C0005091591960915A1970915B1988E597E0BF
:1061D0000E943B4840915C1950915D1960915E1995
:1061E00070915F1985E597E00E943B488091C0005F
:1061F00085FFFCCF8AE08093C600FE018491E5E232
:10620000F0E1882349F09091C00095FFFCCF809386
:10621000C60031968491F5CFE7E3F7E084918823B7
:1062200041F09091C00095FFFCCF8093C60031965D
:10623000F5CF8091C00085FFFCCF8AE08093C60037
:10624000FE018491E5E2F0E1882349F09091C000DD
:1062500095FFFCCF8093C60031968491F5CF409195
:1062600030195091311960913219709133198EE2C1
:1062700097E00E944C484091341950913519609133
:106280003619709137198BE297E00E944C48409183
:1062900038195091391960913A1970913B1988E277
:1062A00097E00E944C4840913C1950913D196091F3
:1062B0003E1970913F1985E297E00E944C48809109
:1062C000C00085FFFCCF8AE08093C600FE01849168
:1062D000E5E2F0E1882349F09091C00095FFFCCF02
:1062E0008093C60031968491F5CFE0EFF6E084917B
:1062F000882341F09091C00095FFFCCF8093C600A9
:106300003196F5CF8091C00085FFFCCF8AE0809365
:10631000C600FE018491E5E2F0E1882349F0909106
:10632000C00095FFFCCF8093C60031968491F5CFD5
:10633000409128195091291960912A1970912B19AF
:1063400087EE96E00E943B48409124195091251910
:10635000609126197091271984EE96E00E943B48BF
:106360008091C00085FFFCCF8AE08093C600FE01CB
:106370008491E5E2F0E1882349F09091C00095FF17
:10638000FCCF8093C60031968491F5CFE1E3F6E02F
:106390008491882341F09091C00095FFFCCF8093B9
:1063A000C6003196F5CF8091C00085FFFCCF8AE012
:1063B0008093C600FE018491E5E2F0E1882349F074
:1063C0009091C00095FFFCCF8093C60031968491D8
:1063D000F5CF40912C1950912D1960912E19709183
:1063E0002F1988E296E00E943B4840911019509185
:1063F0001119609112197091131985E296E00E94AB
:106400003B484091601950916119609162197091F7
:10641000631982E296E00E944C4840911419509111
:10642000151960911619709117198FE196E00E9465
:106430003B48409118195091191960911A1970919F
:106440001B198CE196E00E943B4840911C19509129
:106450001D1960911E1970911F1989E196E00E9423
:106460003B48409120195091211960912219709157
:10647000231986E196E00E943B488091C00085FF89
:10648000FCCF8AE08093C600FE018491E5E2F0E152
:10649000882349F09091C00095FFFCCF8093C600FF
:1064A00031968491F5CFE4E0F6E08491882341F0C1
:1064B0009091C00095FFFCCF8093C6003196F5CF38
:1064C0008091C00085FFFCCF8AE08093C600FE016A
:1064D0008491E5E2F0E1882349F09091C00095FFB6
:1064E000FCCF8093C60031968491F5CF4091D40AB9
:1064F0005091D50A6091D60A7091D70A8BEF95E03A
:106500000E943B484091D80A5091D90A6091DA0A1A
:106510007091DB0A88EF95E00E943B484091DC0ACD
:106520005091DD0A6091DE0A7091DF0A85EF95E0F7
:106530000E943B488091C00085FFFCCF8AE0809399
:10654000C600FE018491E5E2F0E1882349F09091D4
:10655000C00095FFFCCF8093C60031968491F5CFA3
:10656000E7EEF5E08491882341F09091C00095FF1B
:10657000FCCF8093C6003196F5CF8091C00085FF97
:10658000FCCF8AE08093C600FE018491E5E2F0E151
:10659000882349F09091C00095FFFCCF8093C600FE
:1065A00031968491F5CF4091AD025091AE02609149
:1065B000AF027091B0028DED95E00E943B48609172
:1065C000A9027091AA028091AB029091AC020F9443
:1065D0005C37AB01BC018AED95E00E943B486091BD
:1065E000A5027091A6028091A7029091A8020F9433
:1065F0006837AB01BC0187ED95E00E943B48809174
:10660000C00085FFFCCF8AE08093C600FE01849124
:10661000E5E2F0E1882349F09091C00095FFFCCFBE
:106620008093C60031968491F5CFE1ECF5E084913A
:10663000882341F09091C00095FFFCCF8093C60065
:106640003196F5CF8091C00085FFFCCF8AE0809322
:10665000C600FE018491E5E2F0E1882349F09091C3
:10666000C00095FFFCCF8093C60031968491F5CF92
:1066700040919D0250919E0260919F027091A002F4
:1066800087EB95E00E943B486091990270919A02D5
:1066900080919B0290919C020F945C37AB01BC01EE
:1066A00084EB95E00E943B486091950270919602C0
:1066B00080919702909198020F946837AB01BC01CA
:1066C00081EB95E00E943B488091C00085FFFCCFA4
:1066D0008AE08093C600FE018491E5E2F0E1882320
:1066E00049F09091C00095FFFCCF8093C600319691
:1066F0008491F5CFEDE7F5E08491882341F0909106
:10670000C00095FFFCCF8093C6003196F5CF8091F5
:10671000C00085FFFCCF8AE08093C600FE01849113
:10672000E5E2F0E1882349F09091C00095FFFCCFAD
:106730008093C60031968491F5CF40912402509108
:106740002502609126027091270283E795E00E945E
:106750003B4820E030E040E752E460911C02709139
:106760001D0280911E0290911F020F9476C0AB0112
:10677000BC0180E795E00E943B484091C40A5091DB
:10678000C50A6091C60A7091C70A8DE695E00E941D
:106790003B488091C00085FFFCCF8AE08093C60013
:1067A000FE018491E5E2F0E1882349F09091C00078
:1067B00095FFFCCF8093C60031968491F5CFE1E43C
:1067C000F5E08491882341F09091C00095FFFCCFC3
:1067D0008093C6003196F5CF8091C00085FFFCCF35
:1067E0008AE08093C600FE018491E5E2F0E188230F
:1067F00049F09091C00095FFFCCF8093C600319680
:106800008491F5CF4091C00A5091C10A6091C20AAB
:106810007091C30A87E395E00E943B4820E030E096
:1068200040E752E4609118027091190280911A02B7
:1068300090911B020F9476C0AB01BC0184E395E0FC
:106840000E943B488091C00085FFFCCF8AE0809386
:10685000C600FE018491E5E2F0E1882349F09091C1
:10686000C00095FFFCCF8093C60031968491F5CF90
:10687000EAEDF4E08491882341F09091C00095FF07
:10688000FCCF8093C6003196F5CF8091C00085FF84
:10689000FCCF8AE08093C600FE018491E5E2F0E13E
:1068A000882349F09091C00095FFFCCF8093C600EB
:1068B00031968491F5CF4091C90A50E060E070E0D4
:1068C00080ED94E00E944C488091C00085FFFCCF91
:1068D0008AE08093C600FE018491E5E2F0E188231E
:1068E00049F09091C00095FFFCCF8093C60031968F
:1068F0008491F5CF8091F00A8823A1F1EDEBF4E0CB
:106900008491882341F09091C00095FFFCCF809343
:10691000C6003196F5CF8091C00085FFFCCF8AE09C
:106920008093C600FE018491E5E2F0E1882349F0FE
:106930009091C00095FFFCCF8093C6003196849162
:10694000F5CF40914402509145026091460270910A
:10695000470283EB94E00E943B488091C00085FF92
:10696000FCCF11C0E7E9F4E08491882341F09091D5
:10697000C00095FFFCCF8093C6003196F5CF809183
:10698000C00085FFFCCF8AE08093C6001A3008F46F
:106990003EC0FE01C491E5E2F0E1CC2349F08091D4
:1069A000C00085FFFCCFC093C6003196C491F5CFDF
:1069B000EEE7F4E08491882341F09091C00095FFC8
:1069C000FCCF8093C6003196F5CF8091C00085FF43
:1069D000FCCF8AE08093C60040915F135091601312
:1069E000609161137091621384E794E00E943B48C8
:1069F00040915B1350915C1360915D1370915E1335
:106A00008AE694E0DF91CF911F910C943B48DF918F
:106A1000CF911F910895AF92BF92CF92DF92EF92E4
:106A2000FF920F931F93CF93DF93CDB7DEB7E0971D
:106A30000FB6F894DEBF0FBECDBF80E1E3EEF2E00B
:106A4000DE01919601900D928A95E1F780E1E3EFE6
:106A5000F2E0DE01519601900D928A95E1F780E116
:106A6000E3E0F3E0DE01119601900D928A95E1F7E3
:106A70006E0181E2C80ED11C80E4E82E89E1F82E77
:106A80008E010F5E1F4F60E579E1AE014F5F5F4FF2
:106A900090E3A92E99E1B92E20E030E0F601819132
:106AA0009191A191B1916F01F70181939193A1937C
:106AB000B1937F01F80181919191A191B1918F01E1
:106AC000FB0181939193A193B193BF01FA0181914D
:106AD0009191A191B191AF01F50181939193A1930E
:106AE000B1935F012F5F3F4F24303105B9F60F940A
:106AF000BE1380E090E4ACE9B4E48093281990934D
:106B00002919A0932A19B0932B19809324199093D3
:106B10002519A0932619B093271910922C191092B9
:106B20002D1910922E1910922F1980E29EE4A0E0E8
:106B3000B0E08093601990936119A0936219B093AB
:106B400063191092101910921119109212191092C3
:106B5000131980E090E0A0E7B1E4809314199093BA
:106B60001519A0931619B0931719809318199093BB
:106B70001919A0931A19B0931B198DEC9CECACEC6D
:106B8000BEE380931C1990931D19A0931E19B09316
:106B90001F1980E090E0A0E2B0E480932019909368
:106BA0002119A0932219B09323191092DC0A109294
:106BB000DD0A1092DE0A1092DF0A1092D80A1092B3
:106BC000D90A1092DA0A1092DB0A1092D40A1092B3
:106BD000D50A1092D60A1092D70A8DE39AE0A1E85E
:106BE000B1E48093AD029093AE02A093AF02B09354
:106BF000B0026DEC7CEC84E99FE30F945637609310
:106C0000A9027093AA028093AB029093AC0265E84C
:106C10007BEE80E692E40F9462376093A502709356
:106C2000A6028093A7029093A8020F942D2680E0DD
:106C300090E0A0E8BFE38093A1029093A202A0930A
:106C4000A302B093A4021092C90A80E090E0A0E4ED
:106C5000B0E48093240290932502A0932602B0937F
:106C6000270240E050E064E372E440931C0250933A
:106C70001D0260931E0270931F021092C40A1092AC
:106C8000C50A1092C60A1092C70A1092C00A109242
:106C9000C10A1092C20A1092C30A40E050E060E0BC
:106CA00071E4409318025093190260931A02709392
:106CB0001B021092F00A8093440290934502A09325
:106CC0004602B09347020E94BF5EE5E2F0E1849184
:106CD000882341F09091C00095FFFCCF8093C600BF
:106CE0003196F5CFEEE2F4E08491882341F0909163
:106CF000C00095FFFCCF8093C6003196F5CF809100
:106D0000C00085FFFCCF8AE08093C600E0960FB6F6
:106D1000F894DEBF0FBECDBFDF91CF911F910F91D1
:106D2000FF90EF90DF90CF90BF90AF9008951F93AA
:106D3000CF93DF93CDB7DEB72C970FB6F894DEBFB5
:106D40000FBECDBF162F9C878B8786E591E3A0E011
:106D5000B0E089839A83AB83BC8344E0BE016B5F60
:106D60007F4FCE010B962ED843E050E0BE016B5F03
:106D70007F4FCE0101960F9483C6892B09F0FFC087
:106D800040E160E479E1CE010B961CD840E160E57A
:106D900079E1CE010B9616D840E160E379E1CE01AE
:106DA0000B9610D80F94BE1344E068E279E1CE014F
:106DB0000B9608D844E064E279E1CE010B9602D844
:106DC00044E06CE279E1CE010B960E94E22E44E0B1
:106DD00060E179E1CE010B960E94E22E44E060E68C
:106DE00079E1CE010B960E94E22E44E064E179E164
:106DF000CE010B960E94E22E44E068E179E1CE01DB
:106E00000B960E94E22E44E06CE179E1CE010B96F4
:106E10000E94E22E44E060E279E1CE010B960E94EE
:106E2000E22E4CE064ED7AE0CE010B960E94E22E59
:106E300044E06DEC7AE0CE010B960E94E22E44E035
:106E40006DEA72E0CE010B960E94E22E44E069EA00
:106E500072E0CE010B960E94E22E44E065EA72E0F9
:106E6000CE010B960E94E22E44E06DE972E0CE0165
:106E70000B960E94E22E44E069E972E0CE010B9687
:106E80000E94E22E44E065E972E0CE010B960E947A
:106E9000E22E42E0BE01675F7F4FCE010B960E945B
:106EA000E22E41E069EC7AE0CE010B960E94E22EE0
:106EB00044E064E272E0CE010B960E94E22E44E0D0
:106EC0006CE172E0CE010B960E94E22E44E064EC8D
:106ED0007AE0CE010B960E94E22E44E060EC7AE06C
:106EE000CE010B960E94E22E44E068E172E0CE01F2
:106EF0000B960E94E22E41E060EF7AE0CE010B9605
:106F00000E94E22E44E064E472E0CE010B960E94FF
:106F1000E22E1A3070F044E06FE573E1CE010B967B
:106F20000E94E22E44E06BE573E1CE010B960E94D5
:106F3000E22E0E94BF5E0F942D26E5E2F0E18491DF
:106F4000882341F09091C00095FFFCCF8093C6004C
:106F50003196F5CFE0E5F4E08491882341F09091FB
:106F6000C00095FFFCCF8093C6003196F5CF80918D
:106F7000C00085FFFCCF8AE08093C60001C04BDDD6
:106F80002C960FB6F894DEBF0FBECDBFDF91CF9128
:106F90001F910895682F772767FD709580914310A2
:106FA00090914410885B9F4E0F9468C690933A105E
:106FB0008093391021E0892B09F420E0822F089575
:106FC0008091391090913A1060E070E001960D9434
:106FD00011C3282F6091F61B7091F71B90E02A30A7
:106FE00018F0895A9F4F01C0C0960D94D6C6CF9312
:106FF000C82F82958F70EDDF8C2F8F70CF91E9CFE6
:10700000CF93C82F892FF3DF8C2FCF91F0CF6F92C2
:107010007F928F929F92AF92BF92CF92DF92EF9228
:10702000FF920F931F93CF93DF936B017C01EA01D3
:10703000122F209709F455C0123011F48E2DC9DF9C
:10704000C601DEDF6091F61B7091F71B80E290E0D5
:107050000F94D6C6702E7C1A8C2F870D09F438C079
:107060001130D1F088F0123029F5460157018FEF29
:10707000881A980AA80AB80AEE24D7FCE094FE2CD5
:10708000EBBEF601679013C0F60160808FEFC81A5F
:10709000D80AE80AF80A0FC0460157018FEF881A8C
:1070A000980AA80AB80AC6010F941FCA682E75016B
:1070B000640101C0612C6091F61B7091F71B80E2A6
:1070C00090E00F94D6C6862D92DF219709F0C4CFA9
:1070D0006091F61B7091F71B8AE090E00F94D6C682
:1070E000A8CFDF91CF911F910F91FF90EF90DF908C
:1070F000CF90BF90AF909F908F907F906F900895AA
:10710000CF93DF93FB0120E030E0DC01ED018D91B6
:107110008823A1F14115510519F02417350774F59D
:107120008032A1F38A3051F190ED980F9A3020F41B
:10713000682F6295607F08C09FE9980F9630A8F489
:10714000682F6295607F6057CE0102967981A0ED2D
:10715000A70FAA3018F4762F7A2B0CC0AFE9A70F2F
:10716000A63018F47755762B05C088279927821BFF
:10717000930B05C071932F5F3F4FC7CFC901DF91BC
:10718000CF9108958BE693E00F9469C7F894FFCFF1
:10719000E0913910F0913A108181882399F082E4CE
:1071A000F9DE882369F0F89428E088E190E00FB6D2
:1071B000F894A895809360000FBE20936000FFCFE5
:1071C0000C9400000895F894C0E0D0E06FEFCE0179
:1071D0000F944FCA2196C11580E2D807B9F728E06D
:1071E00088E190E00FB6F894A895809360000FBEF8
:1071F00020936000FFCF0F931F93CF93DF93CDB702
:10720000DEB762970FB6F894DEBF0FBECDBF81E444
:10721000C1DE8823A9F08091391090913A10FC01C9
:107220002181283741F440E150E060E070E00296AF
:107230000F9479C403C0C4DE0F9410BE8B0102C04A
:1072400000E010E083E4A6DE882331F0B9DE0F947D
:1072500010BE262F872F02C020E080E21F71422F30
:10726000582F4130F0E25F0710F040E050E2CA01D1
:10727000800F911F8130904220F040E050E2401B8F
:10728000510B88E5498B5A8B85DE49895A898823B9
:10729000D1F08091391090913A1040E150E0BE0158
:1072A0006F5F7F4F01962CDFAC01009761F0FE010C
:1072B0003196CF01840F951FD801E817F90719F00F
:1072C00021912D93FACFB80180E090E000E120E019
:1072D0009EDE62960FB6F894DEBF0FBECDBFDF9183
:1072E000CF911F910F910895AF92BF92CF92DF92ED
:1072F000EF92FF920F931F93CF93DF93CDB7DEB73B
:1073000060970FB6F894DEBF0FBECDBF81E442DEBA
:107310008823A9F08091391090913A10FC012181C5
:10732000283741F440E150E060E070E002960F94AD
:1073300079C403C045DE0F9410BE8B0102C000E08B
:1073400010E083E427DE882331F03ADE0F9410BE8C
:10735000262F872F02C020E080E21F71E22EF82E38
:10736000F1E0EF16F0E2FF0618F0E12C90E2F92EC2
:10737000C701800F911F8130904228F0E12C80E2FC
:10738000F82EE01AF10A88E505DE882361F1809184
:10739000391090913A1040E150E0BE016F5F7F4F8D
:1073A0000196AEDE7C010097F1F0CE0101965C0102
:1073B000C12CD12CCE14DF0461F0F50161915F0185
:1073C000C601800F911F0F944FCAFFEFCF1ADF0A3B
:1073D000F1CFC80115DE6091F61B7091F71B8AE0B2
:1073E00090E00F94D6C6B80180E090E000E121E083
:1073F000A7010DDE60960FB6F894DEBF0FBECDBFBD
:10740000DF91CF911F910F91FF90EF90DF90CF9080
:10741000BF90AF900895CF92DF92EF92FF9280E5F8
:10742000B9DD882309F44CC0CBDD0F9410BE6B018D
:107430007C018FEFC816D10411F008F041C086E43A
:10744000A9DD882379F0BCDD0F9410BE61157105AC
:1074500011F460E004C06130710521F461E08C2D0D
:107460000F94B5B686E596DD882399F0A9DD0F94D3
:1074700010BE6115710511F460E004C06130710542
:10748000F9F461E08C2DFF90EF90DF90CF900D9498
:10749000EEB68C2D0F9423B721E0892B09F420E060
:1074A0001F922F93DF92CF928EE793E09F938F935B
:1074B0000F9435C70F900F900F900F900F900F9073
:1074C000FF90EF90DF90CF900895089508954F9228
:1074D0005F926F927F929F92AF92BF92CF92DF9214
:1074E000EF92FF920F931F93CF93DF9382E398E085
:1074F0009F938F930F9446C786EA9FE00F941FCA0D
:10750000C82FC090691AD0906A1AE0906B1AF09058
:107510006C1AC701B6010E9475642B013C01E09111
:107520003910F0913A1092810F900F909F3311F023
:1075300091114CC091E0C11101C090E01F929F9346
:1075400083E298E09F938F930F9446C70F900F901C
:107550000F900F9000EB1FE0C3E2D0E0912C80E091
:1075600090E023E0A22E28E0B22EBC0180E090E063
:107570000F9441BE209148193091491940914A1900
:1075800050914B190F94A8BD20E030E04AE754E435
:107590000F9476C00F9415BE7F936F93DF93CF93B4
:1075A000BF92AF920F9446C793940F900F900F9095
:1075B0000F900F900F9086E0981609F441C0C80113
:1075C0000F942CCA25960E5F1F4FCFCF913221F515
:1075D00061E086EA9FE00F944FCA68E070E080EBBC
:1075E0009FE00F945DCA68E170E082EB9FE00F942A
:1075F0005DCA60E370E084EB9FE00F945DCA60E5D4
:1076000070E086EB9FE00F945DCA68E770E088EB5E
:107610009FE00F945DCA14C080E5BCDC882319F09C
:10762000CFDC6B017C01C701B6010E9475642B01A0
:107630003C018AE5AFDC882319F0C2DC2B013C0158
:1076400020E030E04AE754E4C301B2010F9476C071
:107650000F9410BECB0168EE73E00F9465C29F9348
:107660008F93C301B2010F9410BE7F936F93C70134
:10767000B6010F9410BE7F936F9383EE97E09F93B4
:107680008F930F9446C78DB79EB708960FB6F894A0
:107690009EBF0FBE8DBFDF91CF911F910F91FF90C5
:1076A000EF90DF90CF90BF90AF909F907F906F90C2
:1076B0005F904F90089566EE87EF9FE00D9431CA7A
:1076C00060E086E69FE00F9431CA60E085E69FE0C7
:1076D0000F9431CA60E084E69FE00D9431CA6F9246
:1076E0007F928F929F92AF92BF92CF92DF92EF9252
:1076F000FF920F931F93CF93DF9382ED97E09F93B9
:107700008F930F9446C788E545DC0F900F90811149
:1077100007C089E53FDC882309F4AAC0C1E001C0A5
:10772000C0E06C2E712CC3010E944A4D8C2F0F9427
:10773000273880E1E0EEFAE0ABEABAE001900D9282
:107740008A95E1F7660C771C660C771CC30185559A
:10775000954F3C0180E090E0A8E4B3E4F30180831E
:107760009183A283B38320E030E040E752E460914C
:1077700058027091590280915A0290915B020F94C5
:10778000A8BD4B015C01E090B30AF090B40A0091EF
:10779000B50A1091B60A2091AF0A3091B00A409113
:1077A000B10A5091B20A6091AB0A7091AC0A809113
:1077B000AD0A9091AE0ACCECDAE0DF93CF93E7EB21
:1077C000CE2EEAE0DE2E0F9433050F94E21E80E108
:1077D000E0EEFAE0ABEABAE001900D928A95E1F7AB
:1077E000F301108211821282138220E030E040E720
:1077F00052E4609158027091590280915A0290911E
:107800005B020F94A8BD4B015C01E090B30AF090BD
:10781000B40A0091B50A1091B60A2091AF0A3091CE
:10782000B00A4091B10A5091B20A6091AB0A7091CE
:10783000AC0A8091AD0A9091AE0ADF93CF930F947A
:1078400033050F94E21E0F9436382FEF2093B202C7
:107850009F938F938FEB97E09F938F930F9446C7DF
:107860008DB79EB708960FB6F8949EBF0FBE8DBF1A
:10787000DF91CF911F910F91FF90EF90DF90CF900C
:10788000BF90AF909F908F907F906F900895E09100
:107890003910F0913A1085818F3311F081112BC08E
:1078A00080913C131F928F9380913D131F928F9371
:1078B00080913F138F9380913E138F93809141135A
:1078C0008F93809140138F93809142131F928F93D7
:1078D000809143131F928F9387E893E09F938F9338
:1078E0000F9435C78DB79EB70E960FB6F8949EBF0E
:1078F0000FBE8DBF0895813229F50E9446FF809109
:107900003C131F928F9380913D131F928F93809110
:107910003F138F9380913E138F93809141138F93E8
:10792000809140138F9389E993E09F938F930F94F5
:1079300035C78DB79EB70A960FB6F8949EBF0FBE97
:107940008DBF089582E526DB81113ADB88E522DBD5
:10795000882339F035DB0F9410BE70934113609388
:10796000401389E517DB882339F02ADB0F9410BE1A
:1079700070933F1360933E138CE40CDB882329F053
:107980001FDB0F9410BE609368020895CF93DF93BE
:10799000EC0160E08E810F94EEB681E090E00F94F0
:1079A00030B561E08E810F94EEB681E090E00F94E7
:1079B00030B560E08E810F94EEB684E690E0DF9102
:1079C000CF910D9430B5CF92DF92EF92FF920F934B
:1079D0001F93CF93DF937C01C0E0D0E0C62ED12C63
:1079E00087010C0F1D1F61E0F80187810F94B5B668
:1079F000B6010C2E02C0759567950A94E2F7617086
:107A0000F80187810F94EEB62196C430D10541F775
:107A1000C701DF91CF911F910F91FF90EF90DF9001
:107A2000CF90B4CFCF92DF92EF92FF920F931F933C
:107A3000CF93DF937C01C0E0D0E0C62ED12C87012C
:107A40000C0F1D1F61E0F80187810F94B5B6B601D8
:107A50000C2E02C0759567950A94E2F76170F801E3
:107A600087810F94EEB62196C830D10541F7C70142
:107A7000DF91CF911F910F91FF90EF90DF90CF900A
:107A800085CF1F93CF93DF93EC01162F642F8C814A
:107A90000F94EEB68D818F3F19F060E00F94EEB633
:107AA0008F85612F84FF05C0CE01DF91CF911F919B
:107AB000B9CF70E084E0759567958A95E1F7CE01BE
:107AC00082DF612FCE01DF91CF911F917CCF40E00B
:107AD000D8CF61E0FCDF80E496E00D9430B562E041
:107AE000F6DF80E496E00D9430B5CF93DF93CDB709
:107AF000DEB728970FB6F894DEBF0FBECDBF28E0E3
:107B0000E3E1F3E0DE01119601900D922A95E1F791
:107B1000FC012389421710F04FEF420FFE0131960E
:107B2000E40FF11DE40FF11D2081260F2068622F64
:107B300028960FB6F894DEBF0FBECDBFDF91CF9170
:107B4000C6CFFC016089262F2460208B6C60BFCFDC
:107B5000CF93DF93EC01423018F08F8588608F87D8
:107B60004B8B1C8A222329F0413019F48F858460C5
:107B70008F8780E593EC0F9430B560E08C810F9493
:107B8000EEB660E08E810F94EEB68D818F3F19F0D6
:107B900060E00F94EEB66F8564FD19C063E0CE011E
:107BA00012DF84E991E10F9430B563E0CE010BDF81
:107BB00084E991E10F9430B563E0CE0104DF86E9FA
:107BC00090E00F9430B562E0CE01FDDE13C060623C
:107BD000CE017DDF84E991E10F9430B56F8560625D
:107BE000CE0175DF86E990E00F9430B56F85606255
:107BF000CE016DDF6F856062CE0169DF8CE390E0BE
:107C00000F9430B584E0888BCE019BDF8CE390E04D
:107C10000F9430B5CE015DDF88EB9BE00F9430B55B
:107C200082E0898B66E0CE0152DF8CE390E00F9416
:107C300030B51D8ADF91CF9108956F927F928F9218
:107C4000AF92CF92EF920F931F93CF93DF93CDB765
:107C5000DEB73C01162F842F5E854F8538899989C0
:107C6000F301848325830683E782C086A18682860A
:107C7000538744873587968761E00F94B5B6F30143
:107C800085818F3F19F061E00F94B5B661E0F30193
:107C900086810F94B5B6112319F0F301178603C03E
:107CA00080E1F301878720E041E060E1C301DF91DB
:107CB000CF911F910F91EF90CF90AF908F907F90C9
:107CC0006F9046CF8F92AF92CF92EF920F93DC01DD
:107CD00013961C921E921297E2EBF3E0ED93FC9345
:107CE0001F921F921F921F928C2CAE2CC02EE22E40
:107CF000042F2FEF462F61E0A0DF0F900F900F9021
:107D00000F900F91EF90CF90AF908F900895CF93F9
:107D1000DF93EC01423018F08F8588608F874B8BA2
:107D20001C8A222329F0413019F48F8584608F87C3
:107D300080E593EC0F9430B560E08C810F94EEB643
:107D400060E08E810F94EEB68D818F3F19F060E078
:107D50000F94EEB66F8564FD19C063E0CE0133DE8B
:107D600084E991E10F9430B563E0CE012CDE84E923
:107D700091E10F9430B563E0CE0125DE86E990E015
:107D80000F9430B562E0CE011EDE13C06062CE01FA
:107D90009EDE84E991E10F9430B56F856062CE017B
:107DA00096DE86E990E00F9430B56F856062CE0173
:107DB0008EDE6F856062CE018ADE8CE390E00F94E8
:107DC00030B584E0888BCE01BCDE8CE390E00F946C
:107DD00030B5CE0184DE80E496E00F9430B582E0C9
:107DE000898B66E0CE0173DE8CE390E00F9430B5B2
:107DF00040E068E0CE0179DE6BEC78E0CE010F94D4
:107E000089B741E068E0CE0170DE6BEC78E0CE012E
:107E10000F9489B742E066E0CE0167DE69EC78E056
:107E2000CE01DF91CF910D9489B7FC0160896D7F00
:107E3000608B68604CCECF93DF93EC01262F8D8949
:107E40008230B0F0FE01E80FF11D658B3E8980EDB8
:107E5000860F8A3058F4316081E090E00D8802C0CE
:107E6000880F991F0A94E2F7382B01C03E7F3E8BA2
:107E70004D8981E0840F8D8B50E04830510508F02A
:107E8000B6C0FA01EE58FF4F0D94B6C22B3109F07F
:107E9000AEC0AEC01E8A2B3509F0A9C0A9C02233DE
:107EA00009F4A6C02F3309F4A3C08E897AC08F8944
:107EB000823331F08F3349F4223309F098C098C0EF
:107EC0002A3419F4CE0105DE92C08E8982FF8FC05C
:107ED0002B3309F066C08CC08F898F3341F4888DB5
:107EE000823309F084C0253309F081C081C08E89B6
:107EF00082FF7DC0988D9B3311F480FD79C083FF94
:107F000076C02B3309F073C073C04F894F3371F4BF
:107F1000888D823309F06BC0898D853309F067C085
:107F20002C3609F064C0CE0180DF61C08E8982FFEB
:107F30005EC0988D9B3339F484FF05C0283489F5E1
:107F40004053698D2CC083FF52C0998D9B3309F03B
:107F50004EC027C08E8982FF4AC0488D4B3361F4E2
:107F6000982F9073903341F4283431F44F89405363
:107F70006A8D6053898D32C083FF39C0998D9B33E0
:107F8000B1F585FF34C0283461F440538F89880FE0
:107F90008056982F990F990F980F490F6A8D60534B
:107FA00024C080FF24C024C08E89982F9C709C30F0
:107FB000F1F4998D9B33D9F480768036C1F428345E
:107FC000B1F4488D40538F89880F8056982F990FB0
:107FD000990F980F490F6B8D60538A8D880F8056CB
:107FE000982F990F990F980F690FCE017EDD1D8A8A
:107FF00081E090E0DF91CF910895CF92DF92EF92F0
:10800000FF920F931F93CF93DF931F921F92CDB7D1
:10801000DEB78C01677088E0689FB001112460644E
:10802000C80149835A8353DD4981C42E5A81D52E14
:10803000E12CF12CD6016D916D01D801ED91FC91EF
:108040000190F081E02DC8011995BFEFEB1AFB0AF2
:10805000E8E0EE16F10471F70F900F90DF91CF91E9
:108060001F910F91FF90EF90DF90CF900895FC014A
:108070002589211102C06B3109F4DDCE41E001DD1B
:1080800081E090E008951F920F920FB60F92112495
:108090000BB60F922F933F934F935F936F938F93F2
:1080A0009F93EF93FF938091C00084FF03C0809162
:1080B000C60019C06091C6002091FF093091000AE6
:1080C000C90101968F7799274091010A5091020AC0
:1080D0008417950741F0F901E158F64F60839093BA
:1080E000000A8093FF09FF91EF919F918F916F910B
:1080F0005F914F913F912F910F900BBE0F900FBE4C
:108100000F901F9018951F920F920FB60F92112487
:108110000BB60F922F933F934F935F936F938F9371
:108120009F93EF93FF938091030A813001F5809133
:10813000D00084FF03C08091D60019C06091D600A2
:108140002091FF093091000AC90101968F77992784
:108150004091010A5091020A8417950741F0F901F4
:10816000E158F64F60839093000A8093FF09FF91D6
:10817000EF919F918F916F915F914F913F912F91CF
:108180000F900BBE0F900FBE0F901F901895CF92BF
:10819000DF92EF92FF926A017B01411581EE580751
:1081A0006105710509F463C082E08093C00060E05E
:1081B00079E08DE390E0A70196010F949AC22150D7
:1081C000310941095109CA01B90122E030E040E01A
:1081D00050E00F949AC291E03093C5002093C40000
:1081E0008091C10080618093C1008091C10088604E
:1081F0008093C1008091C10080688093C10080910C
:10820000030A8130D1F5992341F082E08093D000B8
:1082100060E079E08DE390E006C01092D00060E865
:1082200074E88EE190E0A70196010F949AC2215064
:10823000310941095109CA01B90122E030E040E0A9
:1082400050E00F949AC23093D5002093D4008091CF
:10825000D10080618093D1008091D10088608093AB
:10826000D1008091D10080688093D10006C0109227
:10827000C00090E020E130E0AFCFFF90EF90DF90C2
:10828000CF9008952091010A3091020A8091FF0950
:108290009091000A8217930771F0F901E158F64FA7
:1082A00080812F5F3F4F2F7733273093020A20932F
:1082B000010A90E008958FEF9FEF08958091010AE1
:1082C0009091020A9093000A8093FF0908954F92BB
:1082D0005F926F927F928F929F92AF92BF92CF9256
:1082E000DF92EF92FF920F931F93CF93DF93CDB75F
:1082F000DEB7A0970FB6F894DEBF0FBECDBF5C010E
:108300004115510561057105E9F420E030E040E3D5
:1083100050E060E070E0A0960FB6F894DEBF0FBEAC
:10832000CDBFDF91CF911F910F91FF90EF90DF9024
:10833000CF90BF90AF909F908F907F906F905F9005
:108340004F905BC08E010F5F1F4FC12CD12C760167
:108350004801422E512C612C712C8FEFC81AD80A7B
:10836000E80AF80ACB01BA01A30192010F9478C27E
:10837000CA01F80161938F01A901BC0141155105A2
:108380006105710551F7F1E0CF1AD108E108F10854
:10839000F401EC0DFD1D80818A3010F440E301C032
:1083A00047E3480F552747FD5095652F752F20E06F
:1083B00030E0C50122D081E0C81AD108E108F108F7
:1083C000EFEFCE16DE06EE06FE0611F7A0960FB60C
:1083D000F894DEBF0FBECDBFDF91CF911F910F91FB
:1083E000FF90EF90DF90CF90BF90AF909F908F90D5
:1083F0007F906F905F904F9008952115310539F46B
:108400008091C00085FFFCCF4093C60008952A30BC
:10841000310509F43FC05BCF9A01462F552747FD30
:108420005095652F752FE9CFCF93DF93EC0120E0B6
:1084300030E04DE050E060E070E0DFDF20E030E071
:108440004AE050E060E070E0CE01DF91CF91D5CFFF
:10845000FB012191BF01222339F03091C00035FF8B
:10846000FCCF2093C600F4CFDFCF9A01AB01662783
:1084700057FD6095762FC1CFCF93DF93EC019A0122
:10848000AB01662757FD6095762FB7DFCE01DF91F0
:10849000CF91CACFCF92DF92EF92FF92CF93DF932B
:1084A000EC016A017B0177FF0FC020E030E04DE274
:1084B00050E060E070E0A1DFF094E094D094C094CC
:1084C000C11CD11CE11CF11C2AE0B701A601CE01A0
:1084D000DF91CF91FF90EF90DF90CF90F8CE2115F4
:1084E000310539F48091C00085FFFCCF4093C60070
:1084F0000895EDCECF93DF93EC019A01462F50E023
:1085000060E070E0ECDFCE01DF91CF918DCFCF93B3
:10851000DF93EC019A01AB0160E070E0E0DFCE0197
:10852000DF91CF9181CFCF93DF93EC01D8DFCE01E4
:10853000DF91CF9179CF8F929F92AF92BF92CF92DE
:10854000DF92EF92FF921F93CF93DF93EC016A01CA
:108550007B01122F20E030E0A901C701B6010F9482
:10856000A1BD87FF0CC020E030E04DE250E060E0AC
:1085700070E0CE0142DFF7FAF094F7F8F094B12CF6
:1085800060E070E080E09FE3B11641F020E030E071
:1085900040E251E40F94A8BDB394F6CF9B01AC0127
:1085A000C701B6010F94C8BC6B017C010F9415BEC6
:1085B0004B015C010F9441BE9B01AC01C701B601A8
:1085C0000F94C7BC6B017C012AE0B501A401CE0168
:1085D0007EDE112361F0EDECF5E08191882339F026
:1085E0009091C00095FFFCCF8093C600F6CF112379
:1085F00019F120E030E040E251E4C701B6010F94E8
:1086000076C06B017C010F9410BE4B01AA2497FC2D
:10861000A094BA2CB501A401CE013CDFC501B40180
:108620000F9443BE9B01AC01C701B6010F94C7BCB8
:108630006B017C011150DBCFDF91CF911F91FF9037
:10864000EF90DF90CF90BF90AF909F908F90089564
:1086500072CFCF93DF93EC016EDFCE01DF91CF912C
:10866000E3CE9091C00095FFFCCF8093C60080E0E0
:1086700090E00895FC01659175918591949108951C
:10868000EF92FF920F931F93CF93DF93EC01CC0FE8
:10869000DD1FCC0FDD1FCE018F5F9F4EEBDF9E01F4
:1086A0002052354F79018E010C52154FF80120816F
:1086B0003181428153810F94C8BCF701608371837B
:1086C00082839383CE01875E9F4ED4DF9E012C5C14
:1086D0003D4F7901F80120813181428153810F940E
:1086E000C8BCF7016083718382839383CE01835F6B
:1086F0009F4EC0DFC85DDD4FF8012081318142818E
:1087000053810F94C8BC688379838A839B83DF91EC
:10871000CF911F910F91FF90EF900895CF93C82FA5
:1087200040910C0250910D0260910E0270910F0267
:108730004093970A5093980A6093990A70939A0A03
:1087400020915602309157023093610B2093600BB9
:1087500024E630E030935702209356020F94CAB4B7
:108760006093920A7093930A8093940A9093950A67
:108770008C2FCF910D94671580E00F946715809131
:10878000970A9091980AA091990AB0919A0A8093B9
:108790000C0290930D02A0930E02B0930F028091F1
:1087A000600B9091610B90935702809356020F9447
:1087B000CAB46093920A7093930A8093940A909338
:1087C000950A0895682F772767FD7095809143106B
:1087D00090914410885B9F4E0F9468C690933A1016
:1087E0008093391021E0892B09F420E0822F08952D
:1087F0008091391090913A104AE050E060E070E0CA
:1088000001960F9479C4CB0108958091391090910D
:108810003A104AE050E060E070E001960D9479C4AF
:108820002091431030914410BC01C901885B9F4ED8
:108830000F94A0C690933A108093391021E0892BB1
:1088400009F420E0822F08950F931F93CF93DF93B5
:108850000091391010913A1065E470E0C8010F944E
:1088600068C6EC01009751F460E070E0C801019621
:10887000DF91CF911F910F910D9411C318828091B8
:10888000391090913A1060E070E001960F9411C396
:1088900025E42883DF91CF911F910F910895809156
:1088A000391090913A1060E070E001960D9411C378
:1088B0002F923F924F925F926F927F928F929F92F0
:1088C000AF92BF92CF92DF92EF92FF920F931F93DE
:1088D000CF93DF93CDB7DEB760970FB6F894DEBFC6
:1088E0000FBECDBF1C012A013B014801590120E008
:1088F00030E04CE052E4C301B2010F94C7BC25E55F
:1089000035E547E052E40F94A8BD6B017C010F945C
:108910007EBE0F9410BE8B0177FF12C020E030E0C6
:1089200040E85FE3C701B6010F94A4BF18160CF02E
:108930005DC0C12CD12CE0E8EE2EEFE3FE2E56C038
:1089400066307105DCF02AEA3AE24CE453E4C301F4
:10895000B2010F94C7BC25E535E547E052E40F941A
:10896000A8BD6B017C0120E030E0A9010F94A1BDFE
:1089700087FF3FC0C12CD12C76013BC0882777FDF3
:108980008095982F0F9443BE25E535E547E052E4E6
:108990000F9476C020E030E04CE052E40F94C8BC65
:1089A0009B01AC01C301B2010F94C7BC25E535E5BD
:1089B00047E052E40F94A8BD6B017C0120E030E059
:1089C000A9010F94A1BD87FD17C020E030E040E869
:1089D0005FE3C701B6010F94A4BF181684F4C12C3D
:1089E000D12C70E8E72E7FE3F72E09C000E010E0FD
:1089F00006C005E010E003C0C12CD12C760120E0B8
:108A000030E040EC50E4C501B4010F94C7BC2BEA40
:108A10003AEA42E052E40F94A8BD2B013C010F94C6
:108A20007EBE0F9410BE788B6F8777FF12C020E058
:108A300030E040E85FE3C301B2010F94A4BF181611
:108A40000CF05FC0412C512C60E8662E6FE3762E4F
:108A500058C0AF85B8891697E4F026E535E549E2B8
:108A600053E4C501B4010F94C7BC2BEA3AEA42E0D3
:108A700052E40F94A8BD2B013C0120E030E0A90195
:108A80000F94A1BD87FD40C0E5E0F0E0F88BEF87D3
:108A900046C0882777FD8095982F0F9443BE2BEA18
:108AA0003AEA42E052E40F9476C020E030E040EC35
:108AB00050E40F94C8BC9B01AC01C501B4010F94F4
:108AC000C7BC2BEA3AEA42E052E40F94A8BD2B015E
:108AD0003C0120E030E0A9010F94A1BD87FD1CC03E
:108AE00020E030E040E85FE3C301B2010F94A4BF8F
:108AF0001816ACF4412C512C50E8652E5FE3752E0E
:108B00000EC0188A1F860BC0412C512C320125E063
:108B100030E0388B2F8703C0412C512C3201A70144
:108B2000960160E070E080E89FE30F94C7BC698322
:108B30007A838B839C83C80101969E838D83AF8546
:108B4000B8891196BA87A987A301920160E070E005
:108B500080E89FE30F94C7BC6B877C878D879E87D7
:108B600047E02F853889429FF001439FF00D112483
:108B7000F887EF83E00FF11FEE0FFF1FEE0FFF1FCF
:108B8000E20DF31D218132814381548169817A8113
:108B90008B819C810F9476C04B015C01EF81F8853D
:108BA0008D819E81E80FF91FEE0FFF1FEE0FFF1F53
:108BB000E20DF31D2181328143815481C701B60149
:108BC0000F9476C09B01AC01C501B4010F94C8BCE1
:108BD0009B01AC016B857C858D859E850F9476C04D
:108BE0004B015C0127E0E985FA852E9FD0012F9F7C
:108BF000B00D1124B887AF83FD01E00FF11FEE0F18
:108C0000FF1FEE0FFF1FE20DF31D21813281438113
:108C1000548169817A818B819C810F9476C06983AC
:108C20007A838B839C83AF81B8858D819E81A80FC9
:108C3000B91FAA0FBB1FAA0FBB1FA20DB31D119610
:108C40002D913D914D915C911497C701B6010F9400
:108C500076C09B01AC0169817A818B819C810F94E4
:108C6000C8BC9B01AC01C301B2010F9476C09B014B
:108C7000AC01C501B4010F94C8BC60960FB6F8945E
:108C8000DEBF0FBECDBFDF91CF911F910F91FF903F
:108C9000EF90DF90CF90BF90AF909F908F907F909C
:108CA0006F905F904F903F902F9008954F925F92FA
:108CB0006F927F929F92AF92BF92CF92DF92EF928C
:108CC000FF920F931F93CF93DF937C015B018A0187
:108CD000E90190907612911014C0FC01808191817D
:108CE000A281B381FA0180839183A283B383FB01C4
:108CF00080819181A281B38188839983AA83BB8378
:108D00007FC091FE55C0FC01208131814281538199
:108D10006091661270916712809168129091691249
:108D20000F9476C02B013C01F501208131814281F5
:108D3000538160916A1270916B1280916C129091C4
:108D40006D120F9476C09B01AC01C301B2010F9468
:108D5000C8BCF8016083718382839383F70120810B
:108D600031814281538160916E1270916F128091B6
:108D70007012909171120F9476C06B017C01F50115
:108D800020813181428153816091721270917312FE
:108D900080917412909175120F9476C09B01AC0172
:108DA000C701B6010F94C8BC688379838A839B830B
:108DB00090FE26C020914E1230914F1240915012D9
:108DC00050915112F80160817181828193810F94D9
:108DD000C8BCF8016083718382839383209152120F
:108DE00030915312409154125091551268817981FB
:108DF0008A819B810F94C8BC688379838A839B8313
:108E0000DF91CF911F910F91FF90EF90DF90CF9066
:108E1000BF90AF909F907F906F905F904F9008951C
:108E20002F923F924F925F926F927F928F929F927A
:108E3000AF92BF92CF92DF92EF92FF920F931F9368
:108E4000CF93DF93CDB7DEB728970FB6F894DEBF88
:108E50000FBECDBF8C011B019E012F5F3F4FAE01A6
:108E60004B5F5F4F23DF20E030E0A9016D817E8101
:108E70008F8198850F94A1BD87FF07C01D821E8238
:108E80001F821886FF24F39401C0F12C20E030E00B
:108E900040E850EC69817A818B819C810F94A1BD5F
:108EA00087FF0AC080E090E0A0E8B0EC89839A8355
:108EB000AB83BC83FF24F39420E030E04FE753E41E
:108EC0006D817E818F8198850F94A4BF181654F40C
:108ED00080E090E0AFE7B3E48D839E83AF83B887F3
:108EE000FF24F39420E030E042E553E469817A8185
:108EF0008B819C810F94A4BF18164CF480E090E005
:108F0000A2E5B3E489839A83AB83BC8303C0FF20CB
:108F100009F483C0C980DA80EB80FC808D809E805C
:108F2000AF80B8847090761271100BC0F801808207
:108F30009182A282B382F101C082D182E282F38265
:108F40006AC070FE1CC020914E1230914F124091A9
:108F5000501250915112C501B4010F94C7BC4B017E
:108F60005C01209152123091531240915412509151
:108F70005512C701B6010F94C7BC6B017C0171FE8D
:108F80004AC0209156123091571240915812509178
:108F90005912C501B4010F9476C02B013C012091F8
:108FA0005A1230915B1240915C1250915D12C701D0
:108FB000B6010F9476C09B01AC01C301B2010F94BE
:108FC000C8BCF801608371838283938320915E1211
:108FD00030915F124091601250916112C501B4014D
:108FE0000F9476C04B015C012091621230916312A4
:108FF0004091641250916512C701B6010F9476C07A
:109000009B01AC01C501B4010F94C8BCF1016083A0
:10901000718382839383FF24F3948F2D28960FB658
:10902000F894DEBF0FBECDBFDF91CF911F910F919E
:10903000FF90EF90DF90CF90BF90AF909F908F9078
:109040007F906F905F904F903F902F900895CF93B7
:10905000DF931F92CDB7DEB7BE016F5F7F4F0F94D6
:10906000EB990F90DF91CF910895682F87EF9FE0E4
:109070000D9431CA0895FC012491222341F03091CE
:10908000C00035FFFCCF2093C6000196F4CF22E04C
:1090900030E08EE799E0DCCAFC012491222341F004
:1090A0003091C00035FFFCCF2093C6000196F4CF6D
:1090B0002AE030E08EE799E012CACF9366EB73E0C6
:1090C0008EE799E0C5D9C1E0C093B1026FEF89E6A0
:1090D0009FE00F9431CAC093DF02CF91089566ECF0
:1090E00073E08EE799E0B4D91092B10260E089E6AE
:1090F0009FE00F9431CA1092DF02089587ED93E04C
:109100009F938F930F9435C70F94E21E81E00F94C5
:10911000AC990F94415082E00F94E59686E69FE06B
:109120000F941FCA61E0680F86E69FE00F9431CA72
:1091300081E00F94AC9982E00F94E596E091300BBA
:10914000F0E0EE0FFF1FEE5FFF4B859194910F94BF
:10915000595161E080EE9FE00E94ECC261E08AED2F
:109160009FE00E94ECC20F900F9061E08CEC9FE0BA
:109170000C94ECC210926C0B60E08AE69BE00E94BB
:109180003EBC81E08093B1020895EF92FF920F936D
:109190001F93CF93DF931F92CDB7DEB789830F94D0
:1091A00041508981823009F468C0B4F5882309F4FC
:1091B00042C0813009F0F4C09FB7F8948091020159
:1091C0008460809302019FBFEFEFF1EE24E0E15055
:1091D000F0402040E1F700C000009FB7F894809174
:1091E00002018B7F809302019FBF40E050E0BA01F3
:1091F0008DEE9FE00F9443CA40E050E0BA0181EF4A
:109200009FE00F9443CA0F90DF91CF911F910F9170
:10921000FF90EF900D94E778833009F45CC08430C0
:1092200009F0BEC00F90DF91CF911F910F91FF9079
:10923000EF900D9462A29FB7F89480910201846030
:10924000809302019FBF2FEF81EE94E02150804078
:109250009040E1F700C000009FB7F89480910201B0
:109260008B7F809302019FBF0F90DF91CF911F9161
:109270000F91FF90EF900D94EA500F94EA5080EF19
:10928000F4DE1092911B1092901B6091921B84EC63
:109290009FE00F9431CA60E97BE181EC9FE00F947D
:1092A0006F509FB7F894809102018460809302010F
:1092B0009FBF8FEF91EEE4E081509040E040E1F7F6
:1092C00000C000009FB7F894809102018B7F8093CB
:1092D00002019FBF65C08EEB9FE00F9452674DEA7D
:1092E0005FE062E081E00F942B7D9FB7F89480915E
:1092F00002018460809302019FBFFFEF21EE84E0B2
:10930000F15020408040E1F700C000009FB7F89482
:10931000809102018B7F809302019FBF10927E0A91
:1093200010927D0A46EA5FE063E083E00F942B7DB4
:1093300040917D0A50917E0A63E083E00F944C5087
:10934000E12CF12C09E210E06FEFC7010F944FCA36
:10935000C701B8010F9465C2892BD9F480917D0AA9
:1093600090917E0A019690937E0A80937D0A4FE940
:109370005FE063E083E00F942B7D40917D0A509184
:109380007E0A63E083E00F944C508DE99FE00F94D8
:1093900052679FEFE91AF90AE114E0E1FE06A1F62F
:1093A0000F90DF91CF911F910F91FF90EF90089553
:1093B0006FE67AE08DE69FE00D9408C78F929F924A
:1093C000AF92BF92CF92DF92EF92FF928091921B69
:1093D00081119DC00F94CAB46B017C0120911002D1
:1093E000222309F48CC0409115025091160241309D
:1093F000510509F484C08091110290911202A0914C
:109400001302B091140246015701881A990AAA0A58
:10941000BB0A30E0A8EEB3E00F94BCC286169706F4
:10942000A806B9060CF473C04430510559F13CF458
:10943000423051050CF463C0E5E2F0E10EC0453066
:10944000510509F05CC0E5E2F0E142C09091C00036
:1094500095FFFCCF8093C600319684918111F6CFA1
:10946000EAE8FEE08491882341F09091C00095FFE6
:10947000FCCF8093C6003196F5CF8091C00085FF68
:10948000FCCF3AC0E5E2F0E18491882341F090916D
:10949000C00095FFFCCF8093C6003196F5CFE4E77E
:1094A000FEE08491882341F09091C00095FFFCCFAD
:1094B0008093C6003196F5CF8091C00085FFFCCF28
:1094C0001BC09091C00095FFFCCF8093C6003196E1
:1094D00084918111F6CFEDE5FEE08491882341F07F
:1094E0009091C00095FFFCCF8093C6003196F5CFD8
:1094F0008091C00085FFFCCF8AE08093C600C092B7
:109500001102D0921202E0921302F0921402FF9024
:10951000EF90DF90CF90BF90AF909F908F90089585
:1095200080E1E0EEFAE0ABEABAE001900D928A95B4
:10953000E1F708954F925F926F927F928F929F9280
:10954000AF92BF92CF92DF92EF92FF92CF93DF93D1
:1095500000D01F92CDB7DEB70F94E21E8BE432D954
:10956000882391F071D96B017C0120E030E0A901E2
:109570000F94A4BF87FD08C0C0925F13D092601300
:10958000E0926113F092621382E51CD9882359F0AE
:109590005BD96B017C0120E030E0A9010F94A1BDF3
:1095A00087FF83C006C0C12CD12CE0E8EE2EEFEB84
:1095B000FE2E84E407D9882321F046D94B015C01B3
:1095C00006C0812C912C70E8A72E7FEBB72E87E583
:1095D000F9D8882321F038D92B013C0106C0412C51
:1095E000512C60E8662E6FEB762E88E4EBD888234A
:1095F00031F02AD969837A838B839C8308C080E009
:1096000090E0A0E8BFEB89839A83AB83BC8320E022
:1096100030E0A901C501B4010F94A4BF87FD45C086
:1096200020E030E0A901C301B2010F94A4BF87FD7F
:109630003CC020E030E0A90169817A818B819C8166
:109640000F94A4BF87FD31C020E030E0A901C5011F
:10965000B4010F94A1BD882391F120E030E040E0F7
:109660005FE3C501B4010F9476C06B017C012981D1
:109670003A814B815C81C301B2010F9476C04B01EA
:109680005C01A7019601C701B6010F9476C02BEDCE
:109690003FE049E450E40F9476C09B01AC01C50162
:1096A000B4010F94A8BD6B017C0120E030E0A9015A
:1096B000C701B6010F94A4BF87FF04C00BC0C12C23
:1096C000D12C7601C0925B13D0925C13E0925D13B3
:1096D000F0925E13E5E2F0E18491882341F09091ED
:1096E000C00095FFFCCF8093C6003196F5CFE6E130
:1096F000FBE08491882341F09091C00095FFFCCF5E
:109700008093C6003196F5CF40915F13509160135E
:10971000609161137091621322E030E08EE799E06E
:109720000E9428438091C00085FFFCCF8AE080938F
:10973000C600E0E1FBE08491882341F09091C000F5
:1097400095FFFCCF8093C6003196F5CFC0905B1398
:10975000D0905C13E0905D13F0905E1320E030E059
:10976000A901C701B6010F94A1BD882369F022E0C9
:1097700030E0B701A6018EE799E00E94284380916E
:10978000C00085FFFCCF11C0EBE0FBE08491882393
:1097900041F09091C00095FFFCCF8093C6003196B8
:1097A000F5CF8091C00085FFFCCF8AE08093C60092
:1097B0000F900F900F900F90DF91CF91FF90EF904F
:1097C000DF90CF90BF90AF909F908F907F906F90E1
:1097D0005F904F9008952F923F924F925F926F92B9
:1097E0007F928F929F92AF92BF92CF92DF92EF9231
:1097F000FF920F931F93CF93DF931F92CDB7DEB7E6
:109800000F944150E091300BF0E0EE0FFF1FEA5F44
:10981000FC4B4591549161E080E00F942B7D81E0F9
:109820000F9467158983E8EEFFE0E4918E2F992766
:1098300081950CF490951C0184E00F94BF3AA8EE3A
:10984000BAE01D921D921D921C921397E4EEFAE06D
:109850002081318142815381A0EEBAE06D917D91EA
:109860008D919C91BCEECB2EBAE0DB2EE12CF12C3D
:1098700087010F94E11154DE8DEF9FE00E943A437F
:109880002DEC3CEC4CE85FE30F9476C04B015C019F
:10989000B101882777FD8095982F0F9443BE9B01D7
:1098A000AC01C501B4010F9476C0E3EBFAE020816E
:1098B0003181428153810F94C8BC2B013C01A3EB41
:1098C000BAE06D937D938D939C931397E0E6F2E05D
:1098D000608171818281938160930C0270930D028B
:1098E00080930E0290930F0220E030E040E752E4B4
:1098F0000F94A8BD4B015C01AFEABAE02D913D91F8
:109900004D915C91EBEAFAE06081718182819381F3
:10991000ACECBAE0BF93AF9317EBC12E1AE0D12E97
:10992000830172010F94330582E00F9410380F9475
:10993000E21E0F943F3B80E00F946715A8EEBAE05B
:109940001D921D921D921C921397E4EEFAE0208165
:10995000318142815381A0EEBAE06D917D918D916C
:109960009C910CEEC02E0AE0D02EE12CF12C870148
:109970000F94E111D5DD8AE0829DB001839D700DC9
:109980001124882777FD8095982F0F9443BEE3EB31
:10999000FAE020813181428153810F94C8BC2B01B0
:1099A0003C01A3EBBAE06D937D938D939C93139749
:1099B00020E030E040E05FE3E0E6F2E060817181CA
:1099C000828193810F9476C060930C0270930D0294
:1099D00080930E0290930F0220E030E040E752E4C3
:1099E0000F94A8BD4B015C01AFEABAE02D913D9107
:1099F0004D915C91EBEAFAE0608171818281938103
:109A0000ACECBAE0BF93AF93E7EBCE2EEAE0DE2EEC
:109A1000830172010F9433050F94E21E89810F9424
:109A2000671580E090E0A4E5B3E4E8EEFAE0808317
:109A30009183A283B383A4EEBAE02D913D914D9121
:109A40005C91E0EEFAE06081718182819381FCEEAD
:109A5000CF2EFAE0DF2EE12CF12C04E513E40F9475
:109A6000E11181E00F900F900F900F900F90DF9118
:109A7000CF911F910F91FF90EF90DF90CF90BF900B
:109A8000AF909F908F907F906F905F904F903F909E
:109A90002F9008952F923F924F925F926F927F92F4
:109AA0008F929F92AF92BF92CF92DF92EF92FF92EE
:109AB0000F931F93CF93DF93CDB7DEB729970FB6E0
:109AC000F894DEBF0FBECDBF3C0181E00F94671557
:109AD0008F8382E06816710408F081C2F301EA51B5
:109AE000F04FE491D301AA0FBB1FAA0FBB1FBA838B
:109AF000A983A85ABD4FBE83AD838D919D910D90D2
:109B0000BC91A02D80930C0290930D02A0930E02A5
:109B1000B0930F0281E0062C01C0880F0A94EAF787
:109B20000F94BF3AE981FA81E052F54FF987E8874F
:109B30001082118212821382E090E80AF090E90A02
:109B40000091EA0A1091EB0A2091E40A3091E50AAB
:109B50004091E60A5091E70A6091E00A7091E10AAB
:109B60008091E20A9091E30AECEECE2EEAE0DE2E3E
:109B70000F94E111E981FA81E555F54F2F0180E05D
:109B800090E0A0E4B0E480839183A283B38320E0DB
:109B900030E040E752E460910C0270910D02809138
:109BA0000E0290910F020F94A8BD4B015C01E09052
:109BB000B30AF090B40A0091B50A1091B60A209148
:109BC000AF0A3091B00A4091B10A5091B20A609147
:109BD000AB0A7091AC0A8091AD0A9091AE0AFCEC90
:109BE0002F2EFAE03F2E3F922F92A7EBCA2EAAE02B
:109BF000DA2E0F9433050F94E21E0F944F1580E078
:109C00000F946715A885B9851D921D921D921C920F
:109C10001397E090E80AF090E90A0091EA0A10919F
:109C2000EB0A2091E40A3091E50A4091E60A50914E
:109C3000E70A6091E00A7091E10A8091E20A90914E
:109C4000E30ABCEECB2EBAE0DB2E0F94E11180E0EC
:109C500090E0A0E8BFEBF20180839183A283B383FD
:109C600020E030E040E752E460910C0270910D0278
:109C700080910E0290910F020F94A8BD4B015C01E0
:109C8000E090B30AF090B40A0091B50A1091B60AB8
:109C90002091AF0A3091B00A4091B10A5091B20AB6
:109CA0006091AB0A7091AC0A8091AD0A9091AE0AB6
:109CB0003F922F92E7EBCE2EEAE0DE2E0F94330593
:109CC0000F94E21E81E00F94671589819A818B5071
:109CD000904F0E943A432DEC3CEC4CE85FEB0F9424
:109CE00076C0D2016D937D938D939C93139720E062
:109CF00030E040E752E460910C0270910D028091D7
:109D00000E0290910F020F94A8BD4B015C01E090F0
:109D1000B30AF090B40A0091B50A1091B60A2091E6
:109D2000AF0A3091B00A4091B10A5091B20A6091E5
:109D3000AB0A7091AC0A8091AD0A9091AE0A3F9245
:109D40002F920F9433050F94E21E0F944F1580E06D
:109D50000F946715E885F9851082118212821382AB
:109D6000E090E80AF090E90A0091EA0A1091EB0A03
:109D70002091E40A3091E50A4091E60A5091E70A01
:109D80006091E00A7091E10A8091E20A9091E30A01
:109D9000FCEECF2EFAE0DF2E0F94E11180E090E090
:109DA000A0E2B1E4F20180839183A283B38320E037
:109DB00030E040E752E460910C0270910D02809116
:109DC0000E0290910F020F94A8BD4B015C01E09030
:109DD000B30AF090B40A0091B50A1091B60A209126
:109DE000AF0A3091B00A4091B10A5091B20A609125
:109DF000AB0A7091AC0A8091AD0A9091AE0A3F9285
:109E00002F92A7EBCA2EAAE0DA2E0F9433050F94F7
:109E1000E21E0F944F1581E00F94671580E090E0EB
:109E2000A0E7B1ECF20180839183A283B38320E0A9
:109E300030E040E05FE3AD81BE816D917D918D9119
:109E40009C910F9476C060930C0270930D028093E6
:109E50000E0290930F0220E030E040E752E40F94AE
:109E6000A8BD4B015C01E090B30AF090B40A0091E8
:109E7000B50A1091B60A2091AF0A3091B00A40910C
:109E8000B10A5091B20A6091AB0A7091AC0A80910C
:109E9000AD0A9091AE0A3F922F920F9433050F9422
:109EA000E21EC3010E944043F301EF52F54F81E0EF
:109EB00080830F943F3B0F944F1580E00F946715FC
:109EC0002AE037ED43E25FE3E885F985608171813F
:109ED000828193810F94C7BCA885B9856D937D93CA
:109EE0008D939C931397E090E80AF090E90A009113
:109EF000EA0A1091EB0A2091E40A3091E50A4091B8
:109F0000E60A5091E70A6091E00A7091E10A8091B7
:109F1000E20A9091E30ABCEECB2EBAE0DB2E0F945E
:109F2000E1112AE037ED43E25FE3E885F9856081DE
:109F30007181828193810F94C8BCA885B9856D9386
:109F40007D938D939C931397F20160837183828339
:109F500093832AE939E949E95EE360910C02709143
:109F60000D0280910E0290910F020F9476C020E0B6
:109F700030E040E752E40F94A8BD4B015C01E09053
:109F8000B30AF090B40A0091B50A1091B60A209174
:109F9000AF0A3091B00A4091B10A5091B20A609173
:109FA000AB0A7091AC0A8091AD0A9091AE0A3F92D3
:109FB0002F92E7EBCE2EEAE0DE2E0F9433050F94BE
:109FC000E21E10920C0210920D0210920E021092DC
:109FD0000F020FB6F894DEBF0FBECDBF62C192E094
:109FE0006916710409F05DC1E8EEFFE0749010920B
:109FF000E80A1092E90A1092EA0A1092EB0A2091FC
:10A00000E40A3091E50A4091E60A5091E70A60912E
:10A01000E00A7091E10A8091E20A9091E30ABCEEB5
:10A02000CB2EBAE0DB2EE12CF12C87010F94E1114D
:10A030008DEF9FE00E943A434B015C01672D77272B
:10A0400067FD7095872F972F0F9443BE2B013C011E
:10A0500020E030E040EC5FE3C501B4010F9476C02E
:10A06000A30192010F9476C069837A838B839C83CA
:10A070006093B30A7093B40A8093B50A9093B60ABA
:10A08000609160027091610280916202909163021E
:10A0900060930C0270930D0280930E0290930F0256
:10A0A00020E030E040E752E40F94A8BD4B015C0192
:10A0B0002091AF0A3091B00A4091B10A5091B20A92
:10A0C0006091AB0A7091AC0A8091AD0A9091AE0A92
:10A0D0001CEC212E1AE0312E3F922F9207EBC02E5E
:10A0E0000AE0D02EE980FA800B811C810F943305A1
:10A0F0000F94E21E1092E80A1092E90A1092EA0AFE
:10A100001092EB0A2091E40A3091E50A4091E60AA8
:10A110005091E70A6091E00A7091E10A8091E20AA9
:10A120009091E30AECEECE2EEAE0DE2EE12CF12C4B
:10A1300087010F94E11181EF9FE00E943A4390580C
:10A14000A30192010F9476C069837A838B839C83E9
:10A150006093B30A7093B40A8093B50A9093B60AD9
:10A1600020E030E040E752E460910C0270910D0273
:10A1700080910E0290910F020F94A8BD4B015C01DB
:10A180002091AF0A3091B00A4091B10A5091B20AC1
:10A190006091AB0A7091AC0A8091AD0A9091AE0AC1
:10A1A0003F922F92F7EBCF2EFAE0DF2EE980FA8074
:10A1B0000B811C810F9433050F94E21E81EF9FE009
:10A1C0000E943A439B01AC010F94C8BCA3019201C9
:10A1D0000F9476C02B013C016093B30A7093B40ACC
:10A1E0008093B50A9093B60A20E030E040E05FE348
:10A1F00060916002709161028091620290916302AD
:10A200000F9476C060930C0270930D0280930E023F
:10A2100090930F0220E030E040E752E40F94A8BD95
:10A220004B015C012091AF0A3091B00A4091B10A14
:10A230005091B20A6091AB0A7091AC0A8091AD0A5C
:10A240009091AE0A3F922F92830172010F943305D1
:10A250000F94E21E82E090E00E9440438091E80A61
:10A260009091E90AA091EA0AB091EB0A8093B30AAF
:10A270009093B40AA093B50AB093B60A10920C0258
:10A2800010920D0210920E0210920F020F944F15B1
:10A2900081E08093D30A0F900F900F900F900F9052
:10A2A0000F908F8129960FB6F894DEBF0FBECDBFF9
:10A2B000DF91CF911F910F91FF90EF90DF90CF90A2
:10A2C000BF90AF909F908F907F906F905F904F90D6
:10A2D0003F902F900D946715CF92DF92EF92FF92EF
:10A2E0000F931F931DD980E090E0D4DB81E090E0D4
:10A2F000D1DBE090E80AF090E90A0091EA0A1091B7
:10A30000EB0A2091E40A3091E50A4091E60A509167
:10A31000E70A6091E00A7091E10A8091E20A909167
:10A32000E30AFCEECF2EFAE0DF2E0F94E1111F912D
:10A330000F91FF90EF90DF90CF900D944F150F94F9
:10A34000CAB46093920A7093930A8093940A90938C
:10A35000950A089520E030E0A90168EB71E084E5FA
:10A360000F9422B969E170E080E090E00F94F9B4B5
:10A3700084E50F9446BC64E170E080E090E00D94C9
:10A38000F9B47F928F929F92AF92BF92CF92DF9259
:10A39000EF92FF920F931F93CF93DF9300D01F9202
:10A3A000CDB7DEB71092781A1092771A1092761AFB
:10A3B0001092751A0F9441508BE99EE00F945267EA
:10A3C0008E010F5F1F4F7E0125E0E20EF11C8EE72C
:10A3D00099E00E9442418F3FEFEF9E07C1F3F801E1
:10A3E00081938F01EE15FF0591F789809A80AB80EC
:10A3F000BC808091C00085FFFCCF8BE28093C600BB
:10A40000C12CD12C7601ABE27A2E80912F0B8823C0
:10A4100009F450C000E21AE0C814D904EA04FB04AD
:10A42000A1F08EE799E00E9442418F3FFFEF9F0726
:10A43000C1F32FEFC21AD20AE20AF20AF80181939D
:10A440008F01FAE000361F0739F760E27AE08AE60A
:10A450009BE00E940BBB8091C00085FFFCCF7092F7
:10A46000C6000F94CE2BC814D904EA04FB0469F685
:10A4700071DF60E08AE69BE00E943EBC10922F0BE9
:10A48000E6E9F2E485919491FC012491222341F0C4
:10A490003091C00035FFFCCF2093C6000196F4CF69
:10A4A0008091C00085FFFCCF8AE08093C60080E0E9
:10A4B00090E000C00F900F900F900F90DF91CF9120
:10A4C0001F910F91FF90EF90DF90CF90BF90AF90D2
:10A4D0009F908F907F9008952F923F924F925F921E
:10A4E0006F927F928F929F92AF92BF92CF92DF92A4
:10A4F000EF92FF920F931F93CF93DF931F921F92C0
:10A50000CDB7DEB7382E811112C01092761A109294
:10A51000751A1092781A1092771A10927A1A10926D
:10A52000791A10927C1A10927B1A0F94965080E040
:10A530000F94AC9987E792E10E94CEF90E9430DB3C
:10A540000E941FF91092D10A1092D20A1092D30AD7
:10A5500081E00E948E43E4E7F3E4859194910E94A8
:10A560002748BADE38D9882309F483C1E8DE3110E0
:10A5700058C084E090E09093160280931502E09119
:10A58000300BF0E0EE0FFF1FE055FF4B85919491EB
:10A5900040E060E00F94999B882359F0E091300BE4
:10A5A000F0E0EE0FFF1FEE58FE4B859194910F9453
:10A5B00059A4E091300BF0E0EE0FFF1FE051FD4B8E
:10A5C000859194910F9459A4E091300BF0E0EE0F37
:10A5D000FF1FE453FE4B859194910F9459A482E0A0
:10A5E00090E09093160280931502E091300BF0E01A
:10A5F000EE0FFF1FE257FD4B859194910E94274873
:10A6000041E050E062E080E00F944C50E091300B6C
:10A61000F0E0EE0FFF1FE657FD4B859194910F94EC
:10A62000526780E090E0A0EAB0E48093E80A90935B
:10A63000E90AA093EA0AB093EB0A20E030E040E296
:10A6400052E4609160027091610280916202909187
:10A6500063020F94A8BD4B015C012091E40A309184
:10A66000E50A4091E60A5091E70A6091E00A70918C
:10A67000E10A8091E20A9091E30AECECFAE0FF93A0
:10A68000EF93ECEECE2EEAE0DE2EE12CF12C00EA88
:10A6900010E40F9433050F94E21E86E50E94E24316
:10A6A0000F900F90882361F0E0913910F0913A10EB
:10A6B0008181893039F08F7D41F00E94F84303C0D9
:10A6C0001A8205C081E08A8302C0A1E0AA833320F8
:10A6D000B1F00E94BC430E9485DB0E94A1DD0E9474
:10A6E00075F2882309F4C1C087EF9FE00F941FCA59
:10A6F000803F09F0BAC081E00E943548B6C08FEFB4
:10A700000E94354860E070E088EF9FE00F944BCAEC
:10A710001982BE016F5F7F4F8A810E9446EF3C0124
:10A720000E94BC43212C312C10EA412E10E4512E02
:10A730002092E80A3092E90A4092EA0A5092EB0A23
:10A7400020E030E040E252E46091600270916102EA
:10A7500080916202909163020F94A8BD4B015C014D
:10A760002091E40A3091E50A4091E60A5091E70A07
:10A770006091E00A7091E10A8091E20A9091E30A07
:10A78000ACECBAE0BF93AF930CEEC02E0AE0D02E33
:10A79000820171010F9433050F94E21E0F900F9008
:10A7A00077FC47C0198287E792E10E94CEF90E94A8
:10A7B000F7DA81E00E948E438FDDAE014F5F5F4F7D
:10A7C0006A8181E00E949BF43C010E94BC4320927C
:10A7D000E80A3092E90A4092EA0A5092EB0A20E035
:10A7E00030E040E252E46091600270916102809139
:10A7F0006202909163020F94A8BD4B015C0120910D
:10A80000E40A3091E50A4091E60A5091E70A609126
:10A81000E00A7091E10A8091E20A9091E30AACECBF
:10A82000BAE0BF93AF930F9433050F94E21E0F90DD
:10A830000F906981C3010F94C3A477FC16C086EE04
:10A840000E9435488FE59FE00F941FCA813059F070
:10A85000E091300BF0E0EE0FFF1FE659FC4B8591C5
:10A8600094910F9459A411E001C010E00F943F3B64
:10A8700001C010E081E00F94AC99812F0F900F90F0
:10A88000DF91CF911F910F91FF90EF90DF90CF90CC
:10A89000BF90AF909F908F907F906F905F904F9000
:10A8A0003F902F9008958F929F92AF92BF92CF9238
:10A8B000DF92EF92FF920F931F93CF93DF93159840
:10A8C00081E08093240B82E090E09093220B8093B0
:10A8D000210BE091300BF0E0EE0FFF1FEA5CFD4B27
:10A8E000859194910F94595120E030E04CE852E466
:10A8F0006091EC0A7091ED0A8091EE0A9091EF0A56
:10A900000F94C8BC6093EC0A7093ED0A8093EE0A32
:10A910009093EF0AE090E80AF090E90A0091EA0AC1
:10A920001091EB0A2091E40A3091E50A4091E60A81
:10A930005091E70A6091E00A7091E10A8091E20A81
:10A940009091E30ACCECDAE0DF93CF93812C912C49
:10A95000E0ECAE2EE0E4BE2EFCEECF2EFAE0DF2ED1
:10A960000F94330520E030E048EC51E46091EC0AAC
:10A970007091ED0A8091EE0A9091EF0A0F94C8BC95
:10A980006093EC0A7093ED0A8093EE0A9093EF0ABD
:10A99000E090E80AF090E90A0091EA0A1091EB0AC7
:10A9A0002091E40A3091E50A4091E60A5091E70AC5
:10A9B0006091E00A7091E10A8091E20A9091E30AC5
:10A9C000DF93CF93812C912CA0E8AA2EAFE3BA2E6F
:10A9D0000F9433050F94E21E0F900F900F900F907D
:10A9E0008091921B882331F181E00F94AC9982E031
:10A9F0000F94E596E091300BF0E0EE0FFF1FEE5F55
:10AA0000FF4B859194910F9459511092230B109202
:10AA1000240B1092220B1092210BDF91CF911F91EA
:10AA20000F91FF90EF90DF90CF90BF90AF909F90ED
:10AA30008F9008958091230B8823B1F2E091300B21
:10AA4000F0E0EE0FFF1FE656FD4B8591949141E03B
:10AA500060E00F94999B91E0811101C090E0CCECF3
:10AA6000DAE09111C1CF81E00F94AC9982E00F94AC
:10AA7000E59620E030E048EC51E46091EC0A7091FA
:10AA8000ED0A8091EE0A9091EF0A0F94C8BC609392
:10AA9000EC0A7093ED0A8093EE0A9093EF0AE0902F
:10AAA000E80AF090E90A0091EA0A1091EB0A209175
:10AAB000E40A3091E50A4091E60A5091E70A609174
:10AAC000E00A7091E10A8091E20A9091E30ADF9333
:10AAD000CF93812C912CE0E8AE2EEFE3BE2EFCEE5E
:10AAE000CF2EFAE0DF2E0F9433050F94E21EE09193
:10AAF000300BF0E0EE0FFF1FE656FD4B8591949171
:10AB000041E060E00F94999B0F900F9081116CCF02
:10AB1000AACF0F94CAB46093920A7093930A809359
:10AB2000940A9093950AE0914310F0914410EB5BE6
:10AB3000FF4E80818130B9F4E0EDF1E4859194918C
:10AB4000FC012491222341F03091C00035FFFCCF5D
:10AB50002093C6000196F4CF8091C00085FFFCCF02
:10AB60008AE08093C60008958EE799E00E945E41D6
:10AB7000E0E7F1E485919491FC012491222341F0D6
:10AB80003091C00035FFFCCF2093C6000196F4CF72
:10AB90004091291050912A1060912B1070912C1027
:10ABA0004F5F5F4F6F4F7F4F2AE030E08EE799E0B5
:10ABB0000E94FD418091C00085FFFCCF8AE0809318
:10ABC000C600A7CF8F929F92AF92BF92CF92DF9293
:10ABD000EF92FF920F931F93CF93DF93B9E7EB2E82
:10ABE000B5E0FB2E00EE1AE0CBEADAE082E6C82EF2
:10ABF0008BE0D82EF70181917F010E94E2438823E8
:10AC000019F10E944F444B015C01F60180818111D2
:10AC100003C06091960A01C061E070E080E090E0BE
:10AC20000F9443BEF80120813181428153810F94FA
:10AC300076C09B01AC01C501B4010F94C8BC688308
:10AC400079838A839B8309C0F80180819181A281E5
:10AC5000B38188839983AA83BB830C5F1F4F24969B
:10AC6000FFEFCF1ADF0A8DE7E81685E0F80611F648
:10AC700086E40E94E2438823D9F00E944F446B018E
:10AC80007C0160939B0A70939C0A80939D0A909329
:10AC90009E0A20E030E0A9010F94A4BF181644F4E6
:10ACA000C0920C02D0920D02E0920E02F0920F02BE
:10ACB000DF91CF911F910F91FF90EF90DF90CF9098
:10ACC000BF90AF909F908F9008957CDF89E40E94A1
:10ACD000E243882359F00E944F4460939F0A709387
:10ACE000A00A8093A10A9093A20A08C010929F0A1A
:10ACF0001092A00A1092A10A1092A20A8AE40E945D
:10AD0000E243882359F00E944F446093A30A709352
:10AD1000A40A8093A50A9093A60A08951092A30A04
:10AD20001092A40A1092A50A1092A60A0895CF9232
:10AD3000DF92EF92FF92CF93DF93EC01BC016C5F47
:10AD40007F4F0E94104720E030E0A90160913C0253
:10AD500070913D0280913E0290913F020F94C8BCD9
:10AD60006B017C019B01AC01688579858A859B8597
:10AD70000F94A1BD87FF04C0C886D986EA86FB86EA
:10AD8000C0903002D0903102E0903202F090330255
:10AD9000A7019601688579858A859B850F94A4BF54
:10ADA000181624F4C886D986EA86FB86DF91CF91EF
:10ADB000FF90EF90DF90CF9008952F923F924F92A7
:10ADC0005F926F927F928F929F92AF92BF92CF923B
:10ADD000DF92EF92FF920F931F93CF93DF93CDB744
:10ADE000DEB7AB970FB6F894DEBF0FBECDBF9F871F
:10ADF0008E87798B688B5B8B4A8B3D8B2C8B1F8B63
:10AE00000E8BED82DC018D909D90AD90BC904090BA
:10AE1000E00A5090E10A6090E20A7090E30ADB01D8
:10AE20008D919D910D90BC91A02D88879987AA87BF
:10AE3000BB87C090E40AD090E50AE090E60AF09063
:10AE4000E70A2091E80A3091E90A4091EA0A509114
:10AE5000EB0AEA89FB8960817181828193810F9479
:10AE6000C7BC688F798F8A8F9B8F809177128111F1
:10AE700073C0AE89BF898D909D90AD90BC90EA89DA
:10AE8000FB89E080F18002811381A889B9892D9125
:10AE90003D914D915C91EE85FF856081718182814C
:10AEA0009381FE013596FF93EF93CC88DD880F9454
:10AEB0003305EE85FF8580819181A281B3818093E6
:10AEC000E00A9093E10AA093E20AB093E30AE889CA
:10AED000F98980819181A281B3818093E40A909362
:10AEE000E50AA093E60AB093E70AEA89FB89808124
:10AEF0009181A281B3818093E80A9093E90AA0939B
:10AF0000EA0AB093EB0AEC89FD8980819181A281E4
:10AF1000B3818093EC0A9093ED0AA093EE0AB0936C
:10AF2000EF0A0F900F90AB960FB6F894DEBF0FBEEE
:10AF3000CDBFDF91CF911F910F91FF90EF90DF90E8
:10AF4000CF90BF90AF909F908F907F906F905F90C9
:10AF50004F903F902F900895A3019201C501B40135
:10AF60000F94C7BC2B013C0120E030E0A9010F94F5
:10AF7000A4BF53014201181624F0B7FAB094B7F8F1
:10AF8000B094A7019601688579858A859B850F9481
:10AF9000C7BC688779878A879B8720E030E0A90152
:10AFA0000F94A4BF288539854A855B8518160CF057
:10AFB0005058C501B4010F94C8BC6B017C0120E05E
:10AFC00030E0A9010F94A4BF18160CF052CF20E076
:10AFD00030E040EF51E4C701B6010F94A8BD0F94D3
:10AFE0008EBD0F9410BE7D876C87623071050CF4A6
:10AFF00040CF2091EC0A3091ED0A4091EE0A509139
:10B00000EF0AAC89BD896D917D918D919C910F94D2
:10B01000C7BC6C8F7D8F8E8F9F8F22242394312C01
:10B020008C859D85AA2797FDA095BA2F88A799A7FB
:10B03000AAA7BBA7DE011596BF83AE83B1018827FF
:10B0400077FD8095982F0F9443BE6B017C0168A516
:10B0500079A58AA59BA50F9443BE9B01AC01C701AE
:10B06000B6010F94A8BD6B017C01EE89FF89808039
:10B070009180A280B3802C8D3D8D4E8D5F8D0F947D
:10B0800076C09B01AC016091EC0A7091ED0A809151
:10B09000EE0A9091EF0A0F94C8BC69837A838B8380
:10B0A0009C83288D398D4A8D5B8DC701B6010F9425
:10B0B00076C02091E80A3091E90A4091EA0A50915D
:10B0C000EB0A0F94C8BC68A379A38AA39BA3288525
:10B0D00039854A855B85C701B6010F9476C02091FA
:10B0E000E40A3091E50A4091E60A5091E70A0F948C
:10B0F000C8BC6CA37DA38EA39FA3A3019201C7012B
:10B10000B6010F9476C02091E00A3091E10A409197
:10B11000E20A5091E30A0F94C8BCFF81FF932E818D
:10B120002F93DE0111966D01E8A0F9A00AA11BA1E1
:10B130002CA13DA14EA15FA10F943305BFEF2B1AA7
:10B140003B0A0F900F90EC85FD852E163F0609F007
:10B1500075CF8FCE4F925F926F927F928F929F9218
:10B16000AF92BF92CF92DF92EF92FF920F931F9315
:10B17000CF93DF93CDB7DEB728970FB6F894DEBF35
:10B180000FBECDBF8BEA9AE0D2DD0F94CAB46093B4
:10B19000920A7093930A8093940A9093950A8091EF
:10B1A000AB0A9091AC0AA091AD0AB091AE0A8D8322
:10B1B0009E83AF83B8879C01AD016091E00A7091D6
:10B1C000E10A8091E20A9091E30A0F94A1BD8111F6
:10B1D00097C04090AF0A5090B00A6090B10A70904A
:10B1E000B20AA30192016091E40A7091E50A80918C
:10B1F000E60A9091E70A0F94A1BD811181C020E079
:10B2000030E040E752E460910C0270910D028091B1
:10B210000E0290910F020F94A8BD4B015C01E090CB
:10B22000B30AF090B40A0091B50A1091B60A8CECFA
:10B230009AE09F938F9327EBC22E2AE0D22EA30190
:10B2400092016D817E818F8198850F9433050F90D7
:10B250000F908091AB0A9091AC0AA091AD0AB09189
:10B26000AE0A8093E00A9093E10AA093E20AB093B9
:10B27000E30A8091AF0A9091B00AA091B10AB0910F
:10B28000B20A8093E40A9093E50AA093E60AB09389
:10B29000E70A8091B30A9091B40AA091B50AB091DF
:10B2A000B60A8093E80A9093E90AA093EA0AB09359
:10B2B000EB0A8091B70A9091B80AA091B90AB091AF
:10B2C000BA0A8093EC0A9093ED0AA093EE0AB09329
:10B2D000EF0A28960FB6F894DEBF0FBECDBFDF9100
:10B2E000CF911F910F91FF90EF90DF90CF90BF9083
:10B2F000AF909F908F907F906F905F904F90089548
:10B30000E090CC0A6091560270915702882777FD31
:10B310008095982F0F9443BE20910C0230910D021E
:10B3200040910E0250910F020F9476C02EE333EC41
:10B330004EE259E30F9476C069837A838B839C83B2
:10B340008E010F5F1F4F27EB3AE043EB5AE06FEAA5
:10B350007AE08BEA9AE031DD7CCF4F925F926F9278
:10B360007F928F929F92AF92BF92CF92DF92EF9295
:10B37000FF920F931F93CF93C62FE091CC0AF0E07A
:10B38000882309F4D9C0DF01A853B54F8C918111EE
:10B39000AFC18091E00A9091E10AA091E20AB091D8
:10B3A000E30A8093AB0A9093AC0AA093AD0AB093E2
:10B3B000AE0A8091E40A9091E50AA091E60AB09164
:10B3C000E70A8093AF0A9093B00AA093B10AB093B2
:10B3D000B20A8091E80A9091E90AA091EA0AB09134
:10B3E000EB0A8093B30A9093B40AA093B50AB09382
:10B3F000B60AC090EC0AD090ED0AE090EE0AF09008
:10B40000EF0AC092B70AD092B80AE092B90AF09255
:10B41000BA0AEE0FFF1FEE0FFF1FE05CFD4F208109
:10B42000318142815381662349F0609120027091FD
:10B430002102809122029091230208C0609124028F
:10B440007091250280912602909127020F94A8BD49
:10B450009B01AC01C701B6010F94C8BC6093EC0A14
:10B460007093ED0A8093EE0A9093EF0A8CEE9AE0C7
:10B470000F948C1380900C0290900D02A0900E02FD
:10B48000B0900F0220E030E040E752E460911C02EF
:10B4900070911D0280911E0290911F020F9476C040
:10B4A00060930C0270930D0280930E0290930F0232
:10B4B000E091CC0AF0E0E853F54F81E080834ADE6A
:10B4C0002091C40A3091C50A4091C60A5091C70A1A
:10B4D0006091E80A7091E90A8091EA0A9091EB0A7A
:10B4E0000F94C7BC7B018C016093E80A7093E90A52
:10B4F0008093EA0A9093EB0A2091E40A3091E50ADE
:10B500004091E60A5091E70A6091E00A7091E10AE1
:10B510008091E20A9091E30AECEECE2EEAE0DE2E74
:10B520000F94E11117DE80920C0290920D02A0920E
:10B530000E02B0920F02DCC0E853F54F80818823E1
:10B5400009F4D6C08090E00A9090E10AA090E20A47
:10B55000B090E30A8092AB0A9092AC0AA092AD0A36
:10B56000B092AE0A4090E40A5090E50A6090E60A74
:10B570007090E70A4092AF0A5092B00A6092B10A06
:10B580007092B20A6091E80A7091E90A8091EA0A21
:10B590009091EB0A6093B30A7093B40A8093B50A52
:10B5A0009093B60A0091EC0A1091ED0A2091EE0AF0
:10B5B0003091EF0A0093B70A1093B80A2093B90AA2
:10B5C0003093BA0A2091C40A3091C50A4091C60A44
:10B5D0005091C70A0F94C8BC7B018C016093E80AA4
:10B5E0007093E90A8093EA0A9093EB0A3CEEC32E2B
:10B5F0003AE0D32EA3019201C501B4010F94E111E9
:10B600001091CC0ACC2389F02091BC0A3091BD0A5C
:10B610004091BE0A5091BF0A6091200270912102B0
:10B62000809122029091230210C02091C00A309193
:10B63000C10A4091C20A5091C30A609124027091DC
:10B64000250280912602909127020F94C8BC24E025
:10B65000129FF0011124E05CFD4F20813181428175
:10B6600053810F94A8BD9B01AC016091EC0A7091CD
:10B67000ED0A8091EE0A9091EF0A0F94C7BC609397
:10B68000EC0A7093ED0A8093EE0A9093EF0A8CEE29
:10B690009AE00F948C13C0900C02D0900D02E090B1
:10B6A0000E02F0900F0220E030E040E752E460919B
:10B6B00018027091190280911A0290911B020F9446
:10B6C00076C060930C0270930D0280930E029093EB
:10B6D0000F02E091CC0AF0E0E853F54F10823ADD1A
:10B6E000C0920C02D0920D02E0920E02F0920F0274
:10B6F000CF911F910F91FF90EF90DF90CF90BF906F
:10B70000AF909F908F907F906F905F904F90089533
:10B71000AF92BF92CF92DF92EF92FF920F931F935F
:10B72000CF93DF93D82F2091A30A3091A40A4091A0
:10B73000A50A5091A60A60919F0A7091A00A809173
:10B74000A10A9091A20A0F94B1BFC62F172F082FFC
:10B75000F92E6091560270915702882777FD8095E7
:10B76000982F0F9443BE20910C0230910D0240910E
:10B770000E0250910F020F9476C020E030E040E7B7
:10B7800052E40F94A8BD20E030E048EC52E40F945E
:10B79000A8BD2091CC0A2F93DF93FF920F931F93A4
:10B7A000CF935B016C01B2E0EB2E01E020E04FE9AA
:10B7B0005AE06BEA7AE080EE9AE00E94B3FB809157
:10B7C000AB0A9091AC0AA091AD0AB091AE0A8093F9
:10B7D000E00A9093E10AA093E20AB093E30A809111
:10B7E000AF0A9091B00AA091B10AB091B20A8093C9
:10B7F000E40A9093E50AA093E60AB093E70A8091E1
:10B80000B30A9091B40AA091B50AB091B60A809398
:10B81000E80A9093E90AA093EA0AB093EB0A8091B0
:10B82000B70A9091B80AA091B90AB091BA0A809368
:10B83000EC0A9093ED0AA093EE0AB093EF0A0F94EE
:10B84000CAB46093920A7093930A8093940A909377
:10B85000950A0F900F900F900F900F900F90DF911F
:10B86000CF911F910F91FF90EF90DF90CF90BF90FD
:10B87000AF900895EC01E4E0FBE08491882341F06F
:10B880009091C00095FFFCCF8093C6003196F5CF14
:10B8900070E04AE050E08EE799E00E943C42F89464
:10B8A0000F94DA28179A1092D10A169A1092D20A97
:10B8B000149AEBE2F0E18491882341F09091C0006A
:10B8C00095FFFCCF8093C6003196F5CFEEEBF2E406
:10B8D00085919491FC012491222341F03091C00084
:10B8E00035FFFCCF2093C6000196F4CF8091C000B5
:10B8F00085FFFCCF8AE08093C6002097C9F0FE0147
:10B900008491FE01882349F09091C00095FFFCCFFF
:10B910008093C60031968491F5CF8091C00085FF59
:10B92000FCCF8AE08093C600CE010E94274806C063
:10B93000EAE4F2E4859194910F9484517894C6E0FE
:10B94000D0E0219751F068EC70E080E090E00F9437
:10B95000F9B480E00F94E596F4CFF894A895FECF63
:10B96000CF92DF92EF92FF920F931F93CF93C82F46
:10B9700080913F1090914010039714F40E9498C456
:10B980000F94CAB400918E0A10918F0A2091900AE8
:10B990003091910AC090920AD090930AE090940A54
:10B9A000F090950A6C197D098E099F0906171707F3
:10B9B0002807390740F4012B022B032B21F064E008
:10B9C0008EEF98E057DF4091080250910902609194
:10B9D0000A0270910B02452B462B472B19F10F944D
:10B9E000CAB40091920A1091930A2091940A30915E
:10B9F000950A601B710B820B930B0091080210914A
:10BA0000090220910A0230910B0206171707280736
:10BA1000390740F49091641380916313981302C026
:10BA2000CC2349F0CF911F910F91FF90EF90DF90C1
:10BA3000CF900D946103179A1092D10A169A109222
:10BA4000D20A149AEFCF0F94DA288091800A8111DC
:10BA50003DC081E08093800A8091291090912A1046
:10BA6000A0912B10B0912C1080932510909326104C
:10BA7000A0932710B0932810EBE2F0E18491882383
:10BA800041F09091C00095FFFCCF8093C6003196A5
:10BA9000F5CFE4EBF2E485919491FC01249122230B
:10BAA00041F03091C00035FFFCCF2093C6000196D5
:10BAB000F4CF8091C00085FFFCCF8AE08093C60060
:10BAC000ECEAF0E4859194910D9459510895809198
:10BAD000800A0895CF93DF93EC018091CC0A809384
:10BAE000810A84E50E94E243811102C080E084C0A3
:10BAF0000E944F440F9415BE6093810A6623B1F3F0
:10BB0000E5E2F0E18491882341F09091C00095FF37
:10BB1000FCCF8093C6003196F5CFCD36D10509F420
:10BB200035C064F4C836D105B1F0C936D10509F085
:10BB300052C0EAE2F2E4A591B49124C0CA3DD10515
:10BB400009F432C0CD3DD10509F045C0EAE1F2E487
:10BB5000A591B4913DC0ECE2F2E485919491FC0191
:10BB60002491222309F437C03091C00035FFFCCF67
:10BB70002093C6000196F3CF9091C00095FFFCCFB3
:10BB80008093C6008D918111F7CF25C0E8E2F2E4E1
:10BB9000A591B4918D918823F1F09091C00095FF0B
:10BBA000FCCF8093C600F6CFECE1F2E4A591B4910E
:10BBB0008D91882381F09091C00095FFFCCF8093F8
:10BBC000C600F6CF9091C00095FFFCCF8093C600D1
:10BBD0008D918111F7CF6091810A70E04AE050E0C9
:10BBE0008EE799E00E9435428091C00085FFFCCF2E
:10BBF0008AE08093C60081E0DF91CF9108954F9253
:10BC00005F926F927F928F929F92AF92BF92CF92EC
:10BC1000DF92EF92FF92CF93DF9300D01F92CDB7C8
:10BC2000DEB72B013C0129833A834B835C838DEE85
:10BC30009FE00F941FCA8F3F01F58EEE9FE00F9497
:10BC40001FCA8F3FD1F48FEE9FE00F941FCA8F3F22
:10BC5000A1F480EF9FE00F941FCA8F3F71F440E082
:10BC600050E0BA018DEE9FE00F9443CA40E050E0EF
:10BC7000BA0181EF9FE00F9443CA81EF9FE00F94D8
:10BC800027CA4B015C018DEE9FE00F9427CA6B0120
:10BC90007C0169817A818B819C812CE330E040E0DA
:10BCA00050E00F9478C2C20ED31EE41EF51EB701F9
:10BCB000A6018DEE9FE00F9443CAC301B20128EEA6
:10BCC00033E040E050E00F9478C2BA01A901480D7A
:10BCD000591D6A1D7B1D81EF9FE00F9443CA10928E
:10BCE000290B10922A0B10922B0B10922C0B0F90F9
:10BCF0000F900F900F90DF91CF91FF90EF90DF901A
:10BD0000CF90BF90AF909F908F907F906F905F90FB
:10BD10004F900895CF92DF92EF92FF922091F00A18
:10BD20002223F1F020E030E040E05FE30F9476C0A2
:10BD30006B017C0120E030E0A9010F94A1BD8823B4
:10BD400079F0A7019601C701B6010F9476C02BEDDB
:10BD50003FE049E450E40F9476C09B01AC0104C07D
:10BD600020E030E040E85FE360E070E080E89FE3DF
:10BD70000F94A8BDFF90EF90DF90CF900895609151
:10BD80004402709145028091460290914702C2DFC1
:10BD90006093400270934102809342029093430269
:10BDA0000895CF93DF93EC010F94CE2B81E0D8DD83
:10BDB00080E00F94E596209799F0C233D10540F0CA
:10BDC00062E370E080E090E00F94F9B4E297ECCF8A
:10BDD000BE0180E090E00F94F9B4C0E0D0E0E4CF81
:10BDE000DF91CF9108952F923F924F925F926F9281
:10BDF0007F928F929F92AF92BF92CF92DF92EF92FB
:10BE0000FF921F93CF93DF934B015C01CC24CA9424
:10BE1000DC2C760159EF252E5AE0352E68EE462EA1
:10BE200063E0562E612C712C1AE08091BB0A8111BF
:10BE300026C12FEFC216D206E206F20651F0F7FC39
:10BE40001EC10F94CAB46C197D09683B7B4008F091
:10BE500016C10F94CAB4681979098A099B09693E09
:10BE600073408105910508F47FC08091921B811178
:10BE700077C0E1E0FBE08491882341F09091C0001D
:10BE800095FFFCCF8093C6003196F5CFE091810AF3
:10BE900024E0E29FF0011124E159F54E40815181E7
:10BEA0006281738121E030E08EE799E00E942843AF
:10BEB000EDEFFAE08491882341F09091C00095FF66
:10BEC000FCCF8093C6003196F5CF6091810A70E077
:10BED0004AE050E08EE799E00E943542F1018491FA
:10BEE000E9EFFAE0882349F09091C00095FFFCCF7C
:10BEF0008093C60031968491F5CFF7FE03C0E9ED3B
:10BF0000F8E025C00F94CAB44B015C01C701B6012B
:10BF10006854744F8F4F9F4F681979098A099B099C
:10BF2000A30192010F9478C2BA01A9012AE030E07E
:10BF30008EE799E00E94FD418091C00085FFFCCF13
:10BF40000DC09091C00095FFFCCF8093C6008191F9
:10BF50008111F7CF8091C00085FFFCCF1093C60000
:10BF60000F94CAB44B015C010F94CE2B80E0F8DC37
:10BF700080E00F94E596FFEFCF16DF06EF06FF0691
:10BF800009F046C080917F0AE091810AF0E0EF015C
:10BF9000CC0FDD1FCC0FDD1FC159D54EEE0FFF1F9B
:10BFA000E958F54E8823D1F080819181BC01882722
:10BFB00077FD8095982F0F9443BE20E030E040E855
:10BFC0005FE30F94C7BC9B01AC01688179818A81D2
:10BFD0009B810F94A4BF87FF4DC027CF80819181A3
:10BFE000BC01882777FD8095982F0F9443BE20E0F1
:10BFF00030E040E85FE30F94C8BC9B01AC0168816E
:10C0000079818A819B810F94A1BD18169CF50DCF73
:10C01000F7FC0BCFE091810AF0E0EF01CC0FDD1FC0
:10C02000CC0FDD1FC159D54EEE0FFF1FE958F54E5D
:10C0300080819181BC01882777FD8095982F0F948E
:10C0400043BE9B01AC01688179818A819B810F94F9
:10C05000C7BC0F9410BE97FF07C090958095709550
:10C0600061957F4F8F4F9F4F663071058105910518
:10C070000CF4DBCE0F94CAB46B017C01D6CEDF91F9
:10C08000CF911F91FF90EF90DF90CF90BF90AF9036
:10C090009F908F907F906F905F904F903F902F90E8
:10C0A0000895CF93DF931F921F92CDB7DEB7BE01E5
:10C0B0006F5F7F4F88EF9FE00F94805089819A8156
:10C0C0008156904F803A9F4020F11A821982E0ED0C
:10C0D000FAE08491882341F09091C00095FFFCCF55
:10C0E0008093C6003196F5CF8091C00085FFFCCFCC
:10C0F0008AE08093C600BE016F5F7F4F88EF9FE0AC
:10C100000F946F5083E99AE00F9459A481E00F9443
:10C11000AC990F900F90DF91CF9108952F923F929D
:10C120004F925F926F927F928F929F92AF92BF9247
:10C13000CF92DF92EF92FF920F931F93CF93DF93F3
:10C14000CDB7DEB7CA58D2400FB6F894DEBF0FBEE7
:10C15000CDBFC958DD4F688379838A839B83C757D6
:10C16000D240FE01E75FFD4F88E2DF011D928A9514
:10C17000E9F7E850F24080E991E0DF019C011D926F
:10C1800021503040E1F7C75ADD4F19821882C95556
:10C19000D240CE01875A9D4F5C014E019FE6891A1D
:10C1A0009EEF990ADE01AF51BE4F3D0190EBC92EC3
:10C1B0009FE0D92E23E2E22EF12C00E010E0C359DB
:10C1C000DD4F8882CD56D240CD58DD4F9882C3577F
:10C1D000D240B701882777FD8095982F0F9443BEF2
:10C1E000D3016D937D938D939D933D01F5016191F5
:10C1F00071915F01882777FD8095982F0F9443BE3A
:10C20000D4016D937D938D939D934D010F5F1F4FCF
:10C210000630110559F0B501C6010F948050B5E004
:10C22000EB0EF11CE2E0CE0ED11CD3CFCF51DE4F8E
:10C23000288139814A815B81C15ED140C958DD4F77
:10C24000688179818A819B81C757D2400F94A1BDB3
:10C2500087FD2BC3FE01EF51FE4F7F016E01FFE210
:10C26000CF1AFEEFDF0A3E012BEB621A2DEF720AA6
:10C27000C359DD4F0881CD56D240CD58DD4F1881CE
:10C28000C357D24085E090E0CF58DD4F9983888333
:10C29000C157D240CF58DD4FA881B981C157D24094
:10C2A0001197CF58DD4FB983A883C157D240F7010A
:10C2B000208931894289538964897589868997895A
:10C2C0000F94C7BC4B015C01D80150962D913D9154
:10C2D0004D915C91539754966D917D918D919C9168
:10C2E00057970F94C7BCA50194010F94A8BDF60100
:10C2F00092938293729362936F01D301BE92AE9236
:10C300009E928E923D0104501109B4E0EB1AF1089F
:10C31000CF58DD4FE881F981C157D240EF2B09F0AA
:10C32000B9CF6E01FFECCF1AFDEFDF0A3E0127E423
:10C33000621A2EEF720A2E013DE3430E511CCE010C
:10C3400001967C0101E010E0D6018D909D90AD90AA
:10C35000BC90139714962D913D914D915C91179738
:10C36000C501B4010F94C8BC9B01AC010F94C8BCBB
:10C37000F70164A775A786A797A70130110541F0BB
:10C3800080A691A6A2A6B3A684829582A682B78231
:10C390000F5F1F4FD30114962D913D914D915C91EC
:10C3A000179718966D917D918D919C911B970F9485
:10C3B000C7BC20E030E040EC50E40F9476C0F201BE
:10C3C0006083718382839383F4E0CF0ED11C2CE2CF
:10C3D000E20EF11C34E0630E711C88E2480E511C21
:10C3E0000530110509F0B0CF8E010B5A1F4F6E01B9
:10C3F00091E5C90ED11C22242394312C2C0E3D1E14
:10C40000A8ED2A0E311CF801B897208131814281B4
:10C410005381F80160817181828193810F94A8BD5D
:10C420004B015C01E12CF12C3601F8E26F1A710826
:10C4300026014E0C5F1CF301EE0DFF1D248135819A
:10C4400046815781C501B4010F9476C09B01AC01B0
:10C45000D20114966D917D918D919C9117970F94B7
:10C46000C7BCF2016483758386839783F4E0EF0E83
:10C47000F11C24E1E216F104D9F6045D1F4F38E205
:10C48000C30ED11C0215130509F0BDCF1E0185EBAB
:10C49000280E311C6E0191EBC90ED11C3E01A7EE96
:10C4A0006A1AADEF7A0A14E0E12EF12C270100E0C0
:10C4B00010E0812C912CA12CB12CF601E00FF11F82
:10C4C000D301A00FB11F2D913D914D915C916081E1
:10C4D0007181828193810F9476C09B01AC01B4017C
:10C4E000C5010F94C8BC4B015C01BFEF4B1A5B0A3E
:10C4F0000C5F1F4FE5E04E165104F9F69B01AC01AD
:10C50000D1016D917D918D919C910F94C7BCF601E5
:10C5100020813181428153810F94A8BDD3016D9355
:10C520007D938D939C931397B1E0EB1AF108E8E2A9
:10C530002E1A3108FCE2CF1AD10824E0621A7108E1
:10C54000E114F10409F0B2CFCB50DE4F888199811C
:10C55000AA81BB81C55FD140C957DD4F88839983CC
:10C56000AA83BB83C758D2408E01075F1D4FDE01EF
:10C57000AF5CBD4FC558DD4FB983A883CB57D240C0
:10C58000C359DD4F2880CD56D240CD58DD4F38807D
:10C59000C357D240FE01EF51FE4FC358DD4FF98320
:10C5A000E883CD57D240C358DD4FA881B981CD571C
:10C5B000D240CD90DD90ED90FD90C358DD4FB98312
:10C5C000A883CD57D240C958DD4F288139814A818F
:10C5D0005B81C757D240C701B6010F94A1BD1816A1
:10C5E000B4F0C358DD4FE881F981CD57D2402081A6
:10C5F000318142815381C958DD4F688179818A81B7
:10C600009B81C757D2400F94A1BD1816FCF4CF5898
:10C61000DD4F28813981C157D2402430310509F0DE
:10C620001FC1C957DD4F288139814A815B81C758B5
:10C63000D240C958DD4F688179818A819B81C75773
:10C64000D2400F94A4BF18160CF00AC1D80114965A
:10C650008D919D910D90BC91A02DC158DD4F888387
:10C660009983AA83BB83CF57D240F8014080518081
:10C6700062807380C558DD4FA881B981CB57D24005
:10C680008D919D910D90BC91A02DC359DD4F888354
:10C690009983AA83BB83CD56D240D1018D919D91C0
:10C6A0000D90BC91A02DCD57DD4F88839983AA832F
:10C6B000BB83C358D240A7019601C958DD4F68819A
:10C6C00079818A819B81C757D2400F94C7BCCD58CE
:10C6D000DD4F688379838A839B83C357D24020E0F0
:10C6E00030E040E450E40F94D9C06B017C01A30119
:10C6F0009201C158DD4F688179818A819B81CF5732
:10C70000D2400F94C7BC4B015C0120E030E040EC0C
:10C7100050E4C359DD4F688179818A819B81CD5670
:10C72000D2400F9476C09B01AC01C501B4010F94B7
:10C73000A8BDA70196010F9476C06B017C0120E093
:10C7400030E040E05FE3C301B2010F9476C04B01DB
:10C750005C01CD58DD4F288139814A815B81C35707
:10C76000D240CA01B9010F9476C09B01AC01C5014A
:10C77000B4010F9476C09B01AC01C701B6010F94C0
:10C78000C8BC6B017C01CD57DD4F288139814A81BE
:10C790005B81C358D240F1016481758186819781A4
:10C7A0000F94C7BCC359DD4F288139814A815B8111
:10C7B000CD56D2400F94A8BD4B015C01C359DD4F4B
:10C7C000288139814A815B81CD56D240CA01B901A5
:10C7D0000F94C8BCA30192010F9476C02B013C01B9
:10C7E000C359DD4F288139814A815B81CD56D240C2
:10C7F000C158DD4F688179818A819B81CF57D240B2
:10C800000F9476C09B01AC01C301B2010F94C8BC68
:10C8100020E030E040EC50E40F94A8BD9B01AC0157
:10C82000C501B4010F94C7BCCD58DD4F28813981B3
:10C830004A815B81C357D2400F9476C09B01AC0103
:10C84000C701B6010F94C8BCCD57DD4F288139818F
:10C850004A815B81C358D2400F94C8BC4B015C0134
:10C86000CF58DD4F28813981C157D2402F5F3F4FCC
:10C87000CF58DD4F39832883C157D2400C5F1F4FFB
:10C88000C558DD4F88819981CB57D2400496C55851
:10C89000DD4F99838883CB57D24094E0290E311C19
:10C8A0002530310509F07FCE04C0812C912CA12CBC
:10C8B000B12CB401C501C657DD4F0FB6F894DEBFE9
:10C8C0000FBECDBFDF91CF911F910F91FF90EF90E1
:10C8D000DF90CF90BF90AF909F908F907F906F90A0
:10C8E0005F904F903F902F900895CF92DF92EF92FC
:10C8F000FF926B017C0180915D0B8823A1F086EA99
:10C900009FE00F941FCA882371F0C701B60106DCAF
:10C91000209148193091491940914A1950914B1969
:10C920000F94A8BD03C060E070E0CB01FF90EF90D2
:10C93000DF90CF9008954F925F926F927F928F9287
:10C940009F92AF92BF92CF92DF92EF92FF920F939E
:10C950001F93CF93DF93CDB7DEB728970FB6F89428
:10C96000DEBF0FBECDBF0F94E21E809156029091A4
:10C9700057029093610B8093600BE091CC0AF0E03A
:10C98000EE0FFF1FE958F54E60817181882777FD12
:10C990008095982F0F9443BE6093510B7093520B68
:10C9A0008093530B9093540B8091CA0A9091CB0AB9
:10C9B0009093500B80934F0B0F94CAB46093370B36
:10C9C0007093380B8093390B90933A0B8091E00A67
:10C9D0009091E10AA091E20AB091E30A89839A83D7
:10C9E000AB83BC8380933F0B9093400BA093410B90
:10C9F000B093420B4090E40A5090E50A6090E60A3A
:10CA00007090E70A4092430B5092440B6092450BA2
:10CA10007092460B8091E80A9091E90AA091EA0A87
:10CA2000B091EB0A8D839E83AF83B8878093470BC9
:10CA30009093480BA093490BB0934A0B6091EC0A7A
:10CA40007091ED0A8091EE0A9091EF0A60934B0B82
:10CA500070934C0B80934D0B90934E0B20E030E085
:10CA600040E85FE30F94C7BC6093EC0A7093ED0A53
:10CA70008093EE0A9093EF0A8CEC9AE09F938F9349
:10CA8000812C912CB8ECAB2EB3E4BB2E1CEEC12E46
:10CA90001AE0D12EED80FE800F811885A30192014E
:10CAA00069817A818B819C810F94330520E030E08D
:10CAB00040EA51E46091E80A7091E90A8091EA0A3B
:10CAC0009091EB0A0F94C8BC2B013C010F900F9082
:10CAD00020E030E042E553E40F94A4BF18164CF078
:10CAE0004092E80A5092E90A6092EA0A7092EB0AD0
:10CAF0000CC080E090E0A2E5B3E48093E80A909354
:10CB0000E90AA093EA0AB093EB0AE090E80AF090F1
:10CB1000E90A0091EA0A1091EB0A2091E40A3091A7
:10CB2000E50A4091E60A5091E70A6091E00A7091A7
:10CB3000E10A8091E20A9091E30AACEC6A2EAAE045
:10CB40007A2E7F926F92812C912CB0E7AB2EB1E4BC
:10CB5000BB2EECEECE2EEAE0DE2E0F9433051092C3
:10CB6000781A1092771A10927A1A1092791A1092F3
:10CB70007C1A10927B1A80E090E0A8E4B2E48093E3
:10CB8000E00A9093E10AA093E20AB093E30A80E0FE
:10CB900090E0AEE3B3E48093E40A9093E50AA093B7
:10CBA000E60AB093E70AE090E80AF090E90A0091FB
:10CBB000EA0A1091EB0A7F926F92812C912CF8E493
:10CBC000AF2EF2E4BF2E9C01AD01C501B4010F945C
:10CBD00033051092CB0A1092CA0A0F900F900F9053
:10CBE0000F9028960FB6F894DEBF0FBECDBFDF9131
:10CBF000CF911F910F91FF90EF90DF90CF90BF905A
:10CC0000AF909F908F907F906F905F904F900D941A
:10CC1000E21EE091CC0A84E0E89FF0011124E15982
:10CC2000F54E4081518162817381E0E9FAE084919F
:10CC3000882341F09091C00095FFFCCF8093C600FF
:10CC40003196F5CF22E030E08EE799E00E9428434C
:10CC5000ECE8FAE08491882341F09091C00095FFC0
:10CC6000FCCF8093C6003196F5CF6091CC0A70E07E
:10CC70004AE050E08EE799E00E943542E8E8FAE0A9
:10CC80008491882341F09091C00095FFFCCF809360
:10CC9000C6003196F5CF40915D1A50915E1A6091B1
:10CCA0005F1A7091601A21E030E08EE799E00E94EF
:10CCB00028438091C00085FFFCCF8AE08093C600A6
:10CCC0000895CF93DF93CDB7DEB72B970FB6F894C7
:10CCD000DEBF0FBECDBF0F94CAB46F83788789873C
:10CCE0009A8720916C0B2B87179A1092D10A169A6B
:10CCF0001092D20A6CE082E00F94BE3B6CE082E0BE
:10CD00000F94FF3B64E183E00F94BE3B64E183E05A
:10CD10000F94FF3BE3E8FAE08491882341F090917F
:10CD2000C00095FFFCCF8093C6003196F5CF80916F
:10CD3000C00085FFFCCF8AE08093C60083E40F9497
:10CD4000DB3E1C0140902110509022106090231077
:10CD5000709024100F942614481A590A610871081B
:10CD60000E94D0C9481A590A6108710877FE03C0A9
:10CD7000412C512C320190916413809163139817C8
:10CD800099F0E091631387E5E89FF0011124EB59D6
:10CD9000FC4E20E030E040E752E462A173A184A1A0
:10CDA00095A10F9476C008C060910C0270910D029D
:10CDB00080910E0290910F020F9410BE7E836D83BE
:10CDC0000F94B8030E9476C210926C0B789420E006
:10CDD00030E040E85FE36091EC0A7091ED0A8091E9
:10CDE000EE0A9091EF0A0F94C7BC69837A838B8314
:10CDF0009C83E090E80AF090E90A0091EA0A109119
:10CE0000EB0A2091E40A3091E50A4091E60A50913C
:10CE1000E70A6091E00A7091E10A8091E20A90913C
:10CE2000E30AACECBAE0BF93AF93812C912CE8EC11
:10CE3000AE2EE3E4BE2EDE0111966D010F94330594
:10CE400020E030E040E85FE36091EC0A7091ED0A89
:10CE50008091EE0A9091EF0A0F94C7BC69837A83A0
:10CE60008B839C832AE037ED43E25FE36091E80A1D
:10CE70007091E90A8091EA0A9091EB0A0F94C8BC7C
:10CE80006B017C0167E074E062197309F4E0769548
:10CE90006795FA95E1F780E090E00F9441BE20910C
:10CEA00048193091491940914A1950914B190F94E2
:10CEB000A8BD9B01AC01C701B6010F94C8BC7B01A2
:10CEC0008C012091E40A3091E50A4091E60A5091E4
:10CED000E70A6091E00A7091E10A8091E20A90917C
:10CEE000E30AACECBAE0BF93AF93812C912CA0E2A3
:10CEF000AA2EA2E4BA2EDE0111966D010F9433051D
:10CF0000B301A20181E99FE00F9443CA0F900F90F3
:10CF10000F900F9005E71FE0F12CB3E0EB2E80910E
:10CF20007712882341F18F2D6E2D0F9444C2B5E105
:10CF30008B02F001112423E09202E00DF11D112477
:10CF4000EE0FFF1FEE0FFF1FE958FD4E20E030E00F
:10CF50004AE754E461817281838194810F9476C0A1
:10CF600020E030E040E05FE30F94C8BC0F947EBE49
:10CF70000F9410BE02C060E070E0C8010F944BCA6D
:10CF8000F3940E5F1F4F89E0F812C9CFB10183E718
:10CF90009FE00F944BCA4091E00A5091E10A6091E2
:10CFA000E20A7091E30A8DE99FE00F9443CA409131
:10CFB000E40A5091E50A6091E60A7091E70A81EA75
:10CFC0009FE00F9443CA4091E80A5091E90A6091AA
:10CFD000EA0A7091EB0A8DE89FE00F9443CA4091F2
:10CFE000EC0A5091ED0A6091EE0A7091EF0A8EE61C
:10CFF0009FE00F9443CA6091650B81E0682782E748
:10D000009FE00F9431CABE016B5F7F4F89E89FE0BC
:10D010000F946F50E091CC0AF0E0EE0FFF1FE9583B
:10D02000F54E60818CE89FE00F9431CA6091751ACB
:10D030008BE89FE00F9431CA6091CA0A88E89FE0AC
:10D040000F9431CA9B85992329F061E085EA9FE01E
:10D050000F9431CA0F94E21EEEE7FAE08491882320
:10D0600041F09091C00095FFFCCF8093C6003196AF
:10D07000F5CF83E40F94DB3E4AE050E0BC018EE73D
:10D0800099E00E94874284E69FE00F941FCA61E006
:10D09000680F84E69FE00F9431CAE3E7FAE08491D9
:10D0A000882341F09091C00095FFFCCF8093C6008B
:10D0B0003196F5CF8091C00085FFFCCF8AE0809348
:10D0C000C6000F94CAB4AB01BC018F819885A985B5
:10D0D000BA85481B590B6A0B7B0B2AE030E08EE7C0
:10D0E00099E00E949342F894FFCF6F987798EAE610
:10D0F000F0E080818F7B8083808180688083EF9ADD
:10D1000008951F920F920FB60F9211240BB60F9233
:10D110000F931F932F933F934F935F936F937F933F
:10D120008F939F93AF93BF93EF93FF938091CA0A1E
:10D130009091CB0A8B3491050CF441C080916A0028
:10D1400086FF0BC00F94CAB46093330B7093340BFB
:10D150008093350B9093360B2CC00F94CAB400917A
:10D16000330B1091340B2091350B3091360B601B33
:10D17000710B820B930B2091CA0A3091CB0A253692
:10D1800031052CF003E010E020E030E004C004E0C2
:10D1900010E020E030E0601771078207930748F045
:10D1A0008091120B9091130B02969093130B809326
:10D1B000120B80916A0090E4892780936A00FF91A6
:10D1C000EF91BF91AF919F918F917F916F915F91FF
:10D1D0004F913F912F911F910F910F900BBE0F9088
:10D1E0000FBE0F901F9018956C987498EAE6F0E0C7
:10D1F00080818160808380818D7F8083EC9A089517
:10D200001F920F920FB60F9211240BB60F922F930D
:10D210003F934F935F936F937F938F939F93AF93BE
:10D22000BF93EF93FF93EC98EEE6FAE084918823A6
:10D2300041F09091C00095FFFCCF8093C6003196DD
:10D24000F5CF8091C00085FFFCCF8AE08093C600B7
:10D2500080916C0B811135DDFF91EF91BF91AF9102
:10D260009F918F917F916F915F914F913F912F91FE
:10D270000F900BBE0F900FBE0F901F9018954F92FE
:10D280005F926F927F928F929F92BF92CF92DF9226
:10D29000EF92FF920F931F93CF93DF93CDB7DEB73B
:10D2A000EA970FB6F894DEBF0FBECDBF88E89FE0C7
:10D2B0000F941FCAB82EBE01675C7F4F89E89FE0BC
:10D2C0000F948050EDE0F9E08491882341F0909133
:10D2D000C00095FFFCCF8093C6003196F5CF69ADB5
:10D2E0007AAD4AE050E08EE799E00E943C4283E646
:10D2F0009FE00F941FCA882E912C4AE050E0B401A1
:10D300008EE799E00E943C4203E11FE0E12CF12C02
:10D310003E0184E3680E711CE814F9042CF5FE014B
:10D32000BC962F016801C6010F941FCAF2018193B8
:10D330002F01FFEFCF1ADF0A46145704A1F71CAAEA
:10D34000BE01645D7F4F8EE799E00E942842BE01D6
:10D35000645D7F4F8AE69BE00E9454C08FEFE81A1D
:10D36000F80A085F1F4FD8CF8E01015E1F4F85E975
:10D37000E82E8FE0F82ED02EC12EC7010F941FCAC1
:10D38000F80181938F01FFEFEF1AFF0A8DE9E8168C
:10D390008FE0F80691F71FA2ED2DFC2D81918823D7
:10D3A00039F09091C00095FFFCCF8093C600F6CF76
:10D3B00068E079E08D2D9C2D0F94C3C5CF92DF924C
:10D3C00081E099E09F938F938E010F5F1F4F1F9312
:10D3D0000F930F94F3C70F900F900F900F900F9033
:10D3E0000F907E0195E0E90EF11CF7018081882302
:10D3F00049F0992787FD90950F94B2C5F701819365
:10D400007F01F3CF60E0C8010E94ECC281E99FE098
:10D410000F9427CAF62EE72ED82EC92EE6EEF8E096
:10D420008491882341F09091C00095FFFCCF8093B8
:10D43000C6003196F5CF2AE030E04F2D5E2D6D2DE0
:10D440007C2D8EE799E00E94934261E082EE98E0A5
:10D450000E94ECC26DED78E0C8010F94CEC58DE955
:10D460009FE00F9427CA6DAB7EAB8FAB98AFCE0118
:10D47000C5960F94D154BC01C8010F945DC66AEDE6
:10D4800078E0C8010F94C3C581EA9FE00F9427CAD2
:10D490006DAB7EAB8FAB98AFCE01C5960F94D154D8
:10D4A000BC01C8010F945DC663ED78E0C8010F941C
:10D4B000C3C560E0C8010E94ECC26EEC78E0C80110
:10D4C0000F94CEC58DE89FE00F9427CA6DAB7EAB5D
:10D4D0008FAB98AFCE01C5960F94D154BC01C80153
:10D4E0000F945DC660E0C8010E94ECC261E083EC6D
:10D4F00098E00E94ECC28AAD8F9389AD8F938CEB3C
:10D5000098E09F938F931F930F930F94F3C760E05E
:10D51000C8010E94ECC265EB78E0C8010F94CEC54B
:10D520008B2D90E09EAB8DABCE01C5960F94A65788
:10D53000BC01C8010F945DC660E0C8010E94ECC246
:10D54000CF92DF92EF92FF928CEA98E09F938F93B5
:10D550001F930F930F94F3C760E0C8010E94ECC2C1
:10D5600061E088EA98E00E94ECC20FB6F894DEBF52
:10D570000FBECDBFEA960FB6F894DEBF0FBECDBF8B
:10D58000DF91CF911F910F91FF90EF90DF90CF909F
:10D59000BF909F908F907F906F905F904F90089575
:10D5A0004F925F926F927F92AF92BF92CF92DF9233
:10D5B000EF92FF920F931F93CF93DF93CDB7DEB718
:10D5C000E0970FB6F894DEBF0FBECDBF2B013C0134
:10D5D00069017A0180911F0A8111E5C0F8940F94C6
:10D5E00006148091211090912210A0912310B091E7
:10D5F000241080931B0A90931C0AA0931D0AB093D9
:10D600001E0A0F94261440911B0A50911C0A609127
:10D610001D0A70911E0A481B590B6109710940933C
:10D620001B0A50931C0A60931D0A70931E0A0E94E5
:10D63000D0C940911B0A50911C0A60911D0A70913B
:10D640001E0A481B590B6109710940931B0A50932C
:10D650001C0A60931D0A70931E0A909164138091B6
:10D660006313981799F0E091631387E5E89FF00141
:10D670001124EB59FC4E20E030E040E752E462A177
:10D6800073A184A195A10F9476C008C060910C028B
:10D6900070910D0280910E0290910F026093070A23
:10D6A0007093080A8093090A90930A0A0F94B803AA
:10D6B00080E1E0EEFAE0ABE0BAE001900D928A95ED
:10D6C000E1F78091CC0A8093060A8091070280934B
:10D6D000050A0E9476C210926C0B81E080931F0AAB
:10D6E000789420E030E0A901C301B2010F94A1BDFC
:10D6F00081110AC020E030E0A901C701B6010F94F2
:10D70000A1BD882309F44FC063EA78E0FE01319699
:10D710005F01CF010F94CEC5F50101900020E9F71C
:10D720008F01015011092091130A3091140A409180
:10D73000150A5091160AC301B2010F94C8BC23E028
:10D7400048E00F94F1C260EA78E0C5010F94C3C5C8
:10D75000F50101900020E9F78F010150110923E044
:10D7600046E0C701B6010F94F1C26DE978E0C5014A
:10D770000F94C3C5F50101900020E9F78F01015016
:10D780001109609160027091610280916202909132
:10D79000630223E048E00F94F1C260E0C5010E94FB
:10D7A000ECC20E948BC4E0960FB6F894DEBF0FBEA9
:10D7B000CDBFDF91CF911F910F91FF90EF90DF9040
:10D7C000CF90BF90AF907F906F905F904F900895F3
:10D7D00020E030E0A90160E070E080E291E4E0CE7A
:10D7E0008F929F92AF92BF92CF92DF92EF92FF9271
:10D7F0000F931F93CF93DF9300D01F92CDB7DEB767
:10D800009B01AC0180911F0A882309F497C0809185
:10D81000060A8093CC0A8091070A9091080AA09189
:10D82000090AB0910A0A80930C0290930D02A0930A
:10D830000E02B0930F026091170A7091180A80913E
:10D84000190A90911A0A0F94C7BC69837A838B8353
:10D850009C83CE0101960F948C1320E030E040E5CC
:10D8600051E4609160027091610280916202909136
:10D8700063020F94A8BD4B015C01E090130AF09085
:10D88000140A0091150A1091160A20910F0A30917E
:10D89000100A4091110A5091120A60910B0A70917E
:10D8A0000C0A80910D0A90910E0AECECFAE0FF93BD
:10D8B000EF93E7E1CE2EEAE0DE2E0F9433050F94CE
:10D8C000E21E80E1EBE0FAE0A0EEBAE001900D92FA
:10D8D0008A95E1F780E1E0EEFAE0ABEABAE0019088
:10D8E0000D928A95E1F740911B0A50911C0A6091B4
:10D8F0001D0A70911E0A4093080E5093090E609302
:10D900000A0E70930B0E83E59DE00E945AAA809147
:10D910001B0A90911C0AA0911D0AB0911E0A8093C7
:10D92000211090932210A0932310B093241081E033
:10D9300080936C0B10921F0A0F900F900F900F9016
:10D940000F900F90DF91CF911F910F91FF90EF906B
:10D95000DF90CF90BF90AF909F908F90089560E040
:10D9600070E0CB013DCFFBDF81E08093B1020895F1
:10D97000E8E8F8E08491882341F09091C00095FF99
:10D98000FCCF8093C6003196F5CF4091E00A5091CC
:10D99000E10A6091E20A7091E30A23E030E08EE749
:10D9A00099E00E942843E5E8F8E08491882341F05B
:10D9B0009091C00095FFFCCF8093C6003196F5CFC3
:10D9C0004091E40A5091E50A6091E60A7091E70AF5
:10D9D00023E030E08EE799E00E942843E2E8F8E097
:10D9E0008491882341F09091C00095FFFCCF8093F3
:10D9F000C6003196F5CF4091E80A5091E90A60914E
:10DA0000EA0A7091EB0A23E030E08EE799E00E9489
:10DA10002843E0E8F8E08491882341F09091C00029
:10DA200095FFFCCF8093C6003196F5CF8091C00062
:10DA300085FFFCCF8AE08093C6000895E8E6F8E011
:10DA40008491882341F09091C00095FFFCCF809392
:10DA5000C6003196F5CF0F94511FAB01BC0123E0F6
:10DA600030E08EE799E00E942843E5E6F8E08491F3
:10DA7000882341F09091C00095FFFCCF8093C600B1
:10DA80003196F5CF81E00F94511FAB01BC0123E02B
:10DA900030E08EE799E00E942843E2E6F8E08491C6
:10DAA000882341F09091C00095FFFCCF8093C60081
:10DAB0003196F5CF82E00F94511FAB01BC0123E0FA
:10DAC00030E08EE799E00E942843E0E6F8E0849198
:10DAD000882341F09091C00095FFFCCF8093C60051
:10DAE0003196F5CF8091C00085FFFCCF8AE080930E
:10DAF000C6000895EF92FF920F931F93CF93DF9389
:10DB0000ECE4F8E08491882341F09091C00095FF07
:10DB1000FCCF8093C6003196F5CF07E712E1FAE417
:10DB2000EF2EF8E0FF2EC0E0D0E0F801EC0FFD1F73
:10DB3000418152816381748123E030E08EE799E076
:10DB40000E942843F7018491EAE4F8E0882349F031
:10DB50009091C00095FFFCCF8093C60031968491D0
:10DB6000F5CF2496CC31D10501F7045E1F4FF3E1C8
:10DB70000B331F07C1F6E9E4F8E08491882341F0F4
:10DB80009091C00095FFFCCF8093C6003196F5CFF1
:10DB90008091C00085FFFCCF8AE08093C600DF91B2
:10DBA000CF911F910F91FF90EF9008952F923F9288
:10DBB0004F925F926F927F928F929F92AF92BF929D
:10DBC000CF92DF92EF92FF920F931F93CF93DF9349
:10DBD000CDB7DEB7C355D1090FB6F894DEBF0FBE7F
:10DBE000CDBF82E090E0909316028093150286EEFE
:10DBF00093E00E9410448823B1F0809139109091F5
:10DC00003A106AE270E005960F9468C6009711F02A
:10DC1000DC011C928091391090913A1005960F9476
:10DC20004C510C940B9A87ED93E00E94104488238A
:10DC300021F00E947E480C940B9A8BEE93E00E9498
:10DC40001044882319F08FDE0C940B9A89EF93E02F
:10DC50000E941044882321F00E94BA480C940B9A29
:10DC600086E094E00E941044882309F4C4C18CE04B
:10DC700094E00E941044882391F08091921B8823A5
:10DC800011F40C940B9A0F94CAB46093660B7093C2
:10DC9000670B8093680B9093690B0C940B9A81E14E
:10DCA00094E00E941044882361F060912D0B7091E4
:10DCB0002E0B4AE050E08EE799E00E9487420C94D8
:10DCC0000B9A85E194E00E941044882309F446C031
:10DCD000E9E1F4E08191882339F09091C00095FF4B
:10DCE000FCCF8093C600F6CF80910C0B90910D0B6A
:10DCF0002CE3289FB001299F700D11244AE050E0C9
:10DD00008EE799E00E9435426DE174E08EE799E07C
:10DD10000E942842E2E2F4E08191882339F0909158
:10DD2000C00095FFFCCF8093C600F6CF80910E0B0C
:10DD300090910F0B2CE3289FB001299F700D1124A7
:10DD40004AE050E08EE799E00E9435426DE174E0D0
:10DD50008EE799E00E9428420C940B9A88E294E0A6
:10DD60000E9410448823C1F08091921B882361F0A7
:10DD70006091901B7091911B4AE050E08EE799E012
:10DD80000E943C420C940B9A6BE274E08EE799E09F
:10DD90000E9428420C940B9A8DE394E00E94104458
:10DDA000882379F16091391070913A106D5F7F4F3F
:10DDB00021E041E08AE69BE00E94AEBC80915B0DD1
:10DDC00090915C0DA0915D0DB0915E0D8093080E59
:10DDD0009093090EA0930A0EB0930B0E83E59DE07D
:10DDE0000E9491A92091C00025FFFCCF8093C6001E
:10DDF0000A9721F760E08AE69BE00E943EBC0C9403
:10DE00000B9A80E494E00E941044882399F00E94C9
:10DE1000AA5181E080932F0B6091391070913A10D4
:10DE20006C5F7F4F21E040E08AE69BE00E94AEBC41
:10DE30000C940B9A84E494E00E941044882309F423
:10DE400045C08091921B882309F49ECF1092030A4B
:10DE5000E7E4F4E08191882339F09091C00095FFC8
:10DE6000FCCF8093C600F6CF00E010E0FF24F394CF
:10DE70008091FF099091000A2091010A3091020AD5
:10DE8000821B930B8F779927892B89F08EE799E076
:10DE90000E944241F092030A9091C00095FFFCCF8E
:10DEA0008093C6000F5F1F4F1092030AE1CF03312A
:10DEB0001105F4F281E08093030A8091C00085FF90
:10DEC000FCCF8AE08093C6000C940B9A8AE494E01D
:10DED0000E9410448823A9F0EEE4F4E081918823A5
:10DEE00039F09091C00095FFFCCF8093C600F6CF2B
:10DEF0008091C00085FFFCCF8AE08093C6000C941F
:10DF00000B9A88E594E00E9410448823A9F0ECE580
:10DF1000F4E08191882339F09091C00095FFFCCF07
:10DF20008093C600F6CF8091C00085FFFCCF8AE0C9
:10DF30008093C6000C940B9A8AE794E00E941044E8
:10DF4000882321F00F94EA500C940B9A8FE794E009
:10DF50000E941044882341F060E070E088EF9FE069
:10DF60000F946F500C940B9A82E894E00E94104436
:10DF7000882359F062E874E08EE799E00E94284215
:10DF800040E052EC61E070E010C08DE894E00E9447
:10DF90001044882381F06DE874E08EE799E00E94D8
:10DFA000284240E054E961E170E08EE799E00E9488
:10DFB000C7400C94759B89E994E00E941044882323
:10DFC00061F00F94CAB46093590B70935A0B80930D
:10DFD0005B0B90935C0B0C940B9A8EE994E00E947F
:10DFE0001044882311F40C940B9A61E080E00E94A5
:10DFF000C5480C940B9A8EE50E94E24381110C9463
:10E000000B9A87E40E94E243882311F40C94B77FB3
:10E010000E944F440F9410BE6C34710509F430C453
:10E020007CF56430710509F409C154F4623071055E
:10E0300009F4ECC00CF0F6C077FF78C00C940B9A92
:10E040006C31710509F451C17CF46A30710509F431
:10E0500046C16B30710511F00C940B9A60E080E0C2
:10E060000E94AD590C940B9A6E31710509F44DC3A1
:10E070006B34710511F00C940B9A08E210E0F6C3B2
:10E080006735710511F40C94377F14F5603571050F
:10E0900011F40C9410796CF46F34710511F00C9438
:10E0A0000B9A0FEF10E0AEE0CA2EADE0DA2E0C9422
:10E0B000FB786135710511F40C947E7E663571052F
:10E0C00011F00C940B9A86EE0E9435480C940B9A32
:10E0D0006C35710511F40C94407F7CF46A35710540
:10E0E00011F40C943C7F6B35710511F00C940B9A74
:10E0F00081E08093960A0C940B9A6236710511F4B4
:10E100000C94A27F6336710511F00C940B9A109257
:10E11000921B0F94EF506091921B84EC9FE00F9440
:10E1200031CA82E00F94E5960C940B9A8091800A94
:10E1300081110C940B9A0E94E2556091290B709109
:10E140002A0B80912B0B90912C0B0F9441BE6B01ED
:10E150007C014090EC0A5090ED0A6090EE0A7090BD
:10E16000EF0A8090B70A9090B80AA090B90AB090D0
:10E17000BA0AA5019401C301B2010F94C7BC20E003
:10E1800030E048EC52E40F9476C09B01AC01C7012B
:10E19000B6010F94A4BF1816E4F4A3019201C501BF
:10E1A000B4010F94C7BC20E030E048EC52E40F9477
:10E1B00076C09B01AC01C701B6010F94C8BC0F9497
:10E1C00015BE6093290B70932A0B80932B0B9093B1
:10E1D0002C0B8091C90A8823A9F088E50E94E243AC
:10E1E000811110C089E50E94E24381110BC08AE5CC
:10E1F0000E94E243811106C085E40E94E24381113E
:10E200000C94149A0E94AA580C940B9A8091800A3C
:10E2100081110C940B9A0E94655681E00E94885BE4
:10E220000C940B9A8091800A81110C940B9A0E9495
:10E23000655680E00E94885B0C940B9A80E50E94F2
:10E24000E243882339F00E944F440F9415BE6B01BE
:10E250007C0103C0C12CD12C760183E50E94E243EE
:10E26000882361F00E944F4420E030E04AE754E404
:10E270000F9476C00F9415BE6B017C01C114D104BC
:10E28000E104F10431F0E0EDF2E4859194910F9412
:10E2900059510F94E21E0F94CAB44B015C018C0CCF
:10E2A0009D1CAE1CBF1C0F94CAB46093920A70935D
:10E2B000930A8093940A9093950A0F94CAB46815B0
:10E2C00079058A059B0510F00C940B9A0F94CE2BC0
:10E2D00080E00E94B05C80E00F94E596EECF60E0B5
:10E2E00081E00E94AD590C940B9A0F94E21EECE36E
:10E2F000FEE08491882341F09091C00095FFFCCF0F
:10E300008093C6003196F5CF33DBEEE2FEE08491D8
:10E31000882341F09091C00095FFFCCF8093C60008
:10E320003196F5CF8BDB81E080935E0B88E50E9410
:10E33000E243182F89E50E94E243082F8AE50E94F4
:10E34000E243782E101308C0181711F0012F04C0F3
:10E350007724739401E011E00E9430DB6090771223
:10E360001092771282E00F94511F6093E80A709325
:10E37000E90A8093EA0A9093EB0A71100E9404F96B
:10E3800040910C0250910D0260910E0270910F02AB
:10E390004093970A5093980A6093990A70939A0A47
:10E3A00080915602909157029093610B8093600B7D
:10E3B00084E690E090935702809356020F94CAB47B
:10E3C0006093920A7093930A8093940A9093950AAB
:10E3D00081E00F94671580E1E0EEFAE0ABEABAE085
:10E3E00001900D928A95E1F710920C0210920D02A5
:10E3F00010920E0210920F02112321F080E090E0A3
:10E400000E944A4D002321F081E090E00E944A4D95
:10E4100088E50E94E243882341F00E940544672B6F
:10E42000682B692B11F00C94439A89E50E94E24312
:10E43000882341F00E940544672B682B692B11F05B
:10E440000C94599A772009F4F1C08091D10A88235D
:10E4500021F08091D20A811108C080E090E00E94F2
:10E460004A4D81E090E00E944A4D0E9485DBEAEC33
:10E47000F5E485919591A591B49189839A83AB83B5
:10E48000BC83E6ECF5E485919591A591B4918F8FCD
:10E4900098A3A9A3BAA32FEA3AE04BEA5AE0BE0137
:10E4A0006F5F7F4FCE014F960E9456460E94F7DA6B
:10E4B00020E030E040E850EC6091AF0A7091B00A83
:10E4C0008091B10A9091B20A0F94A1BD87FF0CC050
:10E4D00080E090E0A0E8B0EC8093AF0A9093B00A9F
:10E4E000A093B10AB093B20A80E090E0A0EAB0E451
:10E4F0008093B30A9093B40AA093B50AB093B60A76
:10E5000020E030E040E251E46091600270916102ED
:10E5100080916202909163020F94A8BD60930C02F7
:10E5200070930D0280930E0290930F021092E80AEE
:10E530001092E90A1092EA0A1092EB0A80E00F9416
:10E540006715E090E80AF090E90A0091EA0A109154
:10E55000EB0A2091E40A3091E50A4091E60A5091D5
:10E56000E70A6091E00A7091E10A8091E20A9091D5
:10E57000E30AFCEECF2EFAE0DF2E0F94E11180903B
:10E580000C0290900D02A0900E02B0900F02E0904D
:10E59000B30AF090B40A0091B50A1091B60A20911E
:10E5A000AF0A3091B00A4091B10A5091B20A60911D
:10E5B000AB0A7091AC0A8091AD0A9091AE0AECEC76
:10E5C000FAE0FF93EF93A7EBCA2EAAE0DA2E0F949E
:10E5D00033050F94E21E8091AB0A9091AC0AA09192
:10E5E000AD0AB091AE0A8093E00A9093E10AA0933D
:10E5F000E20AB093E30A8091AF0A9091B00AA09129
:10E60000B10AB091B20A8093E40A9093E50AA0930C
:10E61000E60AB093E70A81E00F9467150F944F154F
:10E6200082E090E00E944A4D0F900F908AE50E9490
:10E63000E243882341F00E940544672B682B692B35
:10E6400011F00C946F9AE090E80AF090E90A0091BA
:10E65000EA0A1091EB0A2091E40A3091E50A409110
:10E66000E60A5091E70A6091E00A7091E10A809110
:10E67000E20A9091E30AECEECE2EEAE0DE2E0F9451
:10E68000E11180E00F9467158091970A9091980AA4
:10E69000A091990AB0919A0A80930C0290930D026E
:10E6A000A0930E02B0930F028091600B9091610BCA
:10E6B00090935702809356020F94CAB46093920AC3
:10E6C0007093930A8093940A9093950A0F944F1530
:10E6D0000E9485DB0E94A1DD88E50E94E243811152
:10E6E0000C94859A89E50E94E24381110C94859AE5
:10E6F00087E50E94E24381110C94859A8AE50E9485
:10E70000E24381110C94859A87C50F94E21E81E043
:10E710000E948E438091600290916102A0916202FA
:10E72000B091630280930C0290930D02A0930E02AD
:10E73000B0930F0220E030E043E060E070E080E260
:10E7400091EC0E9430DEE8E6F3E485919491FC01BF
:10E750002491222341F03091C00035FFFCCF20935B
:10E76000C6000196F4CFE5E0FEE08491882341F0F5
:10E770009091C00095FFFCCF8093C6003196F5CFF5
:10E780004091E00A5091E10A6091E20A7091E30A37
:10E7900025E030E08EE799E00E942843E0E0FEE0CB
:10E7A0008491882341F09091C00095FFFCCF809325
:10E7B000C6003196F5CF4091E40A5091E50A609188
:10E7C000E60A7091E70A25E030E08EE799E00E94C2
:10E7D0002843EBEFFDE08491882341F09091C00045
:10E7E00095FFFCCF8093C6003196F5CF4091E80AA3
:10E7F0005091E90A6091EA0A7091EB0A25E030E055
:10E800008EE799E00E942843E9EFFDE08491882398
:10E8100041F09091C00095FFFCCF8093C6003196E7
:10E82000F5CF0E94BC430C940B9A9091C00095FFC9
:10E83000FCCF8093C60081918111F7CFB801882762
:10E8400077FD8095982F0F9443BE0E948E60AB0198
:10E85000BC0122E030E08EE799E00E9429430F5F7F
:10E860001F4F0F36110511F40C940B9A4AE050E03B
:10E87000B8018EE799E00E943542EDECF8E0DBCF7D
:10E880008091D10A882341F08091D20A882321F017
:10E890008091D30A811109C00E948BC461E082EF8C
:10E8A0009DE00E94D3C30C940B9A81E090E090937A
:10E8B000160280931502E4EDFDE08491882341F077
:10E8C0009091C00095FFFCCF8093C6003196F5CFA4
:10E8D0008091C00085FFFCCF8AE08093C6001A8239
:10E8E0001982C090691AD0906A1AE0906B1AF09061
:10E8F0006C1A20E030E040EA50E4C701B6010F9402
:10E90000A8BD0F9410BE45E0469F9001479F300D73
:10E910001124B901882777FD8095982F0F9443BE65
:10E920002B013C0120E030E04CE052E40F94A1BD0B
:10E9300087FF06C0412C512C2CE0622E22E4722E5F
:10E94000A7019601C301B2010F94A1BD87FF0AC0C0
:10E9500020E030E040EA50E4C301B2010F94C8BCAB
:10E960002B013C01E0ECFDE08491882341F0909183
:10E97000C00095FFFCCF8093C6003196F5CF22E012
:10E9800030E0B301A2018EE799E00E94294320E024
:10E9900030E040EF51E4C301B2010F94C7BC20E066
:10E9A00030E04CE852E40F94C8BC0F9410BE709352
:10E9B000761A6093751A84E090E09093220B80930E
:10E9C000210B81E090E09093200B80931F0BE0914E
:10E9D000300BF0E0EE0FFF1FE456FF4B8591949152
:10E9E00021E0892B09F420E02093240B80E090E0C3
:10E9F000A0EAB1E48093E00A9093E10AA093E20ACE
:10EA0000B093E30A80E090E0A0E7B2E48093E40AE8
:10EA10009093E50AA093E60AB093E70A8AE999E998
:10EA2000A9E1BEE38093E80A9093E90AA093EA0A79
:10EA3000B093EB0A8CEC9AE09F938F93812C912CEE
:10EA400018E4A12E12E4B12E0CEEC02E0AE0D02E56
:10EA50001AE9E12E19E9F12E09E11EE320E030E088
:10EA600040E752E460E070E080EA91E40F943305FF
:10EA70000F94E21E0F900F90A30192016091691A0A
:10EA800070916A1A80916B1A90916C1A0F94A1BDC3
:10EA900087FF07C088EE93E00E94D15E0E9409665E
:10EAA000EBCF60E086EA9FE00F9431CA80E090E00F
:10EAB000A0EAB0E48093E80A9093E90AA093EA0AF6
:10EAC000B093EB0A2091E40A3091E50A4091E60AFE
:10EAD0005091E70A6091E00A7091E10A8091E20AA0
:10EAE0009091E30AECECFAE0FF93EF93812C912CE8
:10EAF000E8E4AE2EE2E4BE2EFCEECF2EFAE0DF2EEE
:10EB0000E12CF12C00EA10E40F943305E6ECF5E477
:10EB100085919591A591B4918093E00A9093E10A33
:10EB2000A093E20AB093E30AEAECF5E4259135916B
:10EB3000459154912093E40A3093E50A4093E60A04
:10EB40005093E70AE090E80AF090E90A0091EA0A97
:10EB50001091EB0A6091E00A7091E10A8091E20A5B
:10EB60009091E30AECECFAE0FF93EF93812C912C67
:10EB7000B8E4AB2EB2E4BB2E0F9433050F94E21E23
:10EB800020E030E043E060E070E080E89FEB0E942E
:10EB900030DE8091E80A9091E90AA091EA0AB091EA
:10EBA000EB0A8AAF9BAFACAFBDAFEFEBFDE084915A
:10EBB0000F900F900F900F904091E80A5091E90A42
:10EBC0006091EA0A7091EB0A882349F09091C000A5
:10EBD00095FFFCCF8093C60031968491F5CF80914C
:10EBE000C00085FFFCCF8AE08093C600E8EBFDE023
:10EBF0008491882341F09091C00095FFFCCF8093D1
:10EC0000C6003196F5CF22E030E08EE799E00E9411
:10EC10002843E7EBFDE08491882341F09091C00008
:10EC200095FFFCCF8093C6003196F5CF8091C00050
:10EC300085FFFCCF8AE08093C6002EEAC22E2FE02B
:10EC4000D22E33E2E32EF12C0FEF1FEF4AE0342EE9
:10EC5000B701882777FD8095982F0F9443BE4B010D
:10EC60005C01E0EBFDE08491882341F09091C000CD
:10EC700095FFFCCF8093C6003196F5CF4AE050E077
:10EC8000B8016E5F7F4F8EE799E00E943542E3EA5C
:10EC9000FDE08491882341F09091C00095FFFCCF66
:10ECA0008093C6003196F5CF8091C00085FFFCCFE0
:10ECB0003092C600EFE8FDE08491882341F0909106
:10ECC000C00095FFFCCF8093C6003196F5CF4AE097
:10ECD00050E0B7018EE799E00E943542E0E8FDE0A0
:10ECE0008491882341F09091C00095FFFCCF8093E0
:10ECF000C6003196F5CF4AE050E060E070E08EE764
:10ED000099E00E943542EFE7FDE08491882341F0CD
:10ED10009091C00095FFFCCF8093C6003196F5CF4F
:10ED20008091C00085FFFCCF3092C6000F3FFFEFFF
:10ED30001F0731F0BE016F5F7F4FC6010F946F5008
:10ED4000A5019401C301B2010F94A1BD181664F48A
:10ED50000F5F1F4F25E0E20EF11C32E0C30ED11C05
:10ED60000530110509F074CF280187E2481A88EFB1
:10ED7000580A440C551C380193E0690E711C85E05B
:10ED8000809F1001819F300C112419AE18AEADE2A6
:10ED90002A0E311CC301029705970CF0CBC168AD58
:10EDA00079AD620D731D882777FD8095982F0F949C
:10EDB00043BE22966CAF7DAF8EAF9FAF2297E8E740
:10EDC000FDE08491882341F09091C00095FFFCCF35
:10EDD0008093C6003196F5CF4AE050E0B3018EE74C
:10EDE00099E00E943542E5E7FDE08491882341F0F7
:10EDF0009091C00095FFFCCF8093C6003196F5CF6F
:10EE00008091C00085FFFCCFFAE0F093C6007092BD
:10EE1000200B60921F0B20E030E040EF51E422967F
:10EE20006CAD7DAD8EAD9FAD22970F94C7BC20E039
:10EE300030E040E251E40F9476C020E030E040EA58
:10EE400050E40F94A8BD20E030E048E452E40F9471
:10EE5000C8BC0F9410BE7093761A6093751A80E048
:10EE600090E0A0EAB1E48093E00A9093E10AA093D5
:10EE7000E20AB093E30A80E090E0A0E7B2E4809376
:10EE8000E40A9093E50AA093E60AB093E70A8AE9B8
:10EE900099E9A9E1BEE38093E80A9093E90AA09377
:10EEA000EA0AB093EB0AACECBAE0BF93AF93812CC3
:10EEB000912CA8E4AA2EA2E4BA2EBCEECB2EBAE086
:10EEC000DB2E1AE9E12E19E9F12E09E11EE320E01B
:10EED00030E040E752E460E070E080EA91E40F94B3
:10EEE00033050F94E21E0F900F9022962CAD3DAD8E
:10EEF0004EAD5FAD22976091691A70916A1A809148
:10EF00006B1A90916C1A0F94A1BD87FF07C088EE11
:10EF100093E00E94D15E0E940966E7CF80E090E016
:10EF2000A0EAB0E48093E80A9093E90AA093EA0A81
:10EF3000B093EB0A2091E40A3091E50A4091E60A89
:10EF40005091E70A6091E00A7091E10A8091E20A2B
:10EF50009091E30AACECBAE0BF93AF93812C912C73
:10EF600018E4A12E12E4B12E0CEEC02E0AE0D02E31
:10EF7000E12CF12C00EA10E40F943305E6ECF5E403
:10EF800085919591A591B4918093E00A9093E10ABF
:10EF9000A093E20AB093E30AEAECF5E425913591F7
:10EFA000459154912093E40A3093E50A4093E60A90
:10EFB0005093E70AE090E80AF090E90A0091EA0A23
:10EFC0001091EB0A6091E00A7091E10A8091E20AE7
:10EFD0009091E30AACECBAE0BF93AF93812C912CF3
:10EFE000F8E4AF2EF2E4BF2E0F9433050F94E21E27
:10EFF00020E030E043E060E070E080E89FEB0E94BA
:10F0000030DE2AAD3BAD4CAD5DAD6091E80A70914C
:10F01000E90A8091EA0A9091EB0A0F94C7BC20910B
:10F0200048193091491940914A1950914B190F9440
:10F0300076C00F9410BE7A836983E4E7FDE0849183
:10F040000F900F900F900F90882349F09091C0007F
:10F0500095FFFCCF8093C60031968491F5CF8091C7
:10F06000C00085FFFCCFFAE0F093C600E0E6FDE0CB
:10F070008491882341F09091C00095FFFCCF80934C
:10F08000C6003196F5CF4091691A50916A1A609185
:10F090006B1A70916C1A22E030E08EE799E00E94C2
:10F0A0002843E1E5FDE08491882341F09091C00080
:10F0B00095FFFCCF8093C6003196F5CF2AAD3BADCE
:10F0C0004CAD5DAD6091E80A7091E90A8091EA0A61
:10F0D0009091EB0A0F94C7BCAB01BC0122E030E079
:10F0E0008EE799E00E942843E0E5FDE084918823C3
:10F0F00041F09091C00095FFFCCF8093C6003196FF
:10F10000F5CF8091C00085FFFCCFFAE0F093C600F8
:10F11000BE016F5F7F4FC2010F946F5022E0420E1D
:10F12000511C3FEF631A730A88AD99AD059699AFEC
:10F1300088AF30CE1092220B1092210B1092240B2C
:10F1400061E086EA9FE00F9431CAE1E1FDE084913D
:10F15000882341F09091C00095FFFCCF8093C600BA
:10F160003196F5CF8091C00085FFFCCF8AE0809377
:10F17000C600179A1092D10A169A1092D20A149ABF
:10F18000E091300BF0E0EE0FFF1FE856FF4B85914A
:10F1900094910F9459A481E00F94AC9982E00F945C
:10F1A000E5961092761A1092751A0C940B9A84E6D2
:10F1B00090E00E94D15E91E0E91AF108C1F74AE0BF
:10F1C00050E0B8018EE799E00E943542F6012491A3
:10F1D000EEE0FDE0211117C060910E0B70910F0B56
:10F1E0004AE050E08EE799E00E943C420550110948
:10F1F00011F40C940B9A1093CB0A0093CA0AF4E60C
:10F20000EF2EF12CD4CF3091C00035FFFCCF2093EE
:10F21000C60031962491DECF0F94E21E10925E0B51
:10F2200081E08093320B86E50E94E243882359F007
:10F23000E0913910F0913A108181893021F08F7D71
:10F2400011F00E94F8432091D10A8091961B909171
:10F25000971B222341F02091D20A222321F02091F2
:10F26000D30A21110FC0029749F00E948BC461E0BC
:10F2700087E09DE00E94D3C30C940B9A1092320B4E
:10F280000C940B9A1092040A029721F41092320BFC
:10F290000C940B9AF091240B2896FFAF289720919D
:10F2A000210B3091220B2A963FAF2EAF2A978091E7
:10F2B0001F0B9091200B2C969FAF8EAF2C9781E067
:10F2C0008093240B81E090E09093220B8093210B9C
:10F2D00083E190E09093200B80931F0B81E00F94CB
:10F2E000E59687E792E10E94CEF90E9404F980E05A
:10F2F00090E0A0EAB0E48093E80A9093E90AA09332
:10F30000EA0AB093EB0A20E030E040E752E4609173
:10F3100060027091610280916202909163020F9489
:10F32000A8BD4B015C012091E40A3091E50A4091AF
:10F33000E60A5091E70A6091E00A7091E10A809133
:10F34000E20A9091E30AECECFAE0FF93EF931CEEF3
:10F35000C12E1AE0D12EE12CF12C00EA10E40F941A
:10F360003305E6ECF5E485919591A591B4918093F0
:10F37000E00A9093E10AA093E20AB093E30AEAEC70
:10F38000F5E485919591A591B4918093E40A9093C9
:10F39000E50AA093E60AB093E70A64EE7AE080EE0D
:10F3A0009AE00E94104720E030E040EF51E4609185
:10F3B00058027091590280915A0290915B020F9409
:10F3C000A8BD4B015C01E090E80AF090E90A0091C9
:10F3D000EA0A1091EB0A2091E40A3091E50A409183
:10F3E000E60A5091E70A6091E00A7091E10A809183
:10F3F000E20A9091E30AECECFAE0FF93EF930F94AA
:10F4000033050F94E21E20E030E040EA51E46091C1
:10F4100058027091590280915A0290915B020F94A8
:10F42000A8BD0F9410BE8B0120E030E040E252E412
:10F43000609160027091610280916202909163021A
:10F440000F94A8BD0F9410BE7B010E94E3DA2396AF
:10F450008FAF239780E00E948E430F900F900F9004
:10F460000F90A6ECB5E4BBAFAAAF212C312CC7019D
:10F47000AA2797FDA095BA2F60968CAF9DAFAEAF2F
:10F48000BFAF6097C801AA2797FDA095BA2F6496D1
:10F490008CAF9DAFAEAFBFAF6497C10163E070E0CA
:10F4A0000F9465C27FAF6EAF99AF88AF9EAD90FFEE
:10F4B00008C0A2E0B0E0E8ADF9ADAE1BBF0BB9AF3C
:10F4C000A8AF2396FFAD2397FF2379F121143104D0
:10F4D00061F18EAD9FAD880F991F2EAD3FAD820FAC
:10F4E000931FA8ADB9AD8A0F9B1F880F991F8D532D
:10F4F000904F0F942CCABC01882777FD8095982FD8
:10F500000F9443BE2AE037ED43E25CE30F9476C0EC
:10F51000209178123091791240917A1250917B1299
:10F520000F94C8BC2B013C0103C0412C512C32016B
:10F5300080E090E0A0EAB0E48093E80A9093E90AC2
:10F54000A093EA0AB093EB0A60966CAD7DAD8EADE8
:10F550009FAD60970F9443BE27966CAF7DAF8EAF83
:10F560009FAF27972091E40A3091E50A4091E60A7F
:10F570005091E70A6091E00A7091E10A8091E20AF5
:10F580009091E30AACECBAE0BF93AF9327968CACB2
:10F590009DACAEACBFAC2797ECEECE2EEAE0DE2EF3
:10F5A000E12CF12C00EA10E40F9433050F94E21ED5
:10F5B000EAADFBAD85919591A591B4918093E00A58
:10F5C0009093E10AA093E20AB093E30AEAADFBAD9F
:10F5D000349685919591A591B4918093E40A909386
:10F5E000E50AA093E60AB093E70A64EE7AE080EEBB
:10F5F0009AE00E94104764966CAD7DAD8EAD9FADD4
:10F6000064970F9443BE4B015C01E090E80AF090D0
:10F61000E90A0091EA0A1091EB0A2091E40A30917C
:10F62000E50A4091E60A5091E70A6091E00A70917C
:10F63000E10A8091E20A9091E30AACECBAE0BF9350
:10F64000AF930F9433050F94E21E0F900F900F901D
:10F650000F902396FFAD2397FF2361F0211431040F
:10F6600049F020E030E040E85FE3C301B2010F94CD
:10F67000C7BC04C060E070E080E291EC20E030E0C4
:10F6800043E00E9430DE811108C0E091300BF0E0D1
:10F69000EE0FFF1FEE5BFC4B1FC0C090E80AD0903E
:10F6A000E90AE090EA0AF090EB0AA701960160E00F
:10F6B00070E080EA90E40F94C7BC2DEC3CEC4CEC7D
:10F6C0005DE30F94A1BD87FF0AC0E091300BF0E02D
:10F6D000EE0FFF1FE25CFC4B65907490ABC023966D
:10F6E0002FAD23972223B9F0A7019601C301B201E0
:10F6F0000F94C7BC9F7720E030E040E85FE30F94B1
:10F70000A4BF181644F4E091300BF0E0EE0FFF1F99
:10F71000EA5BFC4BE1CF6091691A70916A1A8091A3
:10F720006B1A90916C1A0E9475646B017C01E3EF77
:10F73000FCE08491882341F09091C00095FFFCCFBC
:10F740008093C6003196F5CF4091E80A5091E90ABE
:10F750006091EA0A7091EB0A25E030E08EE799E0CB
:10F760000E942843E9EEFCE08491882341F09091C7
:10F77000C00095FFFCCF8093C6003196F5CF25E001
:10F7800030E0B701A6018EE799E00E942843E8EE39
:10F79000FCE08491882341F09091C00095FFFCCF5C
:10F7A0008093C6003196F5CF8091C00085FFFCCFD5
:10F7B000FAE0F093C60087E02EAD3FAD829F800156
:10F7C000839F100D1124A8ADB9AD0A0F1B1F000FA8
:10F7D000111F000F111F09581D4EA70196016091BE
:10F7E000E80A7091E90A8091EA0A9091EB0A0F9475
:10F7F000C7BCF801618372838383948380911F0B5C
:10F800009091200B01979093200B80931F0BFFEF9B
:10F810002F1A3F0A81E00F94E5962AAD3BAD285F91
:10F820003F4F3BAF2AAF39E02316310409F035CE04
:10F83000612C712C80E090E0A0EAB0E48093E80AAB
:10F840009093E90AA093EA0AB093EB0A2091E40AA4
:10F850003091E50A4091E60A5091E70A6091E00A8A
:10F860007091E10A8091E20A9091E30AECECFAE0EF
:10F87000FF93EF9327968CAC9DACAEACBFAC2797B3
:10F88000ECEECE2EEAE0DE2EE12CF12C00EA10E4C4
:10F890000F9433050F94E21E0F900F9089E0281605
:10F8A000310421F060E0C3010C942D850E94BC431B
:10F8B000E5EDFCE08491882341F09091C00095FF34
:10F8C000FCCF8093C6003196F5CF8091C00085FFB4
:10F8D000FCCF8AE08093C6000E94ECF8E4ECFCE0E8
:10F8E0008491882341F09091C00095FFFCCF8093D4
:10F8F000C6003196F5CF8091C00085FFFCCF8AE02D
:10F900008093C60080EC9FE00F941FCAA82EDE01F2
:10F9100011963D01B12C32E5932E46E4842EBCE4D1
:10F92000B9839A828B8282E48C83F30181913F01B7
:10F930000E94E243882319F00E9405441DC0F1E0B3
:10F94000AF1235C1FB1528F0B11009C08FEB9FE055
:10F950000BC022E0B21206C08DEB9FE005C08EEB1B
:10F960009FE002C08CEB9FE00F941FCA682F77279F
:10F9700067FD7095872F972F61157105810591059A
:10F9800009F415C10F9443BE2FE632E143E85AE370
:10F990000F9476C06B017C019F7727E139ED4EEC27
:10F9A0005DE30F94A4BF18160CF037C0EBE2F0E152
:10F9B0008491882341F09091C00095FFFCCF809303
:10F9C000C6003196F5CFE0EAFCE08491882341F04F
:10F9D0009091C00095FFFCCF8093C6003196F5CF83
:10F9E00022E030E0B701A6018EE799E00E942843AB
:10F9F000E7E9FCE08491882341F09091C00095FFF5
:10FA0000FCCF8093C6003196F5CF8091C00085FF72
:10FA1000FCCF8AE08093C600CAC0F2E0BF1609F4AA
:10FA200069C023E0B21609F494C031E0B31689F13D
:10FA300020E030E040E05FE3C701B6010F9476C0FC
:10FA40001B012C0108E712E1A2019101D8011496D3
:10FA50006D917D918D919C9117970F94C8BCF80181
:10FA60006483758386839783A70196016081718182
:10FA7000828193810F94C8BCD8016D937D938D933F
:10FA80009C931397045E1F4FB2E10C3C1B07E1F6F9
:10FA90008EC020E030E040E05FE3C701B6010F9484
:10FAA00076C01B012C010CE712E1A2019101F801C3
:10FAB00060817181828193810F94C8BCD8016D935C
:10FAC0007D938D939C931397A701960114966D9146
:10FAD0007D918D919C9117970F94C8BCF801648318
:10FAE000758386839783045E1F4FF2E1003D1F07F5
:10FAF000E1F65DC020E030E040E05FE3C701B60121
:10FB00000F9476C01B012C0108E712E1A2019101BC
:10FB1000D8015C966D917D918D919C915F970F942A
:10FB2000C8BCF801648F758F868F978FA7019601E7
:10FB300060817181828193810F94C8BCD8016D93DB
:10FB40007D938D939D938D01B2E104381B07F1F6EF
:10FB50002EC020E030E040E05FE3C701B6010F9423
:10FB600076C01B012C0104E912E1A2019101F80108
:10FB700060817181828193810F94C8BCD8016D939B
:10FB80007D938D939D938D01A701960158966D915C
:10FB90007D918D919C915B970F94C8BCF801608F0B
:10FBA000718F828F938FF2E1003A1F07F1F6B394C1
:10FBB00024E0B212B4CEE6E7FCE08491882341F061
:10FBC0009091C00095FFFCCF8093C6003196F5CF91
:10FBD0008091C00085FFFCCF8AE08093C60087E754
:10FBE00092E10E94E9F9E4E6FCE08491882341F087
:10FBF0009091C00095FFFCCF8093C6003196F5CF61
:10FC00008091C00085FFFCCF8AE08093C60081E030
:10FC100080937712E8E4FCE08491882341F090918E
:10FC2000C00095FFFCCF8093C6003196F5CF809140
:10FC3000C00085FFFCCF8AE08093C6000E940FF2CF
:10FC4000E7E3FCE08491882341F09091C00095FFA8
:10FC5000FCCF8093C6003196F5CF8091C00085FF20
:10FC6000FCCF8AE08093C600E091CC0A34E0E39FA9
:10FC7000F0011124E159F54E20E030E042E053E478
:10FC800060817181828193810F94A4BF181694F4CE
:10FC900080915D0B882371F086EA9FE00F941FCA64
:10FCA000882341F08091751A9091761AC29714F0CA
:10FCB0000C94E79A81E090E09093160280931502ED
:10FCC00028968FAD28978093240B2A96AEADBFADB2
:10FCD0002A97B093220BA093210B2C96EEADFFAD8B
:10FCE0002C97F093200BE0931F0B1092320B109285
:10FCF000310B82E00F94E5960C940B9A8091771269
:10FD0000882309F49EC0EDE2FCE08491882341F051
:10FD10009091C00095FFFCCF8093C6003196F5CF3F
:10FD20004AE050E067E070E08EE799E00E943542DB
:10FD3000EBE2FCE08491882341F09091C00095FFB4
:10FD4000FCCF8093C6003196F5CF4AE050E067E0E3
:10FD500070E08EE799E00E943542E8E1FCE0849192
:10FD6000882341F09091C00095FFFCCF8093C6009E
:10FD70003196F5CF4AE050E065E070E08EE799E01B
:10FD80000E943542E6E0FCE08491882341F09091A6
:10FD9000C00095FFFCCF8093C6003196F5CF8091CF
:10FDA000C00085FFFCCF8AE08093C60000E010E031
:10FDB00093E0A92E9CE0B92E21E0822E2CE0922E19
:10FDC000E12CF12C9801215E3C4E6901F5018491F2
:10FDD000E3E0FCE0882349F09091C00095FFFCCF60
:10FDE0008093C60031968491F5CFF601EE0DFF1D8C
:10FDF000418152816381748125E030E08EE799E092
:10FE00000E942843F4E0EF0EF11C2CE1E216F1040D
:10FE1000E9F6F4018491E1E0FCE0882349F0909157
:10FE2000C00095FFFCCF8093C60031968491F5CF3A
:10FE30000C5111090C33FFEF1F0709F0C1CF0C94CF
:10FE40000B9AE3EEFBE08491882341F09091C0008F
:10FE500095FFFCCF8093C6003196F5CF8091C0000E
:10FE600085FFFCCF8AE08093C6000C940B9A81E05A
:10FE70000E9435480C940B9A1092960A0C940B9A97
:10FE800085E40E94E243811102C00F94E21E19E74B
:10FE9000612E15E0712E04ED802E0AE0902E80EE8A
:10FEA000A82E8AE0B82E512CD3018D913D010E94DD
:10FEB000E2438823D9F1B3E05B120CC00E944F44A7
:10FEC000F50160837183828393838CEE9AE00F94B3
:10FED0008C132CC00E944F44D4012D913D914D9123
:10FEE0005C910F94C8BCF501608371838283938316
:10FEF000E090E80AF090E90A0091EA0A1091EB0A12
:10FF00002091E40A3091E50A4091E60A5091E70A0F
:10FF10006091E00A7091E10A8091E20A9091E30A0F
:10FF2000BCEECB2EBAE0DB2E0F94E1115394F4E03B
:10FF30008F0E911C24E0A20EB11C34E05312B4CFFA
:10FF40000C940B9A81E08093921B0F94CAB4609337
:10FF5000660B7093670B8093680B9093690B6091AD
:10FF6000921B84EC9FE00F9431CA0C940B9A8DE4A1
:10FF70000E94E243882311F40C949198E091391087
:10FF8000F0913A10319681918032E9F38930D9F3BA
:10FF900080538A30B0F0E4EDFBE08491882341F097
:10FFA0009091C00095FFFCCF8093C6003196F5CFAD
:10FFB0008091C00085FFFCCF8AE08093C6000C943E
:10FFC0000B9A0E944F440F9410BE6B3C710511F4C4
:10FFD0000C94298D0CF0F7C06135710511F40C9467
:10FFE000A7880CF077C06A31710509F447C3D4F5CE
:10FFF0006431710509F4DDC294F46131710509F4CD
:020000021000EC
:10000000CCC234F46230710508F409C20C947C98B7
:100010006231710511F40C94D6880C947C98673188
:10002000710509F400C37CF46531710509F4F5C26A
:100030006631710511F00C947C988AE69BE00E9471
:10004000FCB70C940B9A6831710509F407C3693148
:10005000710511F00C947C988AE69BE00E9407B829
:100060000C940B9A6F31710509F419C48CF46C313E
:10007000710509F417C30CF40FC36D31710511F448
:100080000C940B9A6E31710509F43BC30C947C9867
:100090006C32710509F4AAC454F46032710509F494
:1000A00068C36A32710509F45AC40C947C986D32A5
:1000B000710509F4AAC46F32710511F00C947C9893
:1000C00084E090E090931602809315020F94B86B31
:1000D0000C940B9A6037710509F4BCC4A4F56C3517
:1000E000710511F40C942A89A4F46335710511F497
:1000F0000C94D18814F40C94CD886435710511F4F6
:100100000C94D6886535710511F40C940F890C9404
:100110007C986A36710509F4E4C754F468367105B1
:1001200009F47AC46936710509F4AAC40C947C9860
:100130006B36710511F40C94A1886D36710509F4C4
:10014000E8C50C947C986837710511F40C941F8BEA
:10015000C4F46237710511F40C94178A14F40C94EA
:10016000AD896337710511F40C94D7896737710530
:1001700011F00C947C98E0E2F2E4859194910C9457
:10018000308B6E3B710509F46EC65CF469377105FE
:1001900011F40C94248B6C38710509F460C40C9430
:1001A0007C98683C710511F40C94978C693C71053E
:1001B00011F00C947C9809E715E020E3E22E29E188
:1001C000F22E0C940E8D673F81E0780711F40C94A9
:1001D00054910CF07EC06C32A1E07A0711F40C94BB
:1001E000598FC4F5603D710511F40C94338EA4F45D
:1001F0006D3C710511F40C94688D14F40C94468DCB
:100200006E3C710511F40C94DF8D6F3C710511F497
:100210000C94FC8D0C947C986D3D710511F40C943C
:10022000CD8E64F4613D710511F40C945B8E6C3DD0
:10023000710511F40C94BC8E0C947C98623E71058F
:1002400011F40C94F78E603F710511F40C940B9A25
:100250000C947C986036E1E07E07E4F46E35F1E0C2
:100260007F0714F00C940B9A6E3221E0720711F4A0
:100270000C94FE9014F40C94918F6F3281E0780707
:1002800011F40C940D916033714011F40C945C9056
:100290000C947C98643FA1E07A0711F40C94469189
:1002A0004CF46039714011F00C947C980F94E21E6C
:1002B0000C940B9A653FF1E07F0711F40C944D917B
:1002C000663F714011F00C947C980E940B350C94A1
:1002D0000B9A6E3833E0730711F40C94BA960CF055
:1002E00047C06D3B92E0790711F40C940B98FCF435
:1002F0006835B2E07B0711F40C9466925CF46D3FB4
:10030000714011F00C947C980F94EA50E5E2F0E112
:100310000C946091693522E0720711F40C94759683
:100320006A35724011F40C9483960C947C9864386E
:1003300083E0780711F40C9491966CF46E3BA2E084
:100340007A0711F40C940E986335734011F40C94F1
:1003500072910C947C986B38E3E07E0711F40C9456
:1003600094966C38734011F40C940B9A0C947C980E
:10037000633923E0720711F40C942497D4F46039A4
:1003800083E0780711F40C94EF9614F40C94BD9666
:100390006139A3E07A0711F40C9421976239734014
:1003A00011F00C947C981092E81A0F94403C0C9435
:1003B0000B9A6639E3E07E0711F40C94D9976CF43C
:1003C000643923E0720711F40C942A97653973405D
:1003D00011F40C94A7970C947C98603A83E078070A
:1003E00009F430C2673E734011F00C947C9810926F
:1003F000800A0F948A518091251090912610A09127
:100400002710B09128108093291090932A10A09360
:100410002B10B0932C100E94B4550C940B9A0091A1
:10042000391010913A100E5F1F4F80E50E94E24391
:10043000882379F00E944F440F9415BE6B017C0114
:10044000BB24B394611571058105910531F4B12C7C
:1004500004C0B12CC12CD12C760183E50E94E2436B
:10046000882399F00E944F4420E030E04AE754E4AA
:100470000F9476C00F9415BE6B017C01AA24A3943F
:10048000611571058105910509F4A12C6AE270E0FE
:10049000C8010F9468C6009711F0DC011C92F801A6
:1004A000CF0121912032E1F3B11007C0A11005C0A6
:1004B000222319F00F944C5106C0E4E7F0E4859133
:1004C00094910F94595181E00F942C510F94E21E96
:1004D0000F94CAB46093920A7093930A8093940A1B
:1004E0009093950AC114D104E104F104F1F00F9442
:1004F000CAB44B015C018C0C9D1CAE1CBF1C84E07B
:1005000090E090931602809315020F94CAB4681578
:1005100079058A059B0510F00C94299B0F94DF52F6
:1005200081110C94299B0C94349B0F94DD528823E9
:1005300011F40C940B9A84E090E09093160280934F
:1005400015020F94DF52811109C00F94CE2B81E068
:100550000E94B05C80E00F94E596F3CF82E090E0DB
:10056000909316028093150280916C0BE091300BF2
:10057000F0E0EE0FFF1F882341F0E859FE4B859114
:1005800094910F9459510C940B9AEE5FFF4B859107
:1005900094910F9459510C940B9AE4EDF1E48591E8
:1005A00094910F94595117981698159814980C9483
:1005B0000B9AE8E1F3E485919491FC0124912223C4
:1005C00041F03091C00035FFFCCF2093C60001966A
:1005D000F4CF8091C00085FFFCCF8AE08093C600F5
:1005E0008AE69BE00E94D1B6E8ECF2E48591949112
:1005F000FC012491222341F03091C00035FFFCCF53
:100600002093C6000196F4CF8091C00085FFFCCFF7
:100610008AE08093C6000C940B9A8AE69BE00E94C5
:1006200027B70C940B9A8091391090913A106AE296
:1006300070E004960F9468C6009711F0DC011C92DC
:100640006091391070913A106C5F7F4F21E041E06A
:100650008AE69BE00E94AEBC0C940B9A8AE69BE073
:100660000E9400B80F94CAB460938A0A70938B0AF0
:1006700080938C0A90938D0A0C940B9A80916D0B49
:10068000882311F40C940B9A83E50E94E2438111B4
:100690000C943E9B0C940B9A8AE69BE00E94B2B9A4
:1006A0000C940B9A8091391090913A106AE270E0A4
:1006B00004960F9468C68C010097A9F080914310AE
:1006C000909144106EE470E0885B9F4E0F9468C672
:1006D00060E270E00F9468C6019690933A108093A0
:1006E0003910F80110826091391070913A106C5FE6
:1006F0007F4F21E040E08AE69BE00E94AEBC0C9474
:100700000B9A80916D0B882311F40C940B9A60E086
:100710008AE69BE00E943EBC8091391090913A108D
:100720006AE270E004960F9468C68C010097A9F005
:1007300080914310909144106EE470E0885B9F4E6E
:100740000F9468C660E270E00F9468C601969093BB
:100750003A1080933910D8011C9260913910709131
:100760003A106C5F7F4F8AE69BE00E9471B80C9450
:100770000B9A80916C0B81110F94E21E009139103D
:1007800010913A100C5F1F4F6AE270E0C8010F949D
:1007900068C67C0161E270E0C8010F9468C60097EA
:1007A00019F08C010F5F1F4FE114F10411F0F701F4
:1007B000108280E50E94E243F82E2091391030919A
:1007C0003A100217130708F4F12C80916D0B88235F
:1007D00011F40C940B9A21E02F2541E0B8018AE630
:1007E0009BE00E94AEBC83E50E94E2438823B9F0FF
:1007F0002091391030913A102017310780F40E946F
:100800000544AB01BC014093080E5093090E609360
:100810000A0E70930B0E83E59DE00E945AAA8AE6A9
:100820009BE00E9400B8F1100C940B9A0F94CAB48C
:1008300060938A0A70938B0A80938C0A90938D0A36
:100840000C940B9A8091391090913A106AE270E002
:1008500005960F9468C68C010097A9F0809143100B
:10086000909144106EE470E0885B9F4E0F9468C6D0
:1008700060E270E00F9468C6019690933A108093FE
:100880003910D8011C926091391070913A106B5F49
:100890007F4F8AE69BE00E94ECBF0C940B9A0F946A
:1008A000CAB46093860A7093870A8093880A9093EB
:1008B000890A00918A0A10918B0A20918C0A309142
:1008C0008D0A601B710B820B930B28EE33E040E026
:1008D00050E00F9478C2CA01B9012CE330E040E047
:1008E00050E00F9478C27F936F933F932F9385ECE2
:1008F0009BE09F938F93CE0101969F938F930F94CC
:10090000F3C7E5E2F0E184910FB6F894DEBF0FBEC5
:10091000CDBFE5E2F0E1882349F09091C00095FF5A
:10092000FCCF8093C60031968491F5CFFE013196BD
:100930008191882339F09091C00095FFFCCF80937E
:10094000C600F6CF8091C00085FFFCCF8AE080937F
:10095000C600CE0101960F944C510C940B9A83E57E
:100960000E94E243882311F40C940B9A0E944F4496
:100970000F9410BEF62EE72E862F9E2D8C0180E55B
:100980000E94E243882331F00F3F110509F010F473
:100990000C944F9B0DE010E0E1E4F5E08191919122
:1009A0008017910711F40C940B9A25E0E937F207B0
:1009B000A9F70630110539F48F2D9E2D9093CB0A9F
:1009C0008093CA0A04C017FF02C00C940B9A61E01E
:1009D000802F0F94B5B66F2D802F0F94EEB66F2D2C
:1009E0007E2D802F0F949DB50C940B9A8FEF0E9453
:1009F000354860E070E088EF9FE00F944BCA0E949A
:100A00009DDA0E9430DB0C940B9A8AE50E94E24347
:100A10000E946C520C940B9A88E690E00E946A5DEA
:100A200081110C940B9A83E50E94E243882371F0B4
:100A30000091810A0E944F4410E0000F111F0958D5
:100A4000154E0F9410BED8016D937C930F94D92846
:100A50000C940B9A63E08EEF98E00E943A5C83E579
:100A60000E94E243882311F40C940B9A0E944F4495
:100A70000F9410BE7093761A6093751A0C940B9AAB
:100A800089E690E00E946A5D81110C940B9AEFEB6D
:100A9000FBE08491882341F09091C00095FFFCCF4A
:100AA0008093C6003196F5CFE091810AB4E0EB9FC8
:100AB000F0011124E159F54E408151816281738129
:100AC00021E030E08EE799E00E942843ECEBFBE068
:100AD0008491882341F09091C00095FFFCCF8093D2
:100AE000C6003196F5CFE091810AF0E0EE0FFF1FCE
:100AF000E958F54E60817181882777FD8095982FA0
:100B00000F9443BEAB01BC0121E030E08EE799E0D9
:100B10000E942843E8EBFBE08491882341F0909108
:100B2000C00095FFFCCF8093C6003196F5CF409171
:100B30005D1A50915E1A60915F1A7091601A21E0FF
:100B400030E08EE799E00E942843E5EBFBE08491DA
:100B5000882341F09091C00095FFFCCF8093C600A0
:100B60003196F5CF6091751A7091761A882777FDC6
:100B70008095982F0F9443BEAB01BC0121E030E07B
:100B80008EE799E00E942843E2EBFBE08491882302
:100B900041F09091C00095FFFCCF8093C600319644
:100BA000F5CF4AE050E060E070E08EE799E00E9407
:100BB0003542E0EBFBE08491882341F09091C00046
:100BC00095FFFCCF8093C6003196F5CF40916F1A08
:100BD0005091701A6091711A7091721A21E030E090
:100BE0008EE799E00E942843EDEAFBE08491882398
:100BF00041F09091C00095FFFCCF8093C6003196E4
:100C0000F5CF6091771A7091781A882777FD8095D3
:100C1000982F0F9443BEAB01BC0121E030E08EE77A
:100C200099E00E942843E9EAFBE08491882341F09F
:100C30009091C00095FFFCCF8093C6003196F5CF10
:100C40008091810A90E00F945A264AE050E0BC015E
:100C50008EE799E00E943542E4EAFBE08491882324
:100C600041F09091C00095FFFCCF8093C600319673
:100C7000F5CF8FEF9FEF0F945A264AE050E0BC016A
:100C80008EE799E00E943542E0EAFBE084918823F8
:100C900041F09091C00095FFFCCF8093C600319643
:100CA000F5CF4091691A50916A1A60916B1A709150
:100CB0006C1A21E030E08EE799E00E942843ECE9CD
:100CC000FBE08491882341F09091C00095FFFCCF18
:100CD0008093C6003196F5CF4091631A5091641A03
:100CE0006091651A7091661A21E030E08EE799E014
:100CF0000E9428438091C00085FFFCCF8AE080934A
:100D0000C60081E090E090931602809315020C9447
:100D1000759B8DE690E00E946A5D81110C940B9AA0
:100D2000E091300BF0E0EE0FFF1FE059FD4B859195
:100D300094910F94595181E090E09093280B809307
:100D4000270B8091921B882321F081E090E00F9483
:100D5000DA6083E50E94E243882391F00091810AE2
:100D60000E944F4410E0000F111F0958154E0F94B8
:100D700010BEF8017183608381E08093060215C084
:100D800082E50E94E243882381F00091810A0E945B
:100D90004F4410E0000F111F0958154E0F9410BE5C
:100DA000D8016D937C93109206020F94D9280F946A
:100DB000CAB46B017C010091810A10E0F801EE0FCA
:100DC000FF1FE958F54E60817181882777FD809576
:100DD000982F0F9443BEF801EE0FFF1FEE0FFF1F79
:100DE000E159F54E11E020813181428153810F9408
:100DF000A4BF18160CF010E010937F0A81E090E079
:100E000090931602809315021092BB0AC701B60197
:100E10000E94F35EE091300BF0E0EE0FFF1FE4590B
:100E2000FD4B859194910F94595182E090E09093FD
:100E30001602809315029093280B8093270B8091C4
:100E4000921B882321F082E090E00F94DA600F94E7
:100E5000CAB46093920A7093930A8093940A909311
:100E6000950A0C940B9AE091300BF0E0EE0FFF1F07
:100E7000E65BFC4B859194910F94595183E090E08F
:100E80009093280B8093270B8091921B882321F04D
:100E900081E090E00F94DA6083E50E94E2438823CA
:100EA00061F00E944F440F9410BE7093761A6093C5
:100EB000751A81E0809306020FC082E50E94E2432A
:100EC000882351F00E944F440F9410BE7093761AFD
:100ED0006093751A109206020F94CAB44B015C011C
:100EE0001092BB0A6091751A7091761A882777FD67
:100EF0008095982F0F9443BE11E020915D1A309198
:100F00005E1A40915F1A5091601A0F94A4BF181690
:100F10000CF010E010937F0A81E090E090931602AD
:100F20008093150209E91BE075E9E72E7BE0F72EB7
:100F3000E1E9CE2EEBE0DE2EFAE07F2E80917F0AF3
:100F40006091751A7091761A882309F490C0809187
:100F5000BB0A81118CC0882777FD8095982F0F944C
:100F600043BE20915D1A30915E1A40915F1A5091F4
:100F7000601A0F94A4BF18160CF090C00F94CAB456
:100F8000681979098A099B09693E734081059105B1
:100F900008F464C08091921B81115CC0E091CC0A7E
:100FA00024E0E29FF0011124E159F54E4081518186
:100FB00062817381F8018491E9E9FBE0882349F0BB
:100FC0009091C00095FFFCCF8093C600319684912C
:100FD000F5CF22E030E08EE799E00E942843F70148
:100FE0008491E5E9FBE0882349F09091C00095FFEA
:100FF000FCCF8093C60031968491F5CF6091CC0AE6
:1010000070E04AE050E08EE799E00E943542F60138
:101010008491E1E9FBE0882349F09091C00095FFBD
:10102000FCCF8093C60031968491F5CF40915D1A34
:1010300050915E1A60915F1A7091601A21E030E061
:101040008EE799E00E9428438091C00085FFFCCF85
:101050007092C6000F94CAB44B015C010F94CE2B62
:1010600080E00E94B05C80E00F94E59667CF88270F
:1010700077FD8095982F0F9443BE20915D1A309193
:101080005E1A40915F1A5091601A0F94A1BD87FFBC
:1010900005C080910602882309F470CFE091300BDF
:1010A000F0E0EE0FFF1FE25BFC4B859194910F94F3
:1010B000595182E090E0909316028093150284E0EB
:1010C00090E09093280B8093270B0F94CAB4609301
:1010D000920A7093930A8093940A9093950A0C94C1
:1010E0000B9A83E50E94E243882319F10E944F4442
:1010F00020E030E0A9010F94A1BD87FD0FC00E9440
:101100004F4420E030E04FE753E40F94A4BF18169B
:1011100044F00E944F440F9410BE05C060E070E0A0
:1011200002C06FEF70E07093CB0A6093CA0A0C9410
:101130000B9A8FEF90E09093CB0A8093CA0A0C949D
:101140000B9A1092CB0A1092CA0A0C940B9A0F9425
:10115000DA280F94E21E149A0F94641F1092CB0A9F
:101160001092CA0A68EE73E080E090E00F94F9B440
:1011700010921702E2EDF1E4459154912FE83BE023
:101180006DE87BE081EA94E00E94CACB0F9459514C
:1011900080E00F94E5960C940B9A1092650B0C94DA
:1011A0000B9A81E08093650B0C940B9A83E50E9467
:1011B000E243882399F00E944F4420E030E04AE760
:1011C00054E40F9476C00F9415BE60930802709398
:1011D000090280930A0290930B021DC088E50E94C9
:1011E000E24381110C94569B89E50E94E2438111F0
:1011F0000C94569B8AE50E94E24381110C94569B05
:1012000085E40E94E24381110C94569B0F94E21EE8
:10121000149A0F94641F10921E0B0C940B9A83E582
:101220000E94E243882311F40C940B9A0E944F44CD
:1012300020E030E04AE754E40F9476C00F9415BEE6
:1012400060938E0A70938F0A8093900A9093910A0C
:101250000C940B9A29E735E039AF28AF00E419E187
:1012600040E5C42E49E1D42E50E0E52E59E1F52E9B
:10127000312CA8ADB9AD8D91B9AFA8AF0E94E243B2
:10128000882309F45CC0B3E03B1252C00E944F4473
:101290002B013C0120E030E040EA51E40F94A1BD75
:1012A00087FF3FC0A3019201F801608171818281B3
:1012B00093810F94A8BD4B015C019B01AC0160912F
:1012C00020197091211980912219909123190F945E
:1012D00076C06093201970932119809322199093FE
:1012E0002319A5019401D6016D917D918D919C9159
:1012F0000F9476C0F6016083718382839383D70154
:101300006D917D918D919C910F9441BEA5019401A9
:101310000F9476C00F9415BEF701608371838283AA
:101320009383D8014D925D926D927C92139707C082
:101330000E944F44F80160837183828393833394C6
:101340000C5F1F4FF4E0CF0ED11C24E0E20EF11C25
:1013500034E033128ECF0C940B9A83E50E94E24363
:10136000882331F00E94F843809310020C940B9A6A
:10137000E5E2F0E18491882341F09091C00095FF6F
:10138000FCCF8093C6003196F5CF4091100250E01B
:1013900060E070E086E89BE00E944C488091C000CD
:1013A00085FFFCCF8AE08093C6000C940B9A86E5FB
:1013B0000E94E2438823B9F00F940DB1FC012491FF
:1013C000222341F03091C00035FFFCCF2093C600AE
:1013D0000196F4CF8091C00085FFFCCF8AE0809316
:1013E000C6000C940B9A85E50E94E243882369F0BD
:1013F0008091391090913A10019690933A10809311
:1014000039100F947EB30C940B9AE6E2F2E48591C6
:101410009491FC012491222311F40C940B9A3091A5
:10142000C00035FFFCCF2093C6000196F2CFE3E861
:10143000FBE08491882341F09091C00095FFFCCFA0
:101440008093C6003196F5CF4091E00A5091E10AB1
:101450006091E20A7091E30A22E030E08EE799E0C1
:101460000E942843EFE7FBE08491882341F09091AC
:10147000C00095FFFCCF8093C6003196F5CF409118
:10148000E40A5091E50A6091E60A7091E70A22E0C9
:1014900030E08EE799E00E942843EBE7FBE084917F
:1014A000882341F09091C00095FFFCCF8093C60047
:1014B0003196F5CF4091E80A5091E90A6091EA0A25
:1014C0007091EB0A22E030E08EE799E00E94284319
:1014D000E7E7FBE08491882341F09091C00095FFFD
:1014E000FCCF8093C6003196F5CF4091EC0A509125
:1014F000ED0A6091EE0A7091EF0A22E030E08EE78B
:1015000099E00E942843E6EEF2E485919491FC0173
:101510002491222341F03091C00035FFFCCF20936D
:10152000C6000196F4CF80E00F94431F0F9443BE92
:10153000209140193091411940914219509143191D
:101540000F94A8BDAB01BC0122E030E08EE799E02A
:101550000E942843E3E7FBE08491882341F09091C7
:10156000C00095FFFCCF8093C6003196F5CF81E097
:101570000F94431F0F9443BE209144193091451995
:1015800040914619509147190F94A8BDAB01BC0179
:1015900022E030E08EE799E00E942843EFE6FBE08E
:1015A0008491882341F09091C00095FFFCCF8093F7
:1015B000C6003196F5CF82E00F94431F0F9443BECF
:1015C000209148193091491940914A1950914B196D
:1015D0000F94A8BDAB01BC0122E030E08EE799E09A
:1015E0000E942843EBE6FBE08491882341F0909130
:1015F000C00095FFFCCF8093C6003196F5CF83E005
:101600000F94431F0F9443BE20914C1930914D19F4
:1016100040914E1950914F190F94A8BDAB01BC01D8
:1016200022E030E08EE799E00E9428438091C000DC
:1016300085FFFCCF8AE08093C6000C940B9A80E073
:101640000F9467150C940B9A81E00F9467150C9416
:101650000B9A3091C00035FFFCCF2093C600019655
:10166000FC0124912111F5CF8091C00085FFFCCFB2
:101670008AE08093C600E8E1F0E485919491FC0152
:101680002491222341F03091C00035FFFCCF2093FC
:10169000C6000196F4CF1E9B10C0ECECF2E48591DD
:1016A0009491FC0124912223C1F03091C00035FFB8
:1016B000FCCF2093C6000196F4CFEAECF2E48591CA
:1016C0009491FC012491222341F03091C00035FF18
:1016D000FCCF2093C6000196F4CF8091C00085FF17
:1016E000FCCF8AE08093C600EAE1F0E48591949112
:1016F000FC012491222341F03091C00035FFFCCF42
:101700002093C6000196F4CF8091060182FF10C09D
:10171000ECECF2E485919491FC0124912223C1F038
:101720003091C00035FFFCCF2093C6000196F4CF66
:10173000EAECF2E485919491FC012491222341F09A
:101740003091C00035FFFCCF2093C6000196F4CF46
:101750008091C00085FFFCCF8AE08093C600ECE05A
:10176000F0E485919491FC012491222341F0309181
:10177000C00035FFFCCF2093C6000196F4CF1D9B1F
:1017800010C0ECECF2E485919491FC0124912223A9
:10179000C1F03091C00035FFFCCF2093C600019608
:1017A000F4CFEAECF2E485919491FC012491222398
:1017B00041F03091C00035FFFCCF2093C600019668
:1017C000F4CF8091C00085FFFCCF8AE08093C600F3
:1017D000EEE0F0E485919491FC012491222341F004
:1017E0003091C00035FFFCCF2093C6000196F4CFA6
:1017F0008091060187FF10C0ECECF2E48591949192
:10180000FC0124912223C1F03091C00035FFFCCFB0
:101810002093C6000196F4CFEAECF2E4859194910E
:10182000FC012491222341F03091C00035FFFCCF10
:101830002093C6000196F4CF8091C00085FFFCCFB5
:101840008AE08093C600E6E0F0E485919491FC0183
:101850002491222341F03091C00035FFFCCF20932A
:10186000C6000196F4CF1C9B10C0ECECF2E485910D
:101870009491FC0124912223C1F03091C00035FFE6
:10188000FCCF2093C6000196F4CFEAECF2E48591F8
:101890009491FC012491222341F03091C00035FF46
:1018A000FCCF2093C6000196F4CF8091C00085FF45
:1018B000FCCF8AE08093C600E8E0F0E48591949143
:1018C000FC012491222341F03091C00035FFFCCF70
:1018D0002093C6000196F4CF019910C0ECECF2E41D
:1018E00085919491FC0124912223C1F03091C00094
:1018F00035FFFCCF2093C6000196F4CFEAECF2E46A
:1019000085919491FC012491222341F03091C000F3
:1019100035FFFCCF2093C6000196F4CF8091C00024
:1019200085FFFCCF8AE08093C6000C940B9A8091CF
:10193000CC0A8093810A84E50E94E243882329F13E
:101940000E944F440F9415BE6093810A6623E9F00C
:10195000E5E2F0E18491882341F09091C00095FF89
:10196000FCCF8093C6003196F5CFEEE1F2E4A5916D
:10197000B4918D91882311F40C940B9A9091C0002E
:1019800095FFFCCF8093C600F4CF84E40E94E2432D
:10199000882311F40C940B9A0E944F4420E030E00D
:1019A000A9010F94A1BD811103C01092F00A32C0A9
:1019B0000091810A10E00E944F44F801EE0FFF1FD2
:1019C000EE0FFF1FEC5BFD4F608371838283938377
:1019D000E0904402F09045020091460210914702C7
:1019E00020E030E0A901B701C8010F94A1BD811129
:1019F00004C0E12CF12C00E410E4C701D80180936D
:101A0000440290934502A0934602B093470281E0BE
:101A10008093F00A0E94BF5E0C940B9AD8018D91BE
:101A20008D010E94E243882349F00E944F440F94A5
:101A300015BEF7016083718382839383F4E0EF0E18
:101A4000F11C25E00D37120749F70F94BE130C94D3
:101A50000B9A09E715E090E5E92E99E1F92ED801F6
:101A60008D918D010E94E243882339F00E944F44FA
:101A7000F7016083718382839383F4E0EF0EF11C9E
:101A800025E00D37120759F70C940B9A83E50E9455
:101A9000E243882351F00E944F44609328197093C9
:101AA000291980932A1990932B1984E50E94E24307
:101AB000882311F40C940B9A0E944F4460932419CC
:101AC0007093251980932619909327190C940B9ADB
:101AD00083E50E94E243882351F00E944F446093C3
:101AE0002C1970932D1980932E1990932F1984E53A
:101AF0000E94E243882351F00E944F4460931019E2
:101B000070931119809312199093131982E40E9413
:101B1000E243882361F00E944F440F9415BE609306
:101B2000601970936119809362199093631988E525
:101B30000E94E243882391F00E944F446093181959
:101B40007093191980931A1990931B1960931419A3
:101B500070931519809316199093171989E50E94AF
:101B6000E243882351F00E944F4460931819709308
:101B7000191980931A1990931B198AE50E94E24360
:101B8000882351F00E944F4460931C1970931D19D3
:101B900080931E1990931F1985E40E94E2438823C5
:101BA00011F40C940B9A0E944F4460932019709387
:101BB000211980932219909323190C940B9A09E709
:101BC00015E084EDE82E8AE0F82ED8018D918D0184
:101BD0000E94E243882339F00E944F44F70160835A
:101BE000718382839383F4E0EF0EF11C25E00C37C0
:101BF000120759F70C940B9A83E50E94E24388235D
:101C000051F00E944F446093240270932502809308
